:100000000C94E92A0D94650A0D943A0A0D940F0A8E
:100010000D94E4090D94B9090D948E090D946309AA
:100020000C9405B50C941A2B0C941A2B0C941A2BC7
:100030000C941A2B0C9449990C941A2B0C941A2B8F
:100040000C941A2B0C9484AD0C941A2B0C941A2B30
:100050000C941A2B0C941A2B0C94E9AB0D94900A67
:100060000C941A2B0C944BB40C941A2B0C941A2B42
:100070000C941A2B0C941A2B0C941A2B0C941A2BEC
:100080000C941A2B0C941A2B0C941A2B0C941A2BDC
:100090000C941A2B0C941A2B0C941A2B0C941A2BCC
:1000A0000C941A2B0C941A2B0C941A2B0C941A2BBC
:1000B0000C941A2B0C941A2B0C941A2B0C941A2BAC
:1000C0000C941A2B0C941A2B0C941A2B0C941A2B9C
:1000D0000C941A2B0C941A2B0C941A2B0C941A2B8C
:1000E0000C941A2B2C432F431E4322432843664370
:1000F000334337433D43414345434B434F435343CE
:10010000664359435D436143586C586C5F6C5F6C48
:100110005F6C666C666C666C736C6D6C6D6C6D6C34
:100120004E905390589062906C90E59076907E90AF
:10013000869090909A90A490B390BD90E590C790CF
:10014000D190DB907FB485B496B4A1B4A9B4BEB409
:10015000ADB4BEB4B1B4B5B4BEB4BBB4084AD73BB9
:100160003BCE016E84BCBFFDC12F3D6C74319ABD86
:1001700056833DDA3D00C77F11BED9E4BB4C3E91AA
:100180006BAAAABE000000803F05A84CCDB2D44E99
:10019000B93836A9020C50B9918688083CA6AAAA9B
:1001A0002ABE000000803F000D9459130D941312D5
:1001B0000D945A010D94C2070D94CD0520746F6FF4
:1001C000206C6F6E6720657874727573696F6E202E
:1001D00070726576656E7465640A0020636F6C6486
:1001E00020657874727573696F6E207072657665BC
:1001F0006E7465640A0047322F47332062616420C1
:10020000706172616D65746572730A00536C656527
:10021000702E2E2E00205A3A200020593A200042FB
:10022000656420583A20004C756C7A426F742054F3
:10023000415A20362072656164792E0052657375CB
:100240006D696E67207072696E7400436C69636BD0
:1002500020746F20726573756D652E2E2E004E6FA3
:10026000206D6F76652E00456E642066696C652092
:100270006C6973740A00426567696E2066696C6513
:10028000206C6973740A004D31323500534420707C
:1002900072696E74696E67206279746520004E6FB2
:1002A00074205344207072696E74696E670A004648
:1002B000696C652064656C657465643A0044656CBE
:1002C0006574696F6E206661696C65642C2046698F
:1002D0006C653A20006F70656E206661696C6564BC
:1002E0002C2046696C653A20002569730025696DEC
:1002F00020256973002569682025696D20256973AB
:1003000000256964202569682025696D20256973A9
:100310000025697920256964202569682025696D93
:1003200020256973005072696E742074696D653A96
:100330002000000125301D0C1824311C0B17232F21
:100340001B0A1E16040308060202222B1A4142034E
:100350003809FF3628294527444350726F74656376
:100360007465642050696E0A00457874727564651E
:1003700072202573004C756C7A426F742054415A78
:1003800020362072656164792E006F6B00436F6FB9
:100390006C696E6720646F6E652E004865617469D4
:1003A0006E6720646F6E652E0020573A00457874A2
:1003B0007275646572202573004C756C7A426F7497
:1003C0002054415A20362072656164792E004265BE
:1003D0006420646F6E652E0020573A0042656420E9
:1003E00068656174696E672E0042656420636F6F93
:1003F0006C696E672E004C756C7A426F74205441A4
:100400005A2036204F66662E004361703A454D45AE
:100410005247454E43595F5041525345523A310A73
:10042000004361703A434153455F4C494748545F2C
:100430004252494748544E4553533A300A004361AB
:10044000703A544F47474C455F4C49474854533ADC
:10045000300A004361703A534F4654574152455F4A
:10046000504F5745523A300A004361703A4C455656
:10047000454C494E475F444154413A310A0043617B
:10048000703A5A5F50524F42453A310A0043617008
:100490003A4155544F4C4556454C3A310A00436158
:1004A000703A5052494E545F4A4F423A310A004323
:1004B00061703A50524F47524553533A300A004305
:1004C00061703A4155544F5245504F52545F544514
:1004D0004D503A310A004361703A454550524F4DF4
:1004E0003A310A004649524D574152455F4E414DFF
:1004F000453A4D61726C696E20204649524D574114
:1005000052455F56455253494F4E3A312E312E35A2
:100510002E34342045585452554445525F54595056
:10052000453A4D4F41527374727564657220534F52
:10053000555243455F434F44455F55524C3A6874AA
:100540007470733A2F2F636F64652E616C657068E9
:100550006F626A656374732E636F6D2F646966667C
:100560007573696F6E2F4D41524C494E2050524F5A
:10057000544F434F4C5F56455253494F4E3A312EDC
:1005800030204D414348494E455F545950453A4CFF
:10059000756C7A426F742054415A20362045585465
:1005A00052554445525F434F554E543A31205555AC
:1005B00049443A38343566303033632D61656264BE
:1005C0002D346535332D613662392D376430393835
:1005D000346664653630390A007A5F70726F62651E
:1005E0003A20007A5F6D61783A20007A5F6D696E1B
:1005F0003A2000795F6D61783A2000795F6D696E0D
:100600003A2000785F6D61783A2000785F6D696EFE
:100610003A20005265706F7274696E6720656E646F
:1006200073746F70207374617475730A0043290AC0
:100630000061626C656420286D696E2074656D7060
:100640002000436F6C642065787472756465732054
:100650006172652000426564204C6576656C696E48
:100660006720004661696C656420746F20656E6167
:10067000626C6520426564204C6576656C696E67C6
:100680000A00426564204C6576656C20436F727287
:10069000656374696F6E204D61747269783A000009
:1006A00000A0C100809743000000004F666673659C
:1006B0007473206170706C696564004572723A20D1
:1006C000546F6F206661722100546F6F20666172F3
:1006D0002066726F6D207265666572656E63652057
:1006E000706F696E740A004E6F2063617365206CD1
:1006F000696768740A004163746976652045787497
:1007000072756465723A2000556E6B6E6F776E205D
:10071000636F6D6D616E643A202200434F4D4D55FD
:100720004E49434154494F4E0044525952554E0090
:100730004552524F525300494E464F004543484F91
:10074000001000C90210012C0140012201700118A3
:1007500001B0010E01F00104015002FA00B002F0F4
:10076000003003E600D003DC009004D2007005C81E
:1007700000A006BE000008B400B009AA00D00BA07B
:1007800000600E960060118C000015820020197820
:1007900000C01D6E00A0226400B0275A00902C50AB
:1007A0000000314600E0343C0010383200903A2816
:1007B00000603C1E00A03D1400803E0A00203F0067
:1007C00000000020002300260029002C002F00320A
:1007D00000000100000301060109010000A0C100A2
:1007E00000A0C1000000000000914300809743007A
:1007F0000087432F2F20004D31343520533C696E44
:100800006465783E206F7574206F662072616E6734
:10081000652028302D31290A003C07370730072989
:10082000071B076F66660044454255473A00207033
:100830006F736974696F6E206F7574206F662072B4
:10084000616E67652E0A003F50726F62652000205E
:10085000496E76616C69642065787472756465723E
:10086000200020643A0020693A0020703A00205AA3
:1008700000205900580020204D61783A2000205A6D
:1008800000205900580020204D696E3A20004F6E1C
:1008900020004F666600536F667420656E64737443
:1008A0006F70733A200020643A0020693A0020708B
:1008B0003A0053657474696E672054726176656C92
:1008C00020416363656C65726174696F6E3A2000E4
:1008D00053657474696E6720526574726163742025
:1008E000416363656C65726174696F6E3A20005391
:1008F000657474696E67205072696E742041636319
:10090000656C65726174696F6E3A2000536574742A
:10091000696E67205072696E7420616E6420547233
:100920006176656C20416363656C65726174696FA3
:100930006E3A200020204D383531205A005A2D5073
:10094000726F6265204F666673657420286D6D292D
:100950003A0A0020440020490020204D3330342042
:10096000500020440020490020204D3330312050D9
:10097000005049442073657474696E67733A0A00C5
:1009800020460020420020480020204D31343520F0
:1009900053004D6174657269616C2068656174759E
:1009A0007020706172616D65746572733A0A00201F
:1009B000204D3432302053004175746F20426564FD
:1009C000204C6576656C696E673A0A00205A0020F3
:1009D000590020204D323036205800486F6D652078
:1009E0006F66667365743A0A00204500205A00203D
:1009F000590020580020420020540020204D323061
:100A000035205300416476616E6365643A20533C3F
:100A10006D696E5F66656564726174653E20543C05
:100A20006D696E5F74726176656C5F666565647230
:100A30006174653E20423C6D696E5F7365676D65EC
:100A40006E745F74696D655F6D733E20583C6D61B7
:100A5000785F78795F6A65726B3E205A3C6D617889
:100A60005F7A5F6A65726B3E20453C6D61785F65B9
:100A70005F6A65726B3E0A002054002052002020FD
:100A80004D323034205000416363656C657261748F
:100A9000696F6E2028756E6974732F7332293A203E
:100AA000503C7072696E745F616363656C3E205286
:100AB0003C726574726163745F616363656C3E2050
:100AC000543C74726176656C5F616363656C3E0A69
:100AD00000204500205A0020590020204D3230319E
:100AE0002058004D6178696D756D20416363656CB8
:100AF00065726174696F6E2028756E6974732F73E7
:100B000032293A0A00204500205A002059002020AE
:100B10004D3230332058004D6178696D756D206617
:100B200065656472617465732028756E6974732FCE
:100B300073293A0A00204500205A0020590020203D
:100B40004D393220580053746570732070657220DF
:100B5000756E69743A0A0020204D323030204430DE
:100B60000A0020204D323030204400204469736157
:100B7000626C65640A0046696C616D656E74207311
:100B8000657474696E67733A0020204D31343920E2
:100B900043203B20556E69747320696E2043656C59
:100BA000736975730A002020473231202020203BD2
:100BB00020556E69747320696E206D6D0A003A20AD
:100BC000007A5F6D696E3A20202D32207A5F6D6168
:100BD000783A202035005A204F66667365742000ED
:100BE0004578747275646572004D6F7665205A00A1
:100BF0004D6F76652059004D6F76652058004D6F1A
:100C000076656D656E74004D6F766520302E316DA2
:100C10006D004D6F766520316D6D004D6F766520EE
:100C200031306D6D004D6F766520617869730045D8
:100C300078747275646572004D6F7665205A004D48
:100C40006F76652059004D6F76652058005344201B
:100C500063617264206F6B0A006F70656E526F6F14
:100C600074206661696C65640A00766F6C756D65E9
:100C70002E696E6974206661696C65640A0053446C
:100C800020696E6974206661696C0A007C3C3E5E76
:100C90002B3D3F2F5B5D3B2C2A225C0043616E6E37
:100CA0006F74206F70656E207375626469722000C6
:100CB000656E7175657565696E6720220045727293
:100CC0006F722077726974696E6720746F20454572
:100CD00050524F4D210A00486F6D652025732573D2
:100CE0002573206669727374002066697273740AD2
:100CF000005A0059005800486F6D6520004361722A
:100D0000642072656D6F766564004361726420696A
:100D10006E7365727465640048617264636F6465C4
:100D2000642044656661756C742053657474696EE3
:100D30006773204C6F616465640A002823000028F3
:100D4000230000640000001027000000009643000C
:100D5000009643000040400000C8410000C9420026
:100D600000C9420000C84400804F44202863616CE1
:100D700063756C6174656429210A0020213D20009F
:100D8000454550524F4D20435243206D69736D616C
:100D9000746368202D202873746F726564292000A5
:100DA000290A002062797465733B20637263200016
:100DB0002073746F7265642073657474696E6773F1
:100DC00020726574726965766564202800204D6123
:100DD000726C696E3D563430290A002845455052E0
:100DE0004F4D3D00454550524F4D20766572736919
:100DF0006F6E206D69736D6174636820001000ADC3
:100E00000330016A0150022B0170030A019004F5BE
:100E100000B005E500D006D800F007CE001009C5E7
:100E200000300ABE00500BB700700CB100900DAB43
:100E300000B00EA600D00FA200F0109D0010129975
:100E400000301395005014920070158E0090168B90
:100E500000B0178700D0188400F0198100101B7EA5
:100E600000301C7B00501D7900701E7600901F73AF
:100E700000B0207000D0216E00F0226B00102469B9
:100E80000030256600502663007027610090285EC0
:100E900000B0295C00D02A5900F02B5600102D54C8
:100EA00000302E5100502F4E0070304B00903148D2
:100EB00000B0324500D0334200F0343E0010363BE3
:100EC00000303737005038330070392E00903A29FF
:100ED00000B03B2300D03C1B00F03D1100103F014F
:100EE00000F03F000000060900FE06018902FE2016
:100EF000FFFE07FE06FE00000006000701060606CC
:100F00000200808080800080030303060103A0A00C
:100F1000A00507070600FF5050F850F8505005098B
:100F2000090600FE2070A8A07028A87020060808F6
:100F30000600FF40A848102048540805070706008F
:100F4000FF60909060989068010303060203808020
:100F5000800207070602FF408080808080400207F1
:100F6000070602FF8040404040408005050506001E
:100F7000008850F850880505050600002020F8205C
:100F8000200204040602FEC0404080050101060064
:100F900002F8020202060200C0C0040606060100B2
:100FA000101020408080040606060100609090909A
:100FB000906003060606010040C0404040E0040681
:100FC000060601006090102040F0040606060100AD
:100FD000F020601010E0050606060000103050906A
:100FE000F810040606060100F080E01010E0040688
:100FF000060601006080E09090600406060601008D
:10100000F010102040400406060601006090609039
:101010009060040606060100609090701060020562
:1010200005060200C0C000C0C00207070602FEC0DD
:10103000C000C040408005050506000018608060C3
:1010400018050303060001F800F805050506000071
:10105000C0300830C00407070601006090106040EF
:1010600000400506060600007090A8B080700506D6
:1010700006060000205088F888880506060600004D
:10108000F088F08888F004060606010060908080F1
:101090009060040606060100E090909090E004063F
:1010A00006060100F080E08080F0040606060100DC
:1010B000F080E0808080040606060100609080B029
:1010C00090600406060601009090F0909090030650
:1010D00006060100E040404040E00506060600002C
:1010E00038101010906004060606010090A0C0A001
:1010F00090900406060601008080808080F005063E
:101100000606000088D8A8A88888040606060100FC
:1011100090D0B090909005060606000070888888F0
:101120008870040606060100E09090E080800407C5
:10113000070601FF609090D0B0601004060606011B
:1011400000E09090E0909004060606010060904058
:10115000209060050606060000F8202020202004CC
:101160000606060100909090909060040606060125
:1011700000909090F060600506060600008888A840
:10118000A8D888050606060000885020205088054B
:101190000606060000888850202020040606060166
:1011A00000F010204080F0030606060100E0808079
:1011B0008080E004060606010080804020101003B5
:1011C0000606060100E020202020E00503030600BB
:1011D000032050880501010600FEF8020202060203
:1011E0000480400404040601007090907004060618
:1011F0000601008080E09090E00404040601007085
:101200008080700406060601001010709090700433
:10121000040406010060B0C0700406060601002048
:101220005040E040400406060601FE6090907010B9
:10123000600406060601008080E090909003060698
:101240000601004000C04040E00308080601FE20FF
:101250000060202020A0400406060601008080A037
:10126000C0A090030606060100C040404040E005D3
:101270000404060000D0A8A888040404060100E0C5
:1012800090909004040406010060909060040606AB
:101290000601FEE09090E080800406060601FE70E4
:1012A0009090701010040404060100A0D080800407
:1012B000040406010070C030E00406060601004088
:1012C00040E0405020040404060100909090700417
:1012D0000404060100909060600504040600008884
:1012E000A8A850040404060100906060900406065B
:1012F0000601FE909090709060040404060100F0D6
:101300002040F003070706010020404080404020B5
:101310000107070602FF8080808080808003070726
:101320000601008040402040408004020206010384
:1013300050A0FFFFFFFFFFFFFFFFFFFFFFFFFFFFCB
:10134000FFFFFFFFFFFFFFFFFFFFFFFFFFFFFFFFAD
:10135000FFFFFF00000006000701060606020080EE
:1013600000808080800406060601FF2070A0A07027
:10137000200507070600FF304840F04040F805050B
:1013800005060000A8508850A8050606060000883B
:1013900050F820F8200107070602FF8080800080B7
:1013A00080800407070601FF708060906010E003F2
:1013B0000101060105A0060707060000788494A431
:1013C00094847803050506010160A06000E005052E
:1013D000050600002850A05028040303060100F071
:1013E0001010040101060102F0060707060000784C
:1013F00084B4A4A48478040101060105F004030365
:101400000601026090600507070600FF2020F82013
:101410002000F803050506010140A02040E0030577
:1014200005060101C0204020C0020202060204405D
:10143000800405050601FF9090B0D08005060606E1
:10144000000078E8E868282801010106020280020D
:1014500002020602FE408003050506010140C0406D
:1014600040E003050506010140A04000E005050538
:10147000060000A0502850A00508080600FF40C044
:101480004050703078100508080600FF40C04050FA
:10149000680810380508080600FFC0204030F0300A
:1014A0007810040707060100200020608090600586
:1014B00007070600004020205070888805070706AF
:1014C00000001020205070888805070706000020C3
:1014D00050205070888805070706000028502050CB
:1014E0007088880507070600005000205070888823
:1014F0000507070600002050205070888805060662
:1015000006000078A0F0A0A0B80408080601FE605C
:10151000908080906020400407070601004020F082
:1015200080E080F00407070601002040F080E080A2
:10153000F00407070601002050F080E080F0040767
:10154000070601005000F080E080F0030707060165
:10155000008040E0404040E00307070601002040D3
:10156000E0404040E003070706010040A0E04040A3
:1015700040E0030707060100A000E0404040E0050E
:1015800006060600007048E8484870040707060190
:101590000050A090D0B090900407070601004020B2
:1015A00060909090600407070601002040609090D2
:1015B000906004070706010020506090909060043E
:1015C000070706010050A06090909060040707068E
:1015D00001005000609090906005050506000088AD
:1015E000502050880408080601FF1070B0B0D0D019
:1015F000E08004070706010040209090909060046E
:1016000007070601002040909090906004070706AD
:101610000100205090909090600407070601005050
:1016200000909090906005070706000010208850F9
:1016300020202004060606010080E09090E080044F
:1016400006060601006090A0A090A004070706010E
:1016500000402000709090700407070601002040B1
:1016600000709090700407070601002050007090F1
:10167000907004070706010050A00070909070045D
:1016800006060601005000709090700407070601DE
:10169000002050207090907005040406000070A88F
:1016A000B0780406060601FE7080807020400407B2
:1016B0000706010040200060B0C070040707060163
:1016C0000020400060B0C0700407070601002050F1
:1016D0000060B0C070040606060100500060B0C093
:1016E00070030707060100804000C04040E0030788
:1016F00007060100204000C04040E0030707060144
:101700000040A000C04040E0030606060100A00023
:10171000C04040E004070706010030601070909060
:101720006004070706010050A000E09090900407B5
:101730000706010040200060909060040707060142
:1017400000204000609090600407070601002050D0
:10175000006090906004070706010050A0006090B0
:101760009060040606060100500060909060050538
:10177000050600002000F8002004040406010070A3
:10178000B0D0E00407070601004020009090907060
:10179000040707060100204000909090700407079E
:1017A000060100205000909090700406060601008B
:1017B0005000909090700409090601FE20400090AE
:1017C00090907090600408080601FE8080E0909080
:1017D000E080800408080601FE5000909090709010
:1017E0006000002200250028002B002E003100346C
:1017F0000002010000050108010B0100000A0B02B4
:10180000090C0D0E08070304010000000000000091
:1018100000000000000000000000000000000000C8
:101820000000000000000012111000000000000085
:1018300000000000000000000000000000000000A8
:1018400000290A002062797465733B20637263206B
:101850000053657474696E67732053746F726564A6
:101860002028000200002100240027002A002D006B
:101870003000330001010000040107010A010102E8
:101880001020200808102040102040800201020192
:10189000080402010102040810204080804020104A
:1018A00008040201800402018040201008040201A3
:1018B000080402010102040810204080010204080B
:1018C00010204080050505050705080808080202E4
:1018D00002020A0A080804040404010101010101CA
:1018E00001010303030303030303040707070C0CAD
:1018F0000C0C0C0C0C0C0202020206060606060674
:1019000006060B0B0B0B0B0B0B0B1FFFFFFFFFFF59
:10191000FF600000000001FF400000000000FF80A9
:1019200000000000007F83CF00000C303F87FF8065
:10193000000C301F867980000C000F8C30C7838C20
:1019400030E78C30CFC7CC31F38C30DCECEC33B9E2
:101950008C30D86C6C33198C30D06C0C33198C30C3
:10196000D86C0C33198C30DC6C0E3B198C30CF7C6E
:10197000079F198C30C77C038F19400000000000BE
:1019800002600000000000061FFFFFFFFFFFF820BD
:1019900020506C616E6E6572427566666572427942
:1019A0007465733A20002046726565204D656D6F41
:1019B00072793A2000436F6D70696C65643A204E0D
:1019C0006F7620323120323031370A00207C2041BE
:1019D0007574686F723A2028416C657068204F6298
:1019E0006A6563747320496E632E2C204C756C7A83
:1019F000426F7420476974205265706F7369746F09
:101A00007279290A004E6F76203231203230313718
:101A100031333A33373A313800204C6173742055F2
:101A20007064617465643A2000312E312E350A00ED
:101A30004D61726C696E0020536F667477617265D8
:101A40002052657365740A00205761746368646F7F
:101A5000672052657365740A002042726F776E20AA
:101A60006F75742052657365740A0020457874653B
:101A7000726E616C2052657365740A00506F7765F1
:101A80007255700A0073746172740A006572726F25
:101A9000722077726974696E6720746F2066696C52
:101AA000650A004572726F723A00456E6473746F16
:101AB0007073202563202563202563202563002083
:101AC000503A00205A3A0020593A0020583A00650E
:101AD0006E6473746F7073206869743A2000656374
:101AE000686F3A00446F6E6520736176696E672097
:101AF00066696C652E0A004D32390052657769704F
:101B0000696E670050726F62696E67206661696C0A
:101B100065640050726F62696E67206661696C650A
:101B2000640050524F4245204641494C20434C45A9
:101B3000414E204E4F5A5A4C450A00526577697003
:101B4000696E670A005265776970696E6700507246
:101B50006F62696E67206661696C65640050726FC0
:101B600062696E67206661696C65640050524F421D
:101B700045204641494C20434C45414E204E4F5A4A
:101B80005A4C450A005265776970696E670A0050C1
:101B9000726F62696E67206661696C65640A0050E5
:101BA000726F62696E67206661696C656400205AB5
:101BB0003A200020593A200042656420583A20001B
:101BC0000A0A426564204C6576656C20436F727228
:101BD000656374696F6E204D61747269783A002094
:101BE0002B000A436F7272656374656420426564FA
:101BF000204865696768742076732E2042656420EA
:101C0000546F706F6C6F67793A0A00202B000A429C
:101C100065642048656967687420546F706F6772E7
:101C2000617068793A0A2020202B2D2D2D20424109
:101C3000434B202D2D2B0A2020207C2020202020EB
:101C40002020202020207C0A204C207C20202020C6
:101C5000282B29202020207C20520A2045207C206F
:101C6000202020202020202020207C20490A2046DF
:101C7000207C20282D29204E20282B29207C20471D
:101C80000A2054207C2020202020202020202020DA
:101C90007C20480A2020207C20202020282D29205C
:101CA0002020207C20540A2020207C20202020205E
:101CB0002020202020207C0A2020204F2D2D20466F
:101CC000524F4E54202D2D2B0A2028302C30290A1B
:101CD000004D65616E206F662073616D706C656488
:101CE00020706F696E74733A200020643A200020DF
:101CF000623A200045716E20636F656666696369AC
:101D0000656E74733A20613A200052756E6E696E8A
:101D10006720696E204452592D52554E206D6F64D4
:101D2000650A00473239204175746F20426564208E
:101D30004C6576656C696E670A0028422961636BA1
:101D400000284629726F6E740028522969676874EA
:101D500000284C29656674003F4E756D62657220DF
:101D60006F662070726F626520706F696E74732089
:101D7000697320696D706C61757369626C65202888
:101D800032206D696E696D756D292E0A003F2856E7
:101D9000296572626F7365206C6576656C20697366
:101DA00020696D706C61757369626C652028302DD7
:101DB00034292E0A004B494C4C45442E200024F473
:101DC000D43050C38E20C2A24017828B7011127A79
:101DD000910D816CD90AA861E108C7586607615165
:101DE00043061E4B5D05C145A7041A411104093D78
:101DF0009803713931034036DB0265339102D430E8
:101E00005402802E1D02632CEE01752AC501B028F4
:101E1000A001102781018F2564012B244B01E022B2
:101E20003401AC211F018D200D01801FFC00841E98
:101E3000ED00971DDF00B81CD200E61BC600201B7A
:101E4000BC00641AB200B219A8000A19A0006A18EE
:101E50009900D117910040178B00B51684003116F8
:101E60007E00B31579003A157300C7146F0058143B
:101E70006A00EE1366008813630025135E00C71224
:101E80005B006C12570015125400C1115100701103
:101E90004F0021114B00D61049008D10470046100D
:101EA000440002104200C00F4000800F3E00420F6D
:101EB0003C00060F3B00CB0E3800930E37005C0E43
:101EC0003500270E3400F30D3200C10D3100900DA6
:101ED0003000600D2E00320D2D00050D2C00D90CA8
:101EE0002B00AE0C2900850C29005C0C2700350C5A
:101EF00027000E0C2600E80B2400C40B2400A00BC6
:101F000023007D0B23005A0B2100390B2100180BF5
:101F10002000F80A1F00D90A1E00BB0A1E009D0AF5
:101F20001D00800A1D00630A1C00470A1B002C0AC2
:101F30001B00110A1A00F7091A00DD091900C4096B
:101F40001900AB091900920917007B0918006309F1
:101F500017004C09160036091600200916000A0958
:101F60001500F5081500E0081400CC081400B808A6
:101F70001400A4081400900813007D0812006B08D8
:101F800013005808120046081200340811002308F4
:101F900011001208110001081100F0071000E007FD
:101FA0001000D0071000C0071000B0070F00A107F5
:101FB000100091070E0083070F0074070F006507DC
:101FC0000E0057070E0049070E003B070D002E07B5
:101FD0000E0020070D0013070D0006070D00F9067F
:101FE0000C00ED060D00E0060C00D4060C00C8063F
:101FF0000C00BC060C00B0060C00A4060B009906F1
:102000000C008D060B0082060B0077060B006C0699
:102010000B0061060A0057060B004C060A00420638
:102020000A0038060A002E060A0024060A001A06CC
:102030000A001006090007060A00FD050900F4055C
:102040000900EB050900E2050900D9050900D005E2
:102050000900C7050900BE050900B5050800AD0562
:102060000800A50509009C050800940508008C05DA
:102070000800840508007C050800740508006C054C
:102080000700650508005D050700560508004E05B8
:10209000070047050700400508003805070031051F
:1020A00007002A050700230507001C050600160582
:1020B00007000F0507000805060002050700FB04DE
:1020C0000600F5040700EE040600E8040600E2043A
:1020D0000700DB040600D5040600CF040600C9048F
:1020E0000600C3040600BD040600B7040600B104E0
:1020F0000500AC040600A6040600A00405009B042D
:10210000060095040500900406008A040500850475
:102110000500800406007A040500750405007004BB
:1021200005006B04050066040500610405005C04FD
:10213000050057040500520405004D04050048043D
:102140000500430405003E0404003A04050035047C
:102150000500300404002C040500270404002304B7
:1021600005001E0404001A040400160405001104EE
:1021700004000D0404000904050004040400000424
:102180000400FC030400F8030400F4030400F0035B
:102190000400EC030400E8030400E4030400E0038B
:1021A0000400DC030400D8030400D4030400D003BB
:1021B0000400CC030400C8030300C503030024F497
:1021C00004D9201BC40C5C0E9804C4095F02650787
:1021D0007101F405F900FB04B30048048700C10352
:1021E00069005803550003034500BE023A0084020B
:1021F000310053022A002902250004022000E401D4
:102200001C00C8011900AF011700980114008401D7
:102210001300710110006101100051010E00430113
:102220000D0036010B002B010B0020010B001501E6
:1022300009000C01090003010800FB000800F3007D
:102240000800EB000700E4000600DE000600D800EE
:102250000600D2000600CC000500C7000500C20041
:102260000500BD000400B9000400B5000400B10081
:102270000400AD000400A9000400A5000300A200B2
:1022800003009F0004009B000300980003009500DA
:10229000020093000300900003008D0002008B00F9
:1022A0000300880002008600020084000300810011
:1022B00002007F0002007D0002007B000200790026
:1022C0000200770001007600020074000200720034
:1022D0000100710002006F0002006D0001006C003F
:1022E00002006A0001006900020067000100660048
:1022F000010065000100640002006200010061004D
:102300000100600001005F0002005D0001005C0050
:1023100001005B0001005A00010059000100580053
:102320000100570001005600010055000100540053
:102330000100530000005300010052000100510051
:102340000100500001004F0001004E0000004E004F
:1023500001004D0001004C0001004B0000004B004B
:1023600001004A0001004900010048000000480047
:102370000100470001004600000046000100450042
:10238000000045000100440001004300000043003C
:102390000100420000004200010041000000410035
:1023A0000100400001003F0000003F0001003E002E
:1023B00000003E0001003D0000003D0001003C0027
:1023C00000003C0000003C0001003B0000003B001E
:1023D00001003A0000003A00010039000000390015
:1023E000010038000000380000003800010037000C
:1023F0000000370001003600000036000000360003
:1024000001003500000035000000350001003400F7
:1024100000003400000034000100330000003300ED
:1024200000003300010032000000320000003200E2
:1024300001003100000031000000310001003000D7
:10244000000030000000300001002F0000002F00CD
:1024500000002F0000002F0001002E0000002E00C1
:1024600000002E0001002D0000002D0000002D00B6
:1024700000002D0001002C0000002C0000002C00AA
:1024800000002C0001002B0000002B0000002B009E
:1024900000002B0001002A0000002A0000002A0092
:1024A00000002A0001002900000029000000290086
:1024B0000000290000002900010028000000280079
:1024C000000028000000280000002800010027006C
:1024D0000000270000002700000027000000270060
:1024E0000100260000002600000026000000260053
:1024F0000000260001002500000025000000250046
:102500000000250000002500000025000100240037
:10251000000024000000240000002400000024002B
:10252000010023000000230000002300000023001E
:10253000000023000000230000002300010022000F
:102540000000220000002200000022000000220003
:1025500000002200010021000000210000002100F5
:1025600000002100000021000000210000002100E7
:1025700001002000000020000000200000002000DA
:1025800000002000000020000000200000002000CB
:1025900001001F0000001F0000001F0000001F00BE
:1025A00000001F0000001F0000001F0001001E00AF
:1025B00000001E0000001E0000001E0000004D383C
:1025C0003420582059205A2045004572723A204D37
:1025D000494E54454D5020424544004D494E5445C6
:1025E0004D50207472696767657265640045727248
:1025F0003A204D494E54454D5020453100457272A8
:102600003A204D494E54454D502045300045727298
:102610003A204D415854454D5020424544004D41CB
:102620005854454D5020747269676765726564003F
:102630004572723A204D415854454D502045310065
:102640004572723A204D415854454D502045300056
:10265000746F20726573756D6500576169742066CB
:102660006F72207072696E74005052494E5420503F
:1026700041555345440045787472756465206D6F0B
:10268000726500526573756D65207072696E7400B5
:10269000524553554D45204F5054494F4E533A00E3
:1026A00020204E6F7A7A6C653A20002000506C65CD
:1026B00061736520776169742E2E2E004865617400
:1026C000696E67206E6F7A7A6C65005052494E547D
:1026D000205041555345440020204E6F7A7A6C6556
:1026E0003A2000200068656174206E6F7A7A6C650C
:1026F0002E00507265737320627574746F6E20744F
:102700006F005052494E54205041555345440020CB
:10271000204E6F7A7A6C653A2000200066696C6101
:102720006D656E74206578747275646500576169B3
:102730007420666F72005052494E542050415553D8
:1027400045440020204E6F7A7A6C653A20002000C4
:1027500066696C616D656E74206C6F6164005761B1
:10276000697420666F72005052494E542050415592
:102770005345440020204E6F7A7A6C653A200074ED
:102780006F20636F6E74696E75652E2E2E00616EFC
:102790006420707265737320627574746F6E004983
:1027A0006E736572742066696C616D656E7400503D
:1027B00052494E54205041555345440020204E6FFD
:1027C0007A7A6C653A2000200066696C616D656EEE
:1027D0007420756E6C6F6164005761697420666F58
:1027E00072005052494E54205041555345440020E8
:1027F000204E6F7A7A6C653A20006368616E676577
:10280000006F66207468652066696C616D656E7422
:10281000005761697420666F72207374617274006E
:102820005052494E54205041555345440020204EAB
:102830006F7A7A6C653A200020004261636B004D2C
:10284000696E696D756D2054656D702069732031F6
:1028500032302E0048656174696E67206661696C6C
:1028600065640001050800FF060121023520FFFF15
:1028700007FF06FF090050221656808080800080E6
:10288000153353A0A0A00257575050F850F850509D
:102890000257572070A07028702013355580A04033
:1028A000A02002475740A0A040A0A050251353806D
:1028B00080801226564080808080401226568040BC
:1028C000404040800245559060F060900255552090
:1028D00020F82020113353604080044151F011331F
:1028E0005340E04002465610102040808012365679
:1028F00040A0A0A0A04012365640C0404040E00298
:1029000046566090106080F0024656F020601090AD
:10291000600246562060A0F02020024656F080E07B
:102920001090600246566080E0909060024656F03B
:102930001020204040024656609060909060024611
:1029400056609090701060122555C0C000C0C01134
:1029500036566060006040801236562040808040CD
:1029600020034353F000F012365680402020408070
:1029700012365640A020400040015858304898A8D0
:10298000A8904030024656609090F09090024656D3
:10299000E090E09090E00246566090808090600267
:1029A0004656E090909090E0024656F080E080809D
:1029B000F0024656F080E0808080024656609080AB
:1029C000B090600246569090F0909090123656E08B
:1029D00040404040E002465670202020A040024681
:1029E0005690A0C0A0A0900246568080808080F0C3
:1029F00002465690F0F090909002465690D0F0B07B
:102A0000B090024656609090909060024656E090DA
:102A100090E08080014757609090D0B060100246EF
:102A200056E09090E0909002465660904020906072
:102A3000123656E0404040404002465690909090FA
:102A4000906002465690909090606002465690903A
:102A500090F0F0900246569090606090900256562A
:102A6000888850202020024656F010204080F01226
:102A70003656E080808080E00246568080402010FC
:102A800010123656E020202020E016325240A001DD
:102A90004151F016225280400244547090907002CE
:102AA00046568080E09090E012345460808060024E
:102AB000465610107090907002445460B0C060028E
:102AC0004656205040E040400145556090701060EF
:102AD0000246568080E09090901236564000C040EA
:102AE00040E01137572000202020A04002465680A9
:102AF0008090E09090123656C040404040E0025432
:102B000054D0A8A8A8024454E09090900244546085
:102B1000909060014555E090E080800145557090AF
:102B2000701010024454A0D0808012345460C02031
:102B3000C00246564040E0405020024454909090DD
:102B400070123454A0A0A04002545488A8A8500287
:102B5000445490606090014555909070906002449C
:102B600054F02040F0024757304020C0204030222F
:102B70001656808080808080024757C020403040B9
:102B800020C006425250A0FFFFFFFFFFFFFFFFFFE4
:102B9000FFFFFFFFFFFFFFFFFFFFFFFFFFFFFFFF45
:102BA000FFFFFFFFFFFFFFFF0900502216568000C6
:102BB000808080800146562070A0A070200246567A
:102BC0002050E04050A00255558870507088025641
:102BD000568850F820F82022175780808000808087
:102BE000800247577080E0907010E0173151A002CA
:102BF000565670A8C8C8A87014355560A06000E08B
:102C000003435350A050123353E02020143151E0BD
:102C100002565670E8D8E8D870173151E015335392
:102C200040A04012355540E04000E014355540A02A
:102C30002040E0143555C020C020C01622524080EC
:102C4000014555909090E08002565678E8E8682853
:102C50002824115180112252408014355540C04023
:102C600040E014355540A04000E0034353A050A07D
:102C7000024757808080A060F0200247578080A0E4
:102C8000D010207002475780408060A0F02012369C
:102C90005640004080A04002475740206090F0908E
:102CA0009002475720406090F09090024757609004
:102CB0006090F0909002475750A06090F090900282
:102CC000475790006090F090900247576090609056
:102CD000F0909002465670A0A0F0A0B00147576057
:102CE0009080809060400247574020F080E080F064
:102CF0000247572040F080E080F00247576090F094
:102D000080E080F00247579000F080E080F01237BA
:102D1000578040E0404040E01237572040E04040BC
:102D200040E012375740A0E0404040E0123757A043
:102D300000E0404040E00256567048E848487002C3
:102D4000475750A090D0B0909002475740206090D5
:102D500090906002475720406090909060024757E3
:102D60006090609090906002475750A06090909063
:102D70006002475790006090909060123353A040DB
:102D8000A002465670B0B0D0D0E002475740209025
:102D9000909090600247572040909090906002473A
:102DA000576090909090906002475790009090905C
:102DB00090600257571020885020202002465680ED
:102DC000E09090E0800246566090A0A090A002475C
:102DD000574020007090907002475720400070903C
:102DE00090700247572050007090907002475750E3
:102DF000A000709090700246565000709090700243
:102E0000475760906070909070025454F068B078AA
:102E1000113555608080604002475740200060B007
:102E2000C06002475720400060B0C0600247576052
:102E3000900060B0C060024656500060B0C06012A2
:102E40003757804000C04040E0123757204000C054
:102E50004040E012375740A000C04040E0123656D4
:102E6000A000C04040E0024757A040A01070906012
:102E700002475750A000E090909002475740200032
:102E80006090906002475720400060909060024739
:102E9000576090006090906002475750A00060908B
:102EA0009060024656900060909060123555400048
:102EB000E0004002445470B0D0E002475740200088
:102EC0009090907002475720400090909070024779
:102ED00057609000909090700246569000909090AD
:102EE00070014858204000909070906001475780D2
:102EF00080E090E080800147579000909070906053
:102F000001050700FE0500FB01F220FFFE05FE059E
:102F1000FE0200400215258080800080053242A01C
:102F2000A002556550F850F8500146562070C03048
:102F3000E020025565901020404802556560806889
:102F400090680512228080022535408080804002F2
:102F500025358040404080043343A040A0033343E4
:102F600040E0400122324080043141E002112180E2
:102F70000255650810204080024555609090906091
:102F8000022535C040404040024555E0106080F0C9
:102F9000024555E0106010E00245552060A0F02089
:102FA000024555F080E010E00245556080E09060F9
:102FB000024555F0102040400245556090609060F9
:102FC0000245556090701060031323800080021446
:102FD0002480008080023545204080402003334318
:102FE000E000E00235458040204080024555E01079
:102FF0006000400255657088B8A870024555609021
:1030000090F090024555E090E090E00235456080F8
:10301000808060024555E0909090E0023545E08068
:10302000E080E0023545E080E08080024555708018
:10303000B090700245559090F09090023545E04078
:103040004040E0024555301010906002455590A078
:10305000C0A09002354580808080E002556588D808
:10306000A8888802455590D0B09090024555609050
:10307000909060024555E09090E080014656609047
:1030800090906010024555E09090E0900245557098
:10309000806010E0023545E04040404002455590D8
:1030A000909090600245559090A0A0400255658890
:1030B000A8A8A85002455590906090900245559060
:1030C00090701060023545E0204080E0022535C058
:1030D000808080C00255658040201008022535C0E0
:1030E000404040C005324240A0024151F00522322A
:1030F00080400244547090907002455580E090905A
:10310000E0023444608080600245551070909070F9
:1031100002445460B0C0600235452040E0404000A9
:10312000465670909070106002455580E0909090E7
:1031300002152580008080800027374000404040F5
:1031400040800245558090A0E09002152580808047
:103150008080025464F0A8A8A8024454E0909090A3
:1031600002445460909060004656E09090E0808069
:10317000004656709090701010023444A0C08080B9
:1031800002445470C030E002354540E04040200227
:103190004454909090700244549090A04002546423
:1031A000A8A85050023444A04040A0004656909039
:1031B00090701060024454F02040F00235456040A9
:1031C0008040600215258080808080023545C040A7
:1031D0002040C005425250A0FFFFFFFFFFFFFFFF4E
:1031E000FFFFFFFFFFFFFFFFFFFFFFFFFFFFFFFFEF
:1031F000FFFFFFFFFFFFFFFFFF020040FFFFFFFF9A
:10320000FFFFFFFFFFFFFFFFFFFFFFFFFFFFFFFFCE
:10321000FFFFFFFFFFFFFFFFFFFFFFFFFFFFFFFFBE
:10322000FFFFFFFFFFFFFFFFFFFFFFFFFFFFFFFFAE
:10323000FFFFFFFFFFFFFFFFFFFFFFFFFFFFFFFF9E
:10324000FFFFFFFFFFFFFFFFFFFFFFFFFFFFFFFF8E
:10325000FFFFFFFFFFFFFFFFFFFFFF01060D00FE67
:1032600009016602D620FFFE0BFE0AFE0D00602259
:103270001969808080808080800080183363A0A0DE
:10328000A00357675050F850F85050025969207801
:10329000A0A0702828F02002596948A850102040AA
:1032A00050A89002586840A0A040A09890682813A9
:1032B00063808080113B6B20404080808080804014
:1032C0004020113B6B804040202020202040408047
:1032D00006556520A870A8200455652020F82020F8
:1032E000113363604080065161F811336340E04060
:1032F0000259690808101020404080800259692056
:1033000050888888888850200259692060A0202031
:10331000202020F80259697088880810204080F821
:10332000025969F80810207008088870025969105D
:103330001030505090F81010025969F88080B0C8D1
:103340000808887002596970888080F088888870C1
:10335000025969F808101020204040400259697055
:103360008888887088888870025969708888887809
:103370000808887011386840E040000040E04011C3
:10338000386840E040000060408002596908102021
:10339000408040201008045464F80000F802596985
:1033A00080402010081020408002596970888808E9
:1033B000102020002002596970888898A8A8B08041
:1033C000780259692050888888F888888802596965
:1033D000F048484870484848F00259697088808031
:1033E0008080808870025969F048484848484848B9
:1033F000F0025969F8808080F0808080F802596975
:10340000F8808080F0808080800259697088808098
:10341000809888887002596988888888F8888888A0
:1034200088123969E040404040404040E00259691C
:10343000381010101010109060025969888890A000
:10344000C0A09088880259698080808080808080B8
:10345000F80259698888D8A8A88888888802596994
:1034600088C8C8A8A89898888802596970888888E8
:103470008888888870025969F0888888F080808000
:1034800080015A6A70888888888888A870080259DC
:1034900069F0888888F0A0908888025969708880CF
:1034A000807008088870025969F8202020202020A8
:1034B00020200259698888888888888888700259FD
:1034C00069888888885050502020025969888888E7
:1034D00088A8A8A8A8500259698888505020505040
:1034E000888802596988885050202020202002595D
:1034F00069F808101020404080F8113B6BE0808094
:1035000080808080808080E00259698080404020F7
:1035100010100808113B6BE02020202020202020E4
:1035200020E0085363205088015161F82A2262800C
:1035300040025666700878889868025969808080D1
:10354000F088888888F002566670888080887002CB
:1035500059690808087888888888780256667088CB
:10356000F880887002596930484040F0404040403F
:103570000058687088888878088870025969808047
:1035800080B0C8888888881238684000C0404040B1
:1035900040E0004A6A100030101010109090600255
:1035A000596980808090A0C0A09088123969C0407D
:1035B000404040404040E0025666D0A8A8A8A888F5
:1035C000025666B0C88888888802566670888888DF
:1035D0008870005868F0888888F08080800058687B
:1035E0007888888878080808025666B0C880808085
:1035F000800256667088601088700258684040F0FB
:10360000404040483002566688888888986802564C
:10361000668888885050200256668888A8A8A850D6
:1036200002566688502020508800586888888898FC
:1036300068088870025666F810204080F8015B6BBD
:103640001820202020C020202020182219698080E6
:1036500080808080808080015B6BC02020202018CB
:1036600020202020C008536348A890FFFFFFFFFFE1
:10367000FFFFFFFFFFFFFFFFFFFFFFFFFFFFFFFF5A
:10368000FFFFFFFFFFFFFFFFFFFFFFFF0D006022B7
:103690001969800080808080808080035868207055
:1036A000A8A0A0A8702002596930484040E04040DE
:1036B00048B00356668870505070880259698888EF
:1036C0005050F820F82020221969808080800080E6
:1036D000808080124A6A6090806090906010906054
:1036E0001A3262A0A00359697088A8D8C8D8A888DF
:1036F00070045767700878887800F8035666285079
:10370000A0A05028045363F80808163161E003595B
:10371000697088E8D8D8E8D888700A5161F81744E9
:1037200064609090600357672020F8202000F8071D
:10373000356540A02040E007356540A04020C02A04
:10374000226240800058688888888898E8808002D3
:10375000596978E8E8E8E868282828262161C02027
:103760002262408007356540C04040E004576770E2
:103770008888887000F8035666A050282850A00258
:103780005A6A40C04040E00818283808025A6A4087
:10379000C04040E01028081038025A6A40A040207B
:1037A000A048182838080259692000202040808845
:1037B0008870025A6A40200020508888F888880261
:1037C0005A6A10200020508888F88888025A6A3087
:1037D000480020508888F88888025A6A28500020BB
:1037E000508888F88888025A6A505000205088888B
:1037F000F88888025A6A20502020508888F88888E3
:1038000002596958A0A0A0B0E0A0A0B8005B6B70FE
:1038100088808080808088702040025A6A40200022
:10382000F88080F08080F8025A6A102000F88080CA
:10383000F08080F8025A6A304800F88080F080807A
:10384000F8025A6A505000F88080F08080F8123AEE
:103850006A804000E04040404040E0123A6A204028
:1038600000E04040404040E0124A6A609000E04082
:1038700040404040E0123A6AA0A000E04040404092
:1038800040E0025969F0484848E8484848F0025A80
:103890006A2850008888C8A8988888025A6A4020F8
:1038A0000070888888888870025A6A1020007088A2
:1038B0008888888870025A6A3048007088888888AA
:1038C0008870025A6A285000708888888888700238
:1038D0005A6A5050007088888888887003556588B7
:1038E00050205088015B6B08709898A8A8A8C8C899
:1038F0007080025A6A402000888888888888700210
:103900005A6A10200088888888888870025A6A302D
:10391000480088888888888870025A6A50500088D1
:10392000888888888870025A6A1020008888502009
:1039300020202002596980F0888888F080808002E9
:103940005969609090A0A0908888B0025969402081
:10395000007008788898680259691020007008780B
:103960008898680259693048007008788898680219
:103970005969285000700878889868025969505031
:1039800000700878889868025A6A304830007008D9
:1039900078889868025666702870A0A85000586809
:1039A00070888080887020400259694020007088AB
:1039B000F88088700259691020007088F88088703B
:1039C0000259693048007088F8808870025969503F
:1039D00050007088F8808870123969804000C040BB
:1039E000404040E0123969204000C040404040E083
:1039F000124969609000C040404040E0123969A01F
:103A0000A000C040404040E0025A6A502060107060
:103A10008888888870025969285000B0C8888888CA
:103A20008802596940200070888888887002596926
:103A300010200070888888887002596930480070AA
:103A4000888888887002596928500070888888881A
:103A500070025969505000708888888870035767D1
:103A6000202000F8002020015868087098A8A8C8F5
:103A700070800259694020008888888898680259B7
:103A80006910200088888888986802596930480041
:103A90008888888898680259695050008888888882
:103AA0009868005B6B102000888888986808887088
:103AB000005A6A8080B0C88888C8B08080005B6B7C
:103AC00050500088888898680888700000000000BE
:103AD00000000000000000000000000000000000E6
:103AE00000000000000000000000000000000C00CA
:103AF0000000000000000C000000000000001200A8
:103B00000000000000002300000000000000210071
:103B10000000000000004C800000000000005E80FB
:103B20000000000000009240000000000000A140E2
:103B300000000000000121200000000000027F9032
:103B40000000000000020010000000000007FFF865
:103B5000000000000004000800000000000800044D
:103B60000000000000080006000000000010000235
:103B70000000000000301E010000000000207F81D6
:103B8000000000000041FFE0800000000043FCF066
:103B90008000000000873B7840000000018EDBFCC5
:103BA00060000000010FEBCC20000000021FEDB60A
:103BB00010000000021FDEB6100000000439CD7FA7
:103BC000080000000436E0FF08000000087EC0BBCB
:103BD00084000000187F005D86000000107FC0EDAB
:103BE00082000000203CC07301000000203B337FB6
:103BF00001000000701BE77E03800000C81DEEDEA0
:103C000004C00000880FDEDC04400001240FDF3C0C
:103C1000092000012607DBF8192000027203E7F0F3
:103C2000139000025101FFE02290000489007F8080
:103C30002448000904801E004824000BFE400000B8
:103C4000DFF40010004000008002001FFFFFFFFFB4
:103C5000FFFE000000000000000000000000000067
:103C600000000000000000000000001022103C3C9A
:103C70000E1F00102210042211040010221008222E
:103C8000110400102210083C110400102210102210
:103C900011040010221020221104001E1C1E3C3CA6
:103CA0000E04000000000000000000000000000002
:103CB0000000000000000000000000000000000004
:103CC00000000000000000000000000000000000F4
:103CD00000000000000000000000000000000000E4
:103CE00000000000000000000000000000000000D4
:103CF00000000000000000000000000000000000C4
:103D00000000000000000000000A003B2045455074
:103D1000524F4D20496E6465783A200055706461B9
:103D200074696E67207A6F666673657420696E20A9
:103D3000454550524F4D3A20000600060006000649
:103D400000060006000600060006003FC01F800FA8
:103D500000060006000F001F803FC0060006000698
:103D60000006000600060006000600060007F80030
:103D70000C0C001002002001006001804000804017
:103D800003E04001C04000804000004000006000AF
:103D9000002000001000000C0C0007F80001FE00DD
:103DA0000303000400800800401800601000207C1D
:103DB000002038002010002000002000002000001B
:103DC0006000004000008003030001FE00FFFFFFD1
:103DD0007F80FFC0FFC0FFC07F807F80FFC0FFC02B
:103DE000FFC03F001E000C005A204F6666736574CA
:103DF000004D6F76652058004D6F76652059004D57
:103E00006F7665205A004578747275646572004D4E
:103E100036303020486F74656E6420746F6F206395
:103E20006F6C6420746F206368616E6765206669DB
:103E30006C616D656E740A004B64200023646566D6
:103E4000696E65202044454641554C545F004B69DE
:103E5000200023646566696E65202044454641550F
:103E60004C545F004B70200023646566696E6520CA
:103E70002044454641554C545F005049442041750B
:103E8000746F74756E652066696E69736865642108
:103E90002050757420746865206C617374204B70B9
:103EA0002C204B6920616E64204B6420636F6E731D
:103EB00074616E74732066726F6D2062656C6F77CB
:103EC00020696E746F20436F6E66696775726174E6
:103ED000696F6E2E680A00504944204175746F74F2
:103EE000756E65206661696C6564212074696D6515
:103EF0006F75740A00504944204175746F74756E73
:103F000065206661696C6564212054656D70657219
:103F1000617475726520746F6F20686967680A0044
:103F2000204B643A2000204B693A2000204B703A25
:103F300020000A20436C6173736963205049442058
:103F40000A002054753A2000204B753A2000206D5D
:103F500061783A2000206D696E3A200020643A2092
:103F60000020626961733A20004B494C4C45442E55
:103F700020004B494C4C2063617573656420627965
:103F8000204B494C4C20627574746F6E2F70696EB3
:103F90000A004B494C4C45442E20004B494C4C20C8
:103FA00063617573656420627920746F6F206D752D
:103FB000636820696E6163746976652074696D65F4
:103FC000202D2063757272656E7420636F6D6D6154
:103FD0006E643A200020746F6F206C6F6E672065EE
:103FE0007874727573696F6E2070726576656E7421
:103FF00065640A0020636F6C642065787472757361
:10400000696F6E2070726576656E7465640A005023
:104010006C65617365207265736574005052494E1A
:104020005445522048414C544544005072696E74C6
:1040300065722068616C7465642E206B696C6C28F5
:10404000292063616C6C6564210A006265640A0062
:104050002C2073797374656D2073746F7070656450
:1040600021204865617465725F49443A20005448D4
:1040700045524D414C2052554E41574159204245E1
:104080004400546865726D616C2052756E61776191
:104090007900544845524D414C2052554E415741AC
:1040A0005920453100544845524D414C2052554EFF
:1040B000415741592045300048656174696E672059
:1040C0006661696C656420424544004865617469B5
:1040D0006E67206661696C65640048656174696E2D
:1040E00067206661696C65640048656174696E6724
:1040F000206661696C656420453000577269746997
:104100006E6720746F2066696C653A20006F706579
:104110006E206661696C65642C2046696C653A2086
:10412000006F70656E206661696C65642C2046695D
:104130006C653A200046696C652073656C65637434
:1041400065640A002053697A653A200046696C6507
:10415000206F70656E65643A20006F70656E206632
:1041600061696C65642C2046696C653A20002066A4
:10417000696C653A20004E6F7720002220706F73C3
:10418000002220706172656E743A220053554252CB
:104190004F5554494E452043414C4C207461726741
:1041A00065743A22004B494C4C45442E20007472F1
:1041B00079696E6720746F2063616C6C207375621F
:1041C0002D67636F64652066696C65732077697419
:1041D0006820746F6F206D616E79206C6576656CF8
:1041E000732E204D4158206C6576656C2069733ABA
:1041F000004F6666004F6E2000456E6473746F70EA
:104200002061626F72740053746570732F6D6D005E
:104210004A65726B00416363656C65726174696FB6
:104220006E0056656C6F63697479005A204F66663C
:1042300073657400416476616E63656420536574D0
:1042400074696E6773005654726176206D696E00F2
:104250005654726176206D696E00565472617620F4
:104260006D696E00566D696E00566D696E00566D13
:10427000696E00566D6178204500566D6178204565
:1042800000566D6178204500566D6178205A0056C1
:104290006D6178205A00566D6178205A00566D6124
:1042A00078205900566D6178205900566D6178204C
:1042B0005900566D6178205800566D61782058007D
:1042C000566D61782058004D6F74696F6E004573AC
:1042D000746570732F6D6D004573746570732F6D09
:1042E0006D005A73746570732F6D6D005A73746529
:1042F00070732F6D6D005973746570732F6D6D0041
:104300005973746570732F6D6D0058737465707395
:104310002F6D6D005873746570732F6D6D004D6F48
:1043200074696F6E0056652D6A65726B0056652D57
:104330006A65726B0056652D6A65726B00567A2D40
:104340006A65726B00567A2D6A65726B0056792D1C
:104350006A65726B0056792D6A65726B0056792D0D
:104360006A65726B0056782D6A65726B0056782DFF
:104370006A65726B0056782D6A65726B004D6F74BA
:10438000696F6E00526573746F7265206661696C47
:1043900073616665004D3530320A4D353030004C62
:1043A0006F61642073657474696E67730053746F12
:1043B00072652073657474696E6773004164766119
:1043C0006E6365642053657474696E6773004D6134
:1043D000696E005072696E742061626F72746564F8
:1043E0000041626F7574204669726D776172650075
:1043F0004E6F2053442063617264005072696E7482
:104400002066726F6D2053440053746F7020707279
:10441000696E7400526573756D65207072696E7493
:10442000005061757365207072696E7400436F6E21
:1044300066696775726174696F6E0054656D706549
:10444000726174757265004D6F76656D656E74008E
:104450004368616E67652066696C616D656E7400A6
:1044600054756E6500496E666F2073637265656E84
:104470000025753A2530327500253032753A2530E1
:1044800032750025756420253032753A2530327535
:104490000000060900FE000000000001090008FEFF
:1044A000000005080806000040F0C88888987810C9
:1044B000050808060000C0F88888888888F805057F
:1044C000050600012030F83020050808060000200D
:1044D00070F820202020E00509090600FF2070A8C0
:1044E000A8B8888870200509090600FFE080C0B0E0
:1044F000A8283028280509090600FFF8A888888818
:104500008888A8F8050A0A0600FE205050505088F6
:10451000A8A8887003030306000340A04000060912
:1045200000FE070192032120FFFF08FF07FF0000A4
:1045300000060000010707060200808080808000DE
:1045400080030202060105A0A0050707060000502F
:1045500050F850F850500507070600002078A0706A
:1045600028F020050707060000C0C8102040981852
:104570000507070600006090A040A89068020303AA
:10458000060104C040800307070601002040808028
:104590008040200307070601008040202020408043
:1045A00005050506000120A870A8200505050600E0
:1045B000012020F820200203030602FFC0408005EE
:1045C0000101060003F8020202060200C0C0050550
:1045D000050600010810204080050707060000704E
:1045E00088888888887003070706010040C040401B
:1045F0004040E0050707060000708808708080F8DA
:10460000050707060000F81020100808F005070746
:1046100006000010305090F8101005070706000043
:10462000F880F00808887005070706000070808091
:10463000F0888870050707060000F8081020202081
:1046400020050707060000708888708888700507B5
:1046500007060000708888780808700205050602C1
:1046600000C0C000C0C00206060602FFC0C000C0F5
:1046700040800407070600001020408040201005FD
:104680000303060002F800F8040707060100804053
:1046900020102040800507070600007088081020C1
:1046A000002005070706000070880868A8A87005A4
:1046B0000707060000708888F888888805070706BD
:1046C0000000F08888F08888F00507070600007071
:1046D000888080808870050707060000F088888839
:1046E0008888F0050707060000F88080F08080F8D1
:1046F000050707060000F88080F080808005070726
:10470000060000708880B8888870050707060000DA
:10471000888888F8888888010707060200808080DA
:104720008080808005070706000038101010109068
:10473000600507070600008890A0C0A090880507C4
:1047400007060000808080808080F805070706004B
:104750000088D8A888888888050707060000888808
:10476000C8A8988888050707060000708888888888
:104770008870050707060000F08888F080808005B3
:10478000070706000070888888A890680507070654
:104790000000F08888F0A0908805070706000078E0
:1047A0008080700808F0050707060000F820202028
:1047B00020202005070706000088888888888870E0
:1047C00005070706000088888888885020050707A5
:1047D0000600008888888888A8500507070600001A
:1047E0008888502050888805070706000088888838
:1047F00050202020050707060000F8081020408000
:10480000F8030707060100E08080808080E005054E
:10481000050600018040201008030707060100E09C
:104820002020202020E005030306000420508805F6
:104830000101060000F8020202060205804005059B
:1048400005060000700878887805070706000080D4
:1048500080B0C88888F00505050600007080808853
:10486000700507070600000808689888887805051D
:10487000050600007088F880700507070600003004
:1048800048E0404040400506060600FF70888878F2
:1048900008700507070600008080B0C88888880176
:1048A00007070602008000808080808003080806D9
:1048B00001FF200020202020A04004070706000060
:1048C000808090A0C0A090030707060100C0404070
:1048D000404040E0050505060000D0A8A8A8A805AE
:1048E0000505060000B0C888888805050506000093
:1048F00070888888700506060600FFF08888F080BA
:10490000800506060600FF788888780808050505F2
:10491000060000B0C8808080050505060000708094
:104920007008F00407070600004040E040404030B7
:1049300005050506000088888898680505050600B5
:104940000088888850200505050600008888A8A8EA
:10495000500505050600008850205088050606060B
:1049600000FF888888780870050505060000F810A3
:104970002040F80307070601002040408040402007
:10498000010707060200808080808080800307077F
:1049900006010080404020404080050202060002DF
:1049A0006890000000060000000000060000000003
:1049B00000060000000000060000000000060000E5
:1049C00000000006000000000006000000000006D5
:1049D00000000000000600000000000600000000CB
:1049E00000060000000000060000000000060000B5
:1049F00000000006000000000006000000000006A5
:104A0000000000000006000000000006000000009A
:104A10000006000000000006000000000006000084
:104A20000000000600000000000600000000000674
:104A3000000000000006000000000006000000006A
:104A40000006000000000006000000000006000054
:104A50000000000600000000000600000000000644
:104A60000000000000060000000000060000010732
:104A7000070602008000808080808005070706000E
:104A8000002070A8A0A8702005070706000030408D
:104A900040E04050A8050505060000887050708869
:104AA000050707060000885020F820F820010707B6
:104AB00006020080808000808080050808060000D3
:104AC0003048205050209060030101060107A005E6
:104AD0000707060000F888B8B8B888F80507070681
:104AE0000001700878887800F8050505060001289F
:104AF00050A05028050303060001F808080202022E
:104B00000602064080050707060000F888A8889876
:104B1000A8F8050101060006F80404040600036075
:104B20009090600507070600002020F8202000F87C
:104B300004050506000360902040F003050506000B
:104B400003E020E020E002020206020640800508A1
:104B5000080600FF8888888898E88080050707068F
:104B6000000078989878181818020202060202C00D
:104B7000C00202020602FF40800305050600034052
:104B8000C04040E005070706000170888888700073
:104B9000F8050505060001A0502850A005070706E6
:104BA00000008890A858B808080507070600008884
:104BB00090B848982038050808060000C040C04852
:104BC000D838080805070706000020002040808824
:104BD000700508080600004020007088F8888805E5
:104BE00008080600001020007088F888880508086A
:104BF0000600002050007088F88888050808060024
:104C0000006890007088F888880508080600005041
:104C100000708888F8888805080806000020502061
:104C20007088F888880507070600003860A0B8E09B
:104C3000A0B80508080600FF708880808870206092
:104C4000050808060000402000F880F080F80508FC
:104C500008060000081000F880F080F80508080633
:104C60000000205000F880F080F8050707060000DB
:104C70005000F880F080F80308080601008040002A
:104C8000E0404040E0030808060100204000E0400A
:104C90004040E003080806010040A000E04040401A
:104CA000E0030707060100A000E0404040E00507E0
:104CB00007060000704848E84848700508080600E4
:104CC0000068900088C8A898880508080600004079
:104CD00020708888888870050808060000102070F9
:104CE00088888888700508080600002050007088B1
:104CF0008888700508080600006890007088888819
:104D000070050808060000500070888888887005C3
:104D1000050506000188502050880508080600FF98
:104D20001070A8A8A8A87040050808060000402038
:104D30008888888888700508080600001020888800
:104D40008888887005080806000020500088888838
:104D500088700508080600005000888888888870D8
:104D60000508080600001020885020202020050992
:104D7000090600FFC040704848704040E004080841
:104D80000601FF609090A09090E080050808060062
:104D90000040200070087888780508080600001098
:104DA0002000700878887805080806000020500068
:104DB0007008788878050808060000689000700878
:104DC0007888780507070600005000700878887812
:104DD000050808060000205020700878887805062D
:104DE00006060000D02878A0A8500506060600FF99
:104DF0007080887020600508080600004020007060
:104E000088F880700508080600001020007088F8F7
:104E100080700508080600002050007088F8807037
:104E200005070706000050007088F8807003080826
:104E300006010080400040C04040E0030808060131
:104E40000020400040C04040E00308080601004048
:104E5000A00040C04040E0030707060100A000405A
:104E6000C04040E0050707060000A040A010788879
:104E700070050808060000689000B0C8888888059A
:104E8000080806000040200070888888700508081F
:104E90000600001020007088888870050808060049
:104EA0000020500070888888700508080600006897
:104EB0009000708888887005070706000050007011
:104EC000888888700505050600012000F800200587
:104ED00007070600FF1070A8A8A87040050808067C
:104EE00000004020008888889868050808060000AF
:104EF000102000888888986805080806000020505F
:104F00000088888898680507070600005000888890
:104F10008898680509090600FF102000888888F82D
:104F200008700407070601FFC04060506040E005BC
:104F300008080600FF50008888887808705A0059D1
:104F400000580009200000000000000000000000E0
:104F500000007FFFE00000000000000000000000F3
:104F6000007000E0000000000000000000000000F1
:104F700061F8600000000000000000000000004137
:104F8000F82000000000000000000000000040F0D9
:104F90002000000000000000000000000040602031
:104FA0000000000000000000000000005801A07F89
:104FB00080000000000000004104005C63A0FFC00E
:104FC000000000000000002082005EF7A0FFC0008B
:104FD0000000000000002082005EF7A0FFC000007B
:104FE00000000000004104005C63A07F800000001E
:104FF000000000008208005801A07F80000000002F
:10500000000001041000406020FFC000000000000C
:10501000000104100040F020FFC00000000000006C
:105020000082080041F820FFC000000000000000DE
:1050300041040061F8603F00000000000000000033
:1050400000007000E01E0000000000000001FFFFF3
:10505000807FFFE00C0000000000000001FFFF80E7
:105060000000000000000000000000000000007FC1
:10507000FFE00000000000000000000000007000E1
:10508000E0000000000000000000000000630C6071
:10509000000000000000000000000000470E20009B
:1050A00000000000000000000000004F0F20000082
:1050B000000000000000000000005F0FA0000000E2
:1050C0000000000000000000005E07A07F800000DC
:1050D0000000000000410400406020FFC00000000C
:1050E0000000000020820040F020FFC0000000000F
:1050F00000000020820040F020FFC00000000000FF
:1051000000004104004060207F800000000000009B
:10511000008208005E07A07F800000000000000100
:105120000410005F0FA0FFC0000000000000010499
:1051300010004F0F20FFC000000000000000820898
:1051400000470E20FFC000000000000000410400E6
:10515000630C603F000000000000000000000070D1
:1051600000E01E0000000000000001FFFF807FFF44
:10517000E00C0000000000000001FFFF80000000C4
:10518000004D3234005072696E7420706175736521
:1051900064004D313235004D6F766520617869735A
:1051A0000044697361626C65207374657070657228
:1051B00073004D383400426564204C6576656C6937
:1051C0006E67004732382058590A4D313039205324
:1051D0003137350A473238205A0A4D31303920529A
:1051E0003134350A4731320A4732390A4D313034C9
:1051F000205330004175746F20686F6D6500473231
:1052000038004D61696E004D363030204230004D1F
:105210003234004D3233202573006175746F256977
:105220002E670043616E6E6F7420656E7465722028
:105230007375626469723A2000022E2E004D616916
:105240006E0045313A200045303A20005A3A20009D
:10525000593A2000583A20004D53312C4D533220FA
:1052600050696E730A002042002050006F6B00529C
:105270006573656E643A2000205A3A0020593A005E
:1052800020436F756E7420583A0020453A00205A2A
:105290003A0020593A00583A005A204F6666736522
:1052A0007400466C6F7700466C6F770046616E2025
:1052B000737065656420310046616E2073706565AA
:1052C0006420310042656400426564004E6F7A7A62
:1052D0006C65004E6F7A7A6C65005370656564008A
:1052E0005370656564004D61696E00416D617820A1
:1052F0004500416D6178204500416D6178205A007C
:10530000416D6178205A00416D6178205900416DEE
:105310006178205900416D6178205800416D6178B5
:10532000205800412D74726176656C00412D7472B5
:105330006176656C00412D72657472616374004121
:105340002D7265747261637400416363656C004122
:105350006363656C004D6F74696F6E00202F0020D1
:1053600042403A0020403A004E6F204C696E652062
:105370004E756D6265722077697468206368656335
:105380006B73756D2C204C617374204C696E653A9B
:10539000200053544F505045442E20005072696EE7
:1053A0007465722073746F70706564206475652015
:1053B000746F206572726F72732E20466978207444
:1053C0006865206572726F7220616E642075736506
:1053D000204D39393920746F20726573746172748D
:1053E0002E202854656D7065726174757265206930
:1053F000732072657365742E205365742069742060
:1054000061667465722072657374617274696E6727
:10541000290A004E6F20436865636B73756D2077B2
:10542000697468206C696E65206E756D6265722C9A
:10543000204C617374204C696E653A200063686586
:10544000636B73756D206D69736D617463682C2077
:105450004C617374204C696E653A20004C696E652E
:10546000204E756D626572206973206E6F74204CDA
:10547000617374204C696E65204E756D6265722B88
:10548000312C204C617374204C696E653A20004DBC
:10549000313130004D3331004D38342058205920FF
:1054A0005A20450053442072656164206572726F12
:1054B000720A00446F6E65207072696E74696E675F
:1054C0002066696C650A005761726E696E673A20E2
:1054D000486F6D696E672042756D7020446976690A
:1054E000736F72203C20310A000202040000A040C9
:1054F0000000A0400000004000009B430080A1434A
:10550000000087430000484200004842000040403D
:1055100000000000FF01FF5A2070726F6265206F6B
:1055200075742E206265640A005A2070726F62657D
:10553000206F75742E2062656400486F6D65205879
:10554000592066697273740A00486F6D6520585956
:1055500020666972737400436F6F6C646F776E00BE
:1055600046616E20737065656420310046616E206F
:1055700073706565642031004265640042656400B3
:105580004E6F7A7A6C65004E6F7A7A6C65004D6169
:10559000696E004E414E494E495459494E46CDCC54
:1055A000CC3D0AD7233C17B7D13877CC2B32959511
:1055B000E6241FB14F0A000020410000C84200400D
:1055C0001C4620BCBE4CCA1B0E5AAEC59D74D400EE
:1055D000E6B411241FBECFEFD1E2DEBFCDBF00E0A5
:1055E0000CBF14E0A0E0B2E0E6E0F0E402E00BBFA4
:1055F00002C007900D92A831B107D9F725E1A8E1C3
:10560000B4E001C01D92A531B207E1F715E5C0ED88
:10561000D5E500E006C022970109FE010BBF0F94FB
:10562000831FCE3CD10780E00807A9F70E9417949A
:105630000D94F21F0C9400002F923F924F925F92B4
:105640006F927F928F929F92AF92BF92CF92DF9292
:10565000EF92FF920F931F93CF93DF93CDB7DEB7F7
:10566000CE56D1090FB6F894DEBF0FBECDBF009164
:10567000170920E6029F800111240956184F8091D6
:10568000900680FF1AC0EEEDFAE184917F013FEFB2
:10569000E31AF30A811102C0780104C00E94AA46ED
:1056A000F701F3CFD7018D917D01882319F00E9476
:1056B000AA46F8CF8AE00E94AA4610925D06109290
:1056C0005C068FE380938F0610928E0610928D06F3
:1056D0001092320410923304109234041092350464
:1056E000F80180810F5F1F4F8032D1F38E34B1F407
:1056F000818190ED980F9A3020F08D3211F08B322D
:1057000069F43296DF0131962C9120532A30D0F380
:10571000CD01FC01019620812032D9F3F093870658
:10572000E09386067F01BFEFEB1AFB0A10816AE265
:1057300070E0C7010F94C31F009739F0DC01119787
:105740008C918032E1F311961C921D3429F01435AE
:1057500019F0173409F0CAC0F7014E2F9F2F81911D
:105760008032D9F380538A3008F0C0C010938F067E
:1057700020918D0630918E06E42FF92F6AE0AF015B
:105780004F5F5F4F629FC001639F900D1124208186
:1057900030E020533109820F931F218120532A309A
:1057A00030F090938E0680938D069A0103C09C0181
:1057B000FA01E5CFD9012F5F3F4F4C914032D1F331
:1057C0001D34D1F48E31910591F03CF4873191056F
:1057D00071F08C31910581F40AC08537910564F030
:1057E0008737910524F0803AE3E09E0729F4B093CF
:1057F0005D06A0935C067AC010925D0610925C066E
:10580000D090860641E050E0FD0131962C91222394
:1058100009F46CC02132A1F41D3491F48032910559
:1058200079F4F0935D06E0935C0663E270E0CF01EB
:105830000F94C31F009709F459C0DC011C9256C095
:105840000FEB020F0A31A0F59F01F90160812F5F74
:105850003F4F6032D1F320ED260F2A3040F023ED88
:10586000260F223020F06B3211F00C94993E9F01EC
:10587000602F70E0DB01B595A795B595A795B59517
:10588000A795AE5CBB4F07707A01002E01C0EE0CED
:105890000A94EAF7FC90FE28FC922115310511F0DC
:1058A0002D1901C020E0DB01A85EBB4F2C930AC07C
:1058B00020915C0630915D06232B21F4B0935D06A8
:1058C000A0935C06208121542A3110F4DF019CCF83
:1058D000DF0131966C9160536A30D0F39D01F9017C
:1058E0002F5F3F4F60816032D1F3F0CF80918F0600
:1058F0008D3409F4C7C4843511F40C94393E8734CF
:1059000011F00C947C3E80918D0690918E068A3128
:10591000910509F472C3A4F48430910544F48230F3
:1059200091050CF01CC197FF28C00C94963E843062
:10593000910509F4DBC20C9709F41DC30C94963E43
:105940008E31910509F4F8C33CF48C31910509F4CA
:10595000DDC30CF459C3DFC38B35910509F489C449
:105960008C35910509F48AC48A35910511F00C949F
:10597000963E10928C060C94963E8091630288238A
:1059800011F40C94963E0E94A44A86E394E00E948F
:10599000C0470E94364D8091900683FD8FC0C09015
:1059A0004204D0904304E0904404F09045042091D8
:1059B0007107309172074091730750917407C701C6
:1059C000B6010F945B18882309F478C080915F06B4
:1059D000811138C06091550270915602882777FD79
:1059E0008095982F0F9461189B01AC01609153062C
:1059F0007091540680915506909156060F945B184D
:105A000087FF20C0C0927107D0927207E09273079F
:105A1000F0927407EEEDFAE184918F010F5F1F4F52
:105A2000882321F00E94AA46F801F6CFEBEDF1E0C1
:105A300084918F010F5F1F4F882321F00E94AA4697
:105A4000F801F6CFC0904204D0904304E0904404A3
:105A5000F0904504209171073091720740917307CF
:105A600050917407C701B6010F948D1C20E030E0FF
:105A700048E453E40F94B41E181604F5C09271075D
:105A8000D0927207E0927307F0927407EEEDFAE19C
:105A900084918F010F5F1F4F882321F00E94AA4637
:105AA000F801F6CFECEBF1E084918F010F5F1F4F0F
:105AB000882321F00E94AA46F801F6CF20913604EF
:105AC0003091370440913804509139046091650752
:105AD0007091660780916707909168070F945B1833
:105AE00081111DC020913A0430913B0440913C0447
:105AF00050913D046091690770916A0780916B072E
:105B000090916C070F945B18811109C060910A0293
:105B100070910B0280910C0290910D021AC060915D
:105B2000A6027091A702882777FD8095982F0F9481
:105B3000611820910A0230910B0240910C025091A1
:105B40000D020F94C0182AE037ED43E25CE30F9496
:105B5000C0180E94DE7D0E941F480C94963E209142
:105B60006302222311F40C94963E11E0029709F08F
:105B700010E00E94A44A19821A821B821C821D8294
:105B80001E821F82188682E50E94BA49882309F482
:105B90005EC10E943E476B017C01209165073091F8
:105BA0006607409167075091680763962CAF3DAF39
:105BB0004EAF5FAF63978090690790906A07A0909F
:105BC0006B07B0906C078091360490913704A091D8
:105BD0003804B091390467968CAF9DAFAEAFBFAFBC
:105BE000679720913A0430913B0440913C045091D6
:105BF0003D046B962CAF3DAF4EAF5FAF6B9720E08F
:105C000030E0A901C701B6010F945B18882309F49D
:105C100034C163962CAD3DAD4EAD5FAD63976796D5
:105C20006CAD7DAD8EAD9FAD67970F945B18811104
:105C30000DC0A50194016B966CAD7DAD8EAD9FAD91
:105C40006B970F945B18882309F417C120E030E0AC
:105C5000A901C701B6010F945B18881F8827881F08
:105C6000181759F080E090E0A0E8BFEBAB968CAF3E
:105C70009DAFAEAFBFAFAB970AC020E030E040E8C9
:105C80005FE3AB962CAF3DAF4EAF5FAFAB97639684
:105C90002CAD3DAD4EAD5FAD639767966CAD7DAD00
:105CA0008EAD9FAD67970F948D1CA3966CAF7DAFA3
:105CB0008EAF9FAFA397A50194016B966CAD7DADA0
:105CC0008EAD9FAD6B970F948D1CA7966CAF7DAF7B
:105CD0008EAF9FAFA797A3962CAD3DAD4EAD5FADF8
:105CE000A397CA01B9010F94C0182B013C01A796D4
:105CF0002CAD3DAD4EAD5FADA797CA01B9010F9474
:105D0000C0189B01AC01C301B2010F948E1C0F940B
:105D1000F91E6F966CAF7DAF8EAF9FAF6F9720E08F
:105D200030E040E05FE30F94C0182B013C01A70175
:105D30009601C701B6010F94C0186B017C01A30145
:105D40009201C301B2010F94C0189B01AC01C701BD
:105D5000B6010F948D1C0F94F91E9B01AC01AB96FC
:105D60006CAD7DAD8EAD9FADAB970F94C0186B0140
:105D70007C0167962CAD3DAD4EAD5FAD67976396E8
:105D80006CAD7DAD8EAD9FAD63970F948E1C20E002
:105D900030E040E05FE30F94C0182B013C01A79670
:105DA0006CAD7DAD8EAD9FADA79790586F962CAD25
:105DB0003DAD4EAD5FAD6F970F946A1D9B01AC0179
:105DC000C701B6010F94C0189B01AC01C301B20119
:105DD0000F948E1C63962CAD3DAD4EAD5FAD6397B9
:105DE0000F948D1C69837A838B839C836B962CAD77
:105DF0003DAD4EAD5FAD6B97C501B4010F948E1CE8
:105E000020E030E040E05FE30F94C0182B013C013C
:105E10006F962CAD3DAD4EAD5FAD6F97A3966CAD5B
:105E20007DAD8EAD9FADA3970F946A1D9B01AC0114
:105E3000C701B6010F94C0189B01AC01C301B201A8
:105E40000F948E1CA50194010F948D1C12C089E43F
:105E50000E94BA49882331F00E943E4769837A83C1
:105E60008B839C838AE40E94BA49882331F00E9484
:105E70003E476D837E838F83988720E030E0A901C1
:105E800069817A818B819C810F945B1881110BC091
:105E900020E030E0A9016D817E818F8198850F948B
:105EA0005B18882349F0612FCE0101960E94F9EB1F
:105EB0000E94364D0C94963EE3EAFAE184918F01FC
:105EC0000F5F1F4F882321F00E94AA46F801F6CFEA
:105ED000E6EFF1E084918F010F5F1F4F882311F4EB
:105EE0000C94963E0E94AA46F801F4CF80E50E94E9
:105EF000BA49882329F00E94FE464B015C0103C089
:105F0000812C912C540183E50E94BA49882361F0C9
:105F10000E943E4720E030E04AE754E40F94C01866
:105F20000F94D71D4B015C010E949D7180910E0260
:105F3000811105C060E08CE092E00E949E840E9486
:105F4000364DC0904604D0904704E0904804F0904D
:105F50004904C80CD91CEA1CFB1C0E94A24C6C19F9
:105F60007D098E099F0997FD02C00C94963E80E042
:105F70000E94A9CDF2CF0E94DD6A81110C94963E59
:105F800080E50E94BA49882319F00E940E4701C09B
:105F900060E06FAF83E50E94BA49882319F00E9440
:105FA0000E4701C06CE06BAF84E50E94BA498823BC
:105FB00019F00E940E4701C063E068A382E50E94C9
:105FC000BA49882319F00E943E4704C060E070E09F
:105FD00080ED90E469837A838B839C839E01205EAD
:105FE0003F4FAE014F5F5F4FBE01655C7F4FCE01FB
:105FF000CF960E94DFF10C94963E81E0809363027D
:10600000109284060C94963E0E94DD6A81110C94D5
:10601000963E80E50E94BA49882321F00E940E47EF
:10602000462F01C040E060916D0770916E0780912E
:106030006F079091700700E010E020E231EC0983D7
:106040001A832B833C8300E010E822E933E40D83BC
:106050001E832F83388700E010E020EA31E40987AF
:106060001A872B873C8700E010E020EC3FE70D8784
:106070001E872F87388B413071F1423021F518A2ED
:1060800019A21AA21BA220E030E040EA51E40F94CA
:106090008E1C7B018C0120E030E047E853E40F9434
:1060A000B41E181624F4E12CF12C07E813E4A70120
:1060B000B8014BAF5CAF6DAF7EAFBE01605E7F4F8E
:1060C000CE01CB9611C020E030E040EA51E40F94BD
:1060D0005B1887FF0BC018A219A21AA21BA2BE014F
:1060E000605E7F4FCE0109960E94D8F118A219A2D6
:1060F0001AA21BA2AE01405E5F4FBE016B5F7F4FD5
:10610000CE0101960E94D4F10C94963E80E00F944B
:10611000770F0C94963E81E08093580724982C9A30
:106120000898109A0E94479D10925807249A2C981C
:10613000089A10980C94963E20E030E0A9016091F6
:1061400065077091660780916707909168070F94C3
:106150008E1C182F88E5AD966FAFAD97AE967FAFCA
:10616000AE97AF969FAFAF970E94BA49AD966FAD0D
:10617000AD97AE967FADAE97AF969FADAF978823A4
:1061800021F00E943E479B0102C09B01812FA90183
:10619000BC0148A359A36AA37BA320E030E0A90176
:1061A0006091690770916A0780916B0790916C0705
:1061B0000F948E1C5B018C0189E50E94BA498823EB
:1061C00021F00E943E475B018C01A501B801498383
:1061D0005A836B837C83409065065090660660907E
:1061E00067067090680620916106309162064091C2
:1061F00063065091640668A179A18AA19BA10F94BE
:106200008D1C6B017C012CE032E040EA51EC0F94D4
:10621000B41E87FF02C00C94963E21E230E041E9B3
:1062200053E4C701B6010F945B18181614F40C94CC
:10623000963EA3019201B501C8010F948D1C6B011C
:106240007C012CE032E040EA51EC0F94B41E87FF51
:1062500002C00C94963E21E230E847E953E4C701BE
:10626000B6010F945B18181614F40C94963E0C9417
:10627000AA3E81E080938C060C94963E0E9404F521
:106280000C94963E80918D0690918E0689379105EB
:1062900011F40C941D3A0CF0F0C08D34910509F402
:1062A0008BC50CF056C08931910509F4FAC21CF572
:1062B0008431910509F473C27CF48131910509F4AC
:1062C00063C22CF4029708F4DCC10C94963E42970A
:1062D00009F4FBC60C94963E8631910509F4A6C2DA
:1062E0000CF4A0C28731910509F4A6C2489709F4BD
:1062F000B9C20C94963E8F31910509F464C47CF4C4
:106300008B31910509F4E9C20CF4D9C28C319105A5
:1063100009F41FC34E9709F426C30C94963E8A32A3
:10632000910509F4F1C444F4809711F00C94963E61
:106330000E94BEF40C94963E8B34910509F439C545
:106340008C34910511F00C94963E0E94346C0C94A0
:10635000963E8B36910509F426C60CF04CC0853567
:10636000910509F4E7C67CF58235910509F4A6C6C6
:1063700004F58135910511F00C94963E0E94A75AC0
:106380000E949D710E9471471092FB101092FA10AA
:106390001092FD101092FC1068EE73E080E090E027
:1063A0000E949AE460E086EF93E00E949E840C9441
:1063B000963E8335910509F484C68435910509F428
:1063C00084C60C94963E8836910509F4F8C44CF4C2
:1063D0008C35910511F00C94963E0E942A790C940C
:1063E000963E8936910509F44EC58A36910509F421
:1063F000B7C50C94963E8337910509F49EC6D4F434
:106400008E36910509F428C534F48D36910509F4CA
:106410007BC50C94963E8F36910509F42EC58237C4
:10642000910511F00C94963E0E949D710F94880383
:106430000C94963E8637910509F410C774F485379D
:10644000910511F00C94963E60E080915C0690916D
:106450005D060E948E840C94963E8737910509F460
:1064600000C78837910511F00C94963E81E0809327
:10647000540780935E060C94963E803331E0930778
:1064800011F40C94C23A0CF077C08D3C910511F4D4
:106490000C94493AACF58E3B910509F44DC5ACF42A
:1064A0008C38910509F4ECC434F48D37910509F466
:1064B00090C50C94963E8139910509F4C3C78B3978
:1064C000910509F4FAC40C94963E893C910509F4AF
:1064D000BCC74CF4883C910511F00C94963E0E9488
:1064E000DB540C94963E8B3C910509F4CFC78C3C51
:1064F000910511F00C94963E0E9480520C94963EA9
:10650000823E910509F4CEC7DCF4833D910509F480
:10651000C3C74CF48E3C910511F00C94963E0E943A
:10652000147A0C94963E8C3D910509F4B8C78D3DC4
:10653000910511F00C94963E0E9428550C94963EBD
:106540008D3251E0950711F40C94BF3A34F48C323B
:10655000914009F4EBC70C94963E8E32E1E09E0721
:1065600011F40C94C53A8F32914011F00C94963E80
:106570000E9462C60C94963E853F21E0920711F47A
:106580000C94623C0CF044C0813941E0940711F452
:106590000C941B3BECF48F35A1E09A0711F40C949A
:1065A000BF3D3CF48E35914011F40C948E3D0C941B
:1065B000963E8336F1E09F0711F40C940E3E80392D
:1065C000914011F00C94963E0E949D710C94963E61
:1065D000843A31E0930711F40C941F3B54F4823950
:1065E000914011F00C94963E80E00E94E8F30C94E8
:1065F000963E8C3AA1E09A0711F40C94743B843FC8
:10660000914011F00C94963E0E949F8B0C94963E04
:106610008335E3E09E0711F40C946E3CB4F4873F9D
:1066200021E0920711F40C94683C14F40C94653C3E
:106630008C3142E0940711F40C946B3C8835924005
:1066400011F40C94713C0C94963E8C38A3E09A079C
:1066500011F40C94743D4CF48B38934011F00C946D
:10666000963E0E94765D0C94963E803AF3E09F073A
:1066700009F49CC2873E934011F40C94273E0C947D
:10668000963E00915C0610915D0680E50E94BA4935
:10669000882369F00E94FE466B017C01BB24B39401
:1066A000611571058105910531F4B12C04C0B12C3F
:1066B000C12CD12C760183E50E94BA498823F9F0D8
:1066C0000E943E4720E030E04AE754E40F94C018AF
:1066D0000F94D71D6B017C01B11013C061157105BA
:1066E0008105910571F40115110559F0D8018C91BE
:1066F000882339F061E0C8010E948E8407C0BB2066
:1067000091F360E08BE492E00E949E8481E08093AC
:1067100032090E949D710E94364DC114D104E104DA
:10672000F104D1F08090460490904704A090480472
:10673000B09049048C0C9D1CAE1CBF1C0E94A24C46
:10674000681979098A099B0997FF1AC08091320953
:1067500081110C94FF3E14C080913209882321F0EE
:1067600080E00E94A9CDF8CF80915E1260E088237E
:1067700019F08CE392E002C087E292E00E949E84CE
:10678000109232090C94963E60E08EE592E00E94F1
:106790009E8417981698159814980C94963EE6E7E0
:1067A000F2E084918F010F5F1F4F882321F00E9438
:1067B000AA46F801F6CF10920A1540E050E0BA015F
:1067C00086EB92E10E948C688BE1E6EBF2E1DE0160
:1067D000159601900D928A95E1F78091B4129091EF
:1067E000B5129C838B8384E293E09A83898340E093
:1067F00050E0BE016F5F7F4F83E893E00E94F86333
:10680000CE0101960E94F163E7E6F2E084918F01E8
:106810000F5F1F4F882311F40C94963E0E94AA46E6
:10682000F801F4CF0E94B1610C94963E10925E1272
:1068300010925F120C94963EE0915C06F0915D061A
:106840008081882329F0803209F410823196F8CFB4
:1068500040E061E080915C0690915D060E943CDE24
:106860000C94963E19821A821B821C8218A219A2CD
:106870001AA21BA280918306882341F040E0BE014A
:106880006F5F7F4FCE0180960E9417CB80915F1281
:10689000882319F081E080935E120E94BD6B0C94F6
:1068A000963E10925E120E94346C87E892E09093BC
:1068B000B7098093B6090E94ECFD0C94963E809136
:1068C0005F12882311F40C94963E83E50E94BA4926
:1068D00081110C94043F0C94963E80915F128823A2
:1068E00051F1ECE8F2E084918F010F5F1F4F882394
:1068F00021F00E94AA46F801F6CF6091011570912F
:10690000021580910315909104154AE00E94DE8AD9
:106910008FE20E94AA466091FD147091FE1480914E
:10692000FF14909100154AE00E94DE8A8AE00E94DE
:10693000AA460C94963EEEE9F2E084918F010F5F37
:106940001F4F882311F40C94963E0E94AA46F8012A
:10695000F4CF40E060E080915C0690915D060E947B
:106960003CDE0C94963E80915F12882311F40C94C7
:10697000963E80E594E10E94A25D80E594E10E944C
:106980009F6110925D1210925C12E0905C06F09094
:106990005D0680915F12882311F40C94963E0E944C
:1069A000A7611D8218861C821B8284E293E09A8371
:1069B000898382EB92E19093D2128093D112F701F6
:1069C00080818F3209F06BC06FE270E0C7010F94D5
:1069D000C31F8C010F5F1F4F9E012F5F3F4F590157
:1069E0000115110509F461C06FE270E0C8010F9450
:1069F000C31F6C01009709F459C00817190708F064
:106A000055C04C01801A910AA401B801CE018096AC
:106A10000F94E31FE0E2F0E0EC0FFD1FE80DF91D1D
:106A200010828E01005E1F4FD8018D918D01882349
:106A300019F00E94AA46F8CF8AE00E94AA46609107
:106A4000D1127091D2126115710519F06C5F7F4FF0
:106A500002C060E070E021E0AE01405E5F4FCE0119
:106A600005960E94FD62811112C0BE01605E7F4FDB
:106A700085ED92E00E94356F8EE20E94AA468AE080
:106A80000E94AA46C5010E94F1630C94963EB09202
:106A9000D212A092D11286010F5F1F4FA1CF83EDBA
:106AA00092E19093D2128093D11287016091D1121A
:106AB0007091D2126115710519F06C5F7F4F02C0A1
:106AC00060E070E018A21BA222E0A801CE0180962F
:106AD0000E94FD62F82E882311F1CE0180960E945B
:106AE000E05DF82E8823D9F06CA57DA58EA59FA525
:106AF00041E00E94E266F82E882389F0E8A9B0E21E
:106B0000EB9FF0011124E65BFB4F309739F085EEE7
:106B100080831BA20E94A466F82E01C0F12CCE0136
:106B200080960E94F862FF2011F19FEAE92E92E020
:106B3000F92EF7018491882331F0FFEFEF1AFF0A55
:106B40000E94AA46F6CFD8018D918D01882319F0B5
:106B50000E94AA46F8CF8AE00E94AA461092011528
:106B600010920215109203151092041519C08DEBA6
:106B7000E82E82E0F82EF7018491882331F0FFEFB0
:106B8000EF1AFF0A0E94AA46F6CFD8018D918D0117
:106B9000882319F00E94AA46F8CF8EE20E94AA46E6
:106BA000CE0101960E94F1630C94963E80915C06A2
:106BB00090915D0621E020935D1240E060E00E942C
:106BC0003CDE0C94963E0E94896B1CE3C12ED12CB6
:106BD000E12CF12CA70196010F94301C162F072FE2
:106BE000CA01B901A70196010F94301CD62EC72EF9
:106BF000CA01B90128E130E040E050E00F94301CB8
:106C0000FB01C9016DE671E00F94561F9B014D2DEC
:106C10005C2DDE0111967D012115310599F00F9350
:106C20001F93CF92DF92FF93EF939F938F933F93A6
:106C30002F9381E193E09F938F93FF92AF930F94F3
:106C4000F51712C00097B1F00F931F93CF92DF9208
:106C5000FF93EF939F938F9381E093E09F938F93A4
:106C6000FF92AF930F94F5170FB6F894DEBF0FBEE7
:106C7000CDBF30C0309779F00F931F93CF92DF9242
:106C8000FF93EF9385EF92E09F938F93FF92AF93E3
:106C90000F94F517E9CF452B69F00F931F93CF920F
:106CA000DF928DEE92E09F938F93FF92AF930F94BC
:106CB000F517DACF0F931F9389EE92E09F938F938E
:106CC000FF92AF930F94F5170F900F900F900F90C6
:106CD0000F900F9060E0C7010E948E84EEEDFAE104
:106CE00084918F010F5F1F4F882321F00E94AA46D5
:106CF000F801F6CFB70185E293E00E94356F8AE094
:106D00000E94AA460C94963E83E50E94BA498823C5
:106D100011F40C94963E0E941E47E82E80E50E94D6
:106D2000BA49811112C081E0E11001C080E0809376
:106D30005807882329F024982C9A0898109AF6C7A7
:106D4000249A2C98089A1098F1C780E50E94BA49B5
:106D5000882339F00E940E4777FF01C0E7C78B01F7
:106D600002C00DE010E0802FE2E3F3E09491891778
:106D700039F0319693E0EA35F907C1F70C94153FE5
:106D8000E3EAFAE184918F010F5F1F4F882321F01E
:106D90000E94AA46F801F6CFEAE5F3E084918F015C
:106DA0000F5F1F4F882309F4C1C70E94AA46F8014C
:106DB000F5CF0E94BD6BBAC70E94746BB7C788E657
:106DC00090E00E949B548111B1C78091900683FF8F
:106DD00001C0ACC783E50E94BA49882309F4A6C75D
:106DE0000E943E470F94D21D7093F20E6093F10EF5
:106DF00080E00E9450870E943E4720E030E040E75C
:106E000052E40F945B1818163CF00E94746B60E01B
:106E100085E793E00E949E840E943E47209153069E
:106E20003091540640915506509156060F94B41E69
:106E300018160CF07BC78EED92E09F938F9389E636
:106E400093E09F938F931F920E94C26A0F900F90BE
:106E50000F900F900F906AC78EE40E94BA49882362
:106E600009F464C70E940E4760934A0670934B066C
:106E700080934C0690934D0659C70E94C64956C749
:106E80000E9471BD53C789E690E00E949B54811116
:106E90000C946F42EAE8F3E084918F010F5F1F4F7B
:106EA000882321F00E94AA46F801F6CF0F94610DC5
:106EB0008AE00E94AA460C946F4283E50E94BA4978
:106EC000882309F433C70E941E47809352068D33EE
:106ED00018F08CE3809352060E94A24C6B017C0157
:106EE0002091520630E0A8EEB3E00F947E1CC60E4F
:106EF000D71EE81EF91EC0924E06D0924F06E092B1
:106F00005006F092510612C78DE690E00E949B5405
:106F100081110CC78091900683FD08C783E50E940C
:106F2000BA4960968FAF609781119CC782E50E9435
:106F3000BA49811197C7FAC68091900683FDF6C6BB
:106F400083E50E94BA4968968FAF689781110C94C7
:106F5000D14082E50E94BA4981110C94D140E6C625
:106F600083E50E94BA49882339F00E940E478B01BD
:106F70006F3F710519F010F00FEF10E080E50E94EF
:106F8000BA49882331F00E941E47823008F0CEC6ED
:106F900001C080E0E82FF0E0EE0FFF1FE650FF4E4B
:106FA00011830083C3C680E50E94BA49882339F063
:106FB0000E940E476230710508F0B8C602C060E05A
:106FC00070E0FB01EE0FFF1FE650FF4E11821082B2
:106FD000ADC68CE40E94C448882319F00E943E4745
:106FE00004C060E070E080E090EC27966CAF7DAF6D
:106FF0008EAF9FAF27978AE50E94BA49882319F080
:107000000E943E4703C060E070E0CB0120E030E02A
:1070100040E251E40F948E1C23966CAF7DAF8EAF8F
:107020009FAF239788E50E94BA49882319F00E94F0
:107030003E4703C060E070E0CB0120E030E040E27A
:1070400051E40F948E1C6BAF7CAF8DAF9EAF89E582
:107050000E94BA49882319F00E943E4703C060E0AD
:1070600070E0CB0120E030E847E953E40F948E1C38
:1070700020E030E040E251E40F948D1C68A379A336
:107080008AA39BA319821A821B821C828091830689
:1070900081114CC6C12CE12C8E010F5F1F4F9E0148
:1070A000205E3F4FAE01455C5F4FBE01615C7F4F8C
:1070B000CE018D5B9F4F0E943FCC38C610928B064D
:1070C00035C681E080938B0631C683E50E94BA49BC
:1070D000882399F00E943E4720E030E04AE754E4DC
:1070E0000F94C0180F94D71D6093510270935202F1
:1070F000809353029093540219C688E50E94C448B5
:1071000081110C94514289E50E94C44881110C946C
:1071100051428AE50E94C44881110C94514285E491
:107120000E94C44881110C9451420E949D710E949A
:107130007147FCC50E94A449F9C5E4EEF4E08491CE
:107140008F010F5F1F4F882321F00E94AA46F8018C
:10715000F6CFE6EDF4E084918F010F5F1F4F882397
:1071600021F00E94AA46F801F6CFEFEBF4E08491FB
:107170008F010F5F1F4F882321F00E94AA46F8015C
:10718000F6CFEFEAF4E084918F010F5F1F4F882361
:1071900021F00E94AA46F801F6CFEEE9F4E08491CE
:1071A0008F010F5F1F4F882321F00E94AA46F8012C
:1071B000F6CFEDE8F4E084918F010F5F1F4F882335
:1071C00021F00E94AA46F801F6CFEEE7F4E08491A0
:1071D0008F010F5F1F4F882321F00E94AA46F801FC
:1071E000F6CFE9E6F4E084918F010F5F1F4F88230B
:1071F00021F00E94AA46F801F6CFE3E5F4E084917D
:107200008F010F5F1F4F882321F00E94AA46F801CB
:10721000F6CFEEE3F4E084918F010F5F1F4F8823D8
:1072200021F00E94AA46F801F6CFE1E2F4E0849151
:107230008F010F5F1F4F882321F00E94AA46F8019B
:10724000F6CFE9E0F4E084918F010F5F1F4F8823B0
:1072500009F46CC50E94AA46F801F5CF0E94F248D5
:1072600065C581E08093580724982C9A0898109A55
:10727000E3E1F6E084918F010F5F1F4F882321F037
:107280000E94AA46F801F6CFEBE0F6E084918F0168
:107290000F5F1F4F882321F00E94AA46F801F6CF06
:1072A0001E9B03C009EF12E002C004EF12E0D801F8
:1072B0008D918D01882319F00E94AA46F8CF8AE0AB
:1072C0000E94AA46E3E0F6E084918F010F5F1F4F12
:1072D000882321F00E94AA46F801F6CF029903C044
:1072E00009EF12E002C004EF12E0F80181918F0172
:1072F000882319F00E94AA46F8CF8AE00E94AA4685
:10730000EBEFF5E084918F010F5F1F4F882321F091
:107310000E94AA46F801F6CF1D9B03C009EF12E0B8
:1073200002C004EF12E0D8018D918D01882319F07D
:107330000E94AA46F8CF8AE00E94AA46E3EFF5E051
:1073400084918F010F5F1F4F882321F00E94AA466E
:10735000F801F6CF019B03C009EF12E002C004EF71
:1073600012E0F80181918F01882319F00E94AA464A
:10737000F8CF8AE00E94AA46EBEEF5E084918F01F7
:107380000F5F1F4F882321F00E94AA46F801F6CF15
:107390001C9903C009EF12E002C004EF12E0D8010B
:1073A0008D918D01882319F00E94AA46F8CF8AE0BA
:1073B0000E94AA46E3EEF5E084918F010F5F1F4F14
:1073C000882321F00E94AA46F801F6CF379B03C01C
:1073D00009EF12E002C004EF12E0F80181918F0181
:1073E000882319F00E94AA46F8CF8AE00E94AA4694
:1073F000E9EDF5E084918F010F5F1F4F882321F0A5
:107400000E94AA46F801F6CF009903C009EF12E0E6
:1074100002C004EF12E0D8018D918D01882319F08C
:107420000E94AA46F8CF8AE00E94AA461092580706
:10743000249A2C98089A109879C4109254071092A4
:107440005E0674C40E942F4A71C40CE213E053E03C
:10745000E52E51E1F52EF80181918F010E94C4487B
:10746000882351F00E943E470F94D71DD7016D939A
:107470007D938D939C931397B4E0EB0EF11CE3E0A6
:1074800000331E0741F70E94344650C40E948749CA
:107490004DC40E9423494AC40E94815347C40E949C
:1074A0009A4A44C480E50E94C448882309F43EC433
:1074B0000E940E47F62E062F172F83E50E94BA4929
:1074C000882321F00E940E476B0103C0CC24CA948C
:1074D000DC2C96012F5F3F4F2330310508F026C486
:1074E00017FD24C40E949D71FFEFCF16DF0631F017
:1074F000CA94CD2871F000E010E00DC08F2D0E94DD
:107500003F4C31E020E0892B09F030E0032F122FAF
:1075100002C001E010E08F2D0E943F4C80179107C0
:1075200009F404C480E00E94A9CDF5CF83E50E9450
:10753000BA49882319F00E940E4702C064E071E046
:1075400079A368A380E50E94BA49882339F00E9494
:107550000E47693833E1730730F402C068EE73E018
:107560007A83698304C088E893E19A838983BE01A2
:10757000605E7F4FCE0101960E94ADE3D7C30E94AB
:10758000E552D4C30E941154D1C383E50E94C4487C
:10759000182F882371F00E943E470F94D21D7093DC
:1075A00056026093550221E0672B09F020E02093FA
:1075B0005F0680E50E94C448882369F080915502E7
:1075C00090915602892B19F00E942F4701C081E04B
:1075D00080935F06ABC31111A9C3EEEDFAE184916C
:1075E0008F010F5F1F4F882321F00E94AA46F801E8
:1075F000F6CF80915F06882319F066EF72E002C033
:1076000063E073E082E496E00E94356F609155027A
:107610007091560281E396E00E946A8BEDE2F6E0FB
:1076200084918F010F5F1F4F882309F47FC30E944D
:10763000AA46F801F5CF81E00E94E8F377C386E51A
:107640000E94C448882321F082E896E00F942D031D
:1076500083E50E94C448882321F00E942F47182FF9
:1076600001C010E083E50E94C448882319F0812FEF
:107670000E94B8BCF0906006111103C0EEEDFAE173
:107680001AC0F110FBCFE3EAFAE184918F010F5F9A
:107690001F4F882321F00E94AA46F801F6CFE3E6A7
:1076A000F6E084918F010F5F1F4F882339F30E940A
:1076B000AA46F801F6CF84918F010F5F1F4F8823F0
:1076C00021F00E94AA46F801F6CFFF2019F067E0EA
:1076D00073E002C06BE073E085E596E00E94356FD1
:1076E0008AE00E94AA4622C399E5892E97E0992E46
:1076F00025E6A22E27E0B22E39E7232E36E0332EE0
:1077000000E010E0422D409560964FAF6097D101A8
:107710008D911D01882309F4A3C0F501408051809B
:1077200062807380F801E95AFD4F208131814281E6
:107730005381F801E359F94F60817181828193810E
:107740000F948E1C20E030E040E05FE30F94C018FF
:107750009B01AC01C301B2010F94B41E181644F48E
:10776000F801E156F94FC590D590E590F49003C02B
:10777000C12CD12C7601F801EF59F94F20813181CC
:1077800042815381C301B2010F948D1C9B01AC0156
:10779000C701B6010F948D1C6B017C0120E030E025
:1077A00040EA51EC0F94B41E87FD2BC020E030E07E
:1077B00040EA51E4C701B6010F945B1818160CF1AA
:1077C000D4012D913D914D915C91C701B6010F946B
:1077D0008D1C9B01AC01C301B2010F948E1CF501FD
:1077E0006083718382839383D401CD92DD92ED9285
:1077F000FC92139760968FAD6097820D0E94294886
:107800002FC0E3EAFAE184918F010F5F1F4F8823B5
:1078100021F00E94AA46F801F6CFE9ECF6E0849147
:107820008F010F5F1F4F882321F00E94AA46F801A5
:10783000F6CF61E08BEB96E00E949E840E94178653
:1078400088E290E09A83898388EC90E099A388A3EA
:10785000BE016F5F7F4FCE0180960E94ADE366C28E
:10786000B4E08B0E911C0C5F1F4FE4E0AE0EB11C18
:107870000C30110509F04BCF0E94C3790F94880397
:1078800060E08BEA96E00E949E8483E992E099A3EF
:1078900088A304E610E01A830983BE01605E7F4F6F
:1078A000CE0101960E94ADE38AEB92E099A388A3F2
:1078B0001A830983BE01605E7F4FCE0101960E944C
:1078C000ADE334C20E94467431C20E9400732EC2DE
:1078D0000E9474522BC20E947F4928C20E94F14D1F
:1078E00025C20E94DD6A882319F081E00F94770F8A
:1078F00085E40E94C448882319F00E943E4704C0D2
:1079000060E070E080E090EC2F966CAF7DAF8EAFC2
:107910009FAF2F978AE50E94BA49882319F00E94E9
:107920003E4704C060E070E080E291E42B966CAFCB
:107930007DAF8EAF9FAF2B9788E50E94BA49882311
:1079400019F00E943E4704C060E070E080E291E4DC
:1079500027966CAF7DAF8EAF9FAF279789E50E94CA
:10796000BA49882319F00E943E4704C060E070E8DD
:1079700082E993E423966CAF7DAF8EAF9FAF2397E0
:1079800085E50E94C448882319F00E943E4704C040
:1079900060E070E088EC92EC6BAF7CAF8DAF9EAF97
:1079A0008CE40E94C448882319F00E943E4703C01B
:1079B00060E070E0CB0168A379A38AA39BA382E473
:1079C0000E94BA49882321F00E940E47F62E02C079
:1079D00085E0F82ED0904F128091830681117EC0F1
:1079E000CC24C394EF2C8E01055C1F4F9E01215CBB
:1079F0003F4FAE014D5B5F4FBE01695B7F4FCE01D4
:107A0000855B9F4F0E943FCC882309F467C081E0CB
:107A10008093320911E080913209882309F44AC029
:107A200060E08F2D0E9423E4809182068823F1F18B
:107A300010937D0640E050E0BA0180E098EB0E9490
:107A4000BF8580913209882321F081E00E94A9CD71
:107A5000F8CF10927E0610927F0610928006109248
:107A60008106109282060E9450870E94E9DB1093E3
:107A70007D0640E050E0BA0180E596EB0E94BF85AC
:107A80000E94A24C685370458F4F9F4F60937E06B3
:107A900070937F06809380069093810610928206F1
:107AA0001093320961E08F2D0E9423E481E00E944F
:107AB000A9CDB1CF00E010E028E432E409831A83B5
:107AC0002B833C8380918306882341F04F2DBE0198
:107AD0006F5F7F4FCE0180960E9417CBF1E0DF12DF
:107AE00025C10E94BD6B22C183E50E94BA4988234B
:107AF00021F00E940E478B0102C000E010E080E5FB
:107B00000E94BA49882321F00E940E47CB0102C08F
:107B100080E090E0B8010E94475D08C183E50E94C3
:107B2000C448811104C00CE213E0F12C0EC010E037
:107B30000E941E47682F812F40D71F5F1530C1F765
:107B4000F2CFF394B4E0FB1669F0D8018D918D016A
:107B50000E94C4488823A9F30E941E47682F8F2DD6
:107B60002CD7EFCF82E40E94C448882329F00E94DA
:107B70001E47682F84E021D70F941705D7C083E5EF
:107B80000E94BA49882309F446C00E941E478130EA
:107B900039F0823009F03FC00CE213E0F12C22C032
:107BA0000CE213E0F12CF80181918F010E94BA4997
:107BB000882331F00E941E474FEF682F8F2D53D638
:107BC000F394F4E0FF12EFCF82E40E94BA498823D5
:107BD00011F10E941E474FEF682F1BC0F394B4E0D1
:107BE000FB1671F0D8018D918D010E94BA4988234E
:107BF000A9F30E941E47482F6FEF8F2D34D6EECF8A
:107C000082E40E94BA49882331F00E941E47482F1F
:107C10006FEF84E028D60F94170588C0E3EAFAE1F5
:107C200084918F010F5F1F4F882321F00E94AA4685
:107C3000F801F6CFE7EEF6E084918F010F5F1F4F5A
:107C4000882309F473C00E94AA46F801F5CF81E0A9
:107C5000809363021092840683E50E94C4488111D8
:107C600003C00F94AD0462C00E942F4781115EC013
:107C7000F8CFF0908D06FF2039F1EEEDFAE1849116
:107C80008F010F5F1F4F882321F00E94AA46F80141
:107C9000F6CF84E50E94AA466F2D70E080E090E068
:107CA0004AE00E94DE8A80E20E94AA460FE013E0CA
:107CB000F80181918F01882319F00E94AA46F8CF1C
:107CC0008AE00E94AA4632C010928506EEEDFAE1E3
:107CD00084918F010F5F1F4F882321F00E94AA46D5
:107CE000F801F6CF60E070E086EF96E00E946A8BC4
:107CF0008AE00E94AA461AC0EEEDFAE184918F0153
:107D00000F5F1F4F882321F00E94AA46F801F6CF8B
:107D1000609186067091870688E097E00E94356F33
:107D200082E20E94AA468AE00E94AA460F94430477
:107D3000D6C320915C0630915D06232B39F49F0158
:107D40002150310930935D0620935C0620E030E03D
:107D50000C94382C80E00E94B8BC0E94594D83E5F9
:107D60000E94C448882309F448C00E942F4721E09C
:107D7000482FBE016F5F7F4FCE0180960E94E89929
:107D80006B017C019B01AC010F943A1F811130C043
:107D90002CEA35EC47E257E368A179A18AA19BA1BF
:107DA0000F948E1CAB01BC018FE192E00F946C0329
:107DB0002CEA35EC47E257E369817A818B819C811B
:107DC0000F948E1CAB01BC018AE192E00F946C030E
:107DD0002CEA35EC47E257E3C701B6010F948E1C3D
:107DE000AB01BC0185E192E00F946C038AE0B2D74D
:107DF0000E94404D0F94880399CF81E0B8CF80E076
:107E00000E94A9CD0C949E330E940E47AB01BC0189
:107E10004093011550930215609303157093041558
:107E200080E594E10E948C6881CF802F0E940B90A6
:107E30006E2D802F0E94684CF12CB701802F0E947C
:107E40002A900630110529F4F092FD10E092FC1002
:107E50006DCF0830110509F069CFF092FB10E09268
:107E6000FA1064CF0E943E470F94D21D7093F20E19
:107E70006093F10E80E00E9450870E943E4720E010
:107E800030E040E752E40F945B18181644F00E946B
:107E9000746B60E089EB93E00E949E8402C00E94B4
:107EA000BD6B6091F10E7091F20E882777FD809581
:107EB000982F0F94611820915306309154064091E9
:107EC0005506509156060F94B41E18160CF061C159
:107ED0008EED92E09F938F938DEA93E09F938F9323
:107EE0001F920E94C26A0F900F900F900F900F90F8
:107EF00081E08093890267961CAE1DAE1EAE1FAE58
:107F000067976F961CAE1DAE1EAE1FAE6F9710E04A
:107F1000A0961FAEA097ACE3A496AFAFA497BCE128
:107F2000A896BFAFA897E6E4AC96EFAFAC97C12C8C
:107F3000D12CA0E8EA2EBFEBFB2E812C912C540112
:107F40006091F10E7091F20E882777FD8095982F41
:107F50000F946118062F772E682E592E262F372F53
:107F6000482F592FB601C7010F945B188823D9F009
:107F70002091530630915406409155065091560673
:107F8000602F772D862D952D0F945B18182F111FBC
:107F90001127111F6096FFAD6097FF2341F0112359
:107FA00031F011E0E4C00C2D7D2C6E2C5F2C0E9472
:107FB000A24C6B017C01DC01CB016F962CAD3DAD79
:107FC0004EAD5FAD6F97821B930BA40BB50BB7FD46
:107FD00038C0D701C60188519C4FAF4FBF4F6F9635
:107FE0008CAF9DAFAEAFBFAF6F970F94610DE9EA55
:107FF000F3E084911F019FEF291A390A882319F0B1
:10800000A9D6F101F6CF81149104A104B104A9F01D
:10801000C501B40168517C4F8F4F9F4F6C197D098A
:108020008E099F0928EE33E040E050E00F94301CA9
:10803000CA01B9010E944F8B02C08FE38BD68AE040
:1080400089D680E00E94A9CD0E94364DA0915306AA
:108050006896AFAF689720905406309055064090D0
:1080600056062A2F322D432D542D602F772D862D25
:10807000952D0F948D1C9F7720E030E040E251E475
:1080800081149104A104B10429F40F945B1887FDB5
:1080900005C006C00F94B41E181614F4460157010B
:1080A000112309F44AC067962CAD3DAD4EAD5FADCE
:1080B0006797211531054105510541F0D701C601EA
:1080C000821B930BA40BB50BB7FD37C068962FAD81
:1080D0006897322D432D542DA0966FADA097A4968E
:1080E0007FADA497A8968FADA897AC969FADAC979F
:1080F0000F948D1C20E030E040EC5FE30F945B18A0
:1081000087FD4FCFD701C601805A9541AF4FBF4F72
:1081100067968CAF9DAFAEAFBFAF679768969FADC8
:108120006897A0969FAFA097A4962FAEA497A89605
:108130003FAEA897AC964FAEAC978091890288234A
:10814000B1F081149104A104B10429F4C02ED72CFC
:10815000E62CF52CF5CEA8EECA1AA3E0DA0AE1085F
:10816000F108C818D908EA08FB08F7FCEFCF80919E
:108170008902882309F4DACD60E0112329F08DE823
:1081800093E00E949E84D2CD8BE993E00E949E846E
:10819000CDCD6096FFAD6097F111AACE89EE92E049
:1081A00099CE6CD60F94D21D6739710514F066E92B
:1081B00070E07093EE0E6093ED0E0E9405875ED620
:1081C00020E030E040EA50E40F94B41E181614F496
:1081D0000E94BD6B6091ED0E7091EE0E882777FDC9
:1081E0008095982F0F94611820915706309158066A
:1081F0004091590650915A060F945B1860E087FF32
:1082000003C089EE93E002C08CED93E00E949E844F
:1082100081E0809389028091850680935B06679652
:108220001CAE1DAE1EAE1FAE67976F961CAE1DAE88
:108230001EAE1FAE6F9760961FAE6097A0961FAEE2
:10824000A097BCE3A496BFAFA497ECE1A896EFAFCC
:10825000A897F6E4AC96FFAFAC97C12CD12CE0E820
:10826000EE2EFFEBFF2E812C912C54016091ED0E30
:108270007091EE0E882777FD8095982F0F946118E6
:10828000162F072F782E692E262F372F482F592F7C
:10829000B601C7010F945B18882331F1209157066E
:1082A000309158064091590650915A06612F702F0F
:1082B000872D962D0F945B18881F8827881F60963E
:1082C0008FAF609768962FAD6897222389F0882337
:1082D00079F080918902882309F428CD60E08EEC42
:1082E00093E00E949E8422CD1C2D0D2D7E2C6F2CA0
:1082F0000E94A24C6B017C01DC01CB016F962CAD7E
:108300003DAD4EAD5FAD6F97821B930BA40BB50BCC
:10831000B7FD38C0D701C60188519C4FAF4FBF4F42
:108320006F968CAF9DAFAEAFBFAF6F970F94610DDF
:10833000E8EDF3E084912F019FEF491A590A882351
:1083400019F008D5F201F6CF81149104A104B1040B
:10835000A9F0C501B40168517C4F8F4F9F4F6C1934
:108360007D098E099F0928EE33E040E050E00F942C
:10837000301CCA01B9010E944F8B02C08FE3EAD4BE
:108380008AE0E8D480E00E94A9CD0E94364D20907A
:108390005706309058064090590650905A06910161
:1083A000A201612F702F872D962D0F948D1C9F7722
:1083B00020E030E040EA50E481149104A104B104CB
:1083C00029F40F945B1887FD05C006C00F94B41EF6
:1083D000181614F4460157016096AFAD6097AA23B2
:1083E00009F443C067962CAD3DAD4EAD5FAD6797C8
:1083F000211531054105510541F0D701C601821B08
:10840000930BA40BB50BB7FD30C09101A201A09650
:108410006FADA097A4967FADA497A8968FADA897AF
:10842000AC969FADAC970F948D1C20E030E040ECF3
:108430005FE30F945B1887FD4CCFD701C601805ACC
:108440009541AF4FBF4F67968CAF9DAFAEAFBFAFFB
:108450006797A0962FAEA097A4963FAEA497A89634
:108460004FAEA897AC965FAEAC97809189028823F7
:1084700009F42FCF81149104A104B10429F4C12E71
:10848000D02EE72CF62CF2CE98EEC91A93E0D90A3A
:10849000E108F108C818D908EA08FB08F7FE19CF67
:1084A000EECF0E949D7188E56FD6882319F0179A48
:1084B0001092550789E568D6882319F0169A10920C
:1084C00056078AE561D6882319F0159A1092570746
:1084D00085E45AD6882309F429CC01D527CCC25982
:1084E000DF4F0FB6F894DEBF0FBECDBFDF91CF9147
:1084F0001F910F91FF90EF90DF90CF90BF90AF90C2
:108500009F908F907F906F905F904F903F902F90B3
:108510000895CF93DF932FB7F89494E08902E00198
:108520001124FE01E455F14F6081718182819381B4
:108530002FBF0F946118C658D84F288139814A81BE
:108540005B810F94C018DF91CF910895CF92DF9295
:10855000EF92FF920F931F93CF93DF937C016A01F9
:10856000EB0100E010E00C151D0571F06991D701D9
:10857000ED91FC910190F081E02DC7011995892BB7
:1085800019F00F5F1F4FEFCFC801DF91CF911F91FF
:108590000F91FF90EF90DF90CF900895089580E0C5
:1085A00090E0089580E00895FC01E60FF11D8491AC
:1085B00090E0982F88273196E4918E0F911D0895B1
:1085C0000895DC011696ED91FC91179712968C9107
:1085D0001297481B15968C91483018F0E80FF11D42
:1085E0004770869586958695489F402D1124E40F07
:1085F000F11D362F377080E890E002C09595879581
:108600003A95E2F7669566956695E60FF11D30811D
:10861000222311F0832B02C0809583238083089549
:1086200081E00895089590E0FC013197E231F10571
:1086300008F04CC0EE58FF4F0D947D1F80918000D4
:108640008F7703C0809180008F7D80938000089594
:1086500080918000877FF9CF84B58F7702C084B581
:108660008F7D84BD08958091B0008F7703C0809185
:10867000B0008F7D8093B0000895809190008F7737
:1086800007C0809190008F7D03C080919000877F0C
:108690008093900008958091A0008F7707C080910B
:1086A000A0008F7D03C08091A000877F8093A000F1
:1086B0000895809120018F7707C0809120018F7DE0
:1086C00003C080912001877F8093200108953FB7E8
:1086D000F8948091281190912911A0912A11B091BC
:1086E0002B1126B5A89B05C02F3F19F00196A11D9F
:1086F000B11D3FBF6627782F892F9A2F620F711DFA
:10870000811D911D42E0660F771F881F991F4A95B2
:10871000D1F708954F925F926F927F928F929F92BE
:10872000AF92BF92CF92DF92EF92FF920F931F937F
:10873000CF93DF932C0125E437E081E090E0F9014D
:1087400045915491441655060CF062C0AC0141505D
:108750005109DA01AA0FBB1FAA0FBB1FAD5BB84FAF
:10876000FD0165917491440F551F440F551F4F5BD8
:10877000584FFA0165907490FC01EE0FFF1FEE0F49
:10878000FF1FED5BF84FA590B490FD01059114918A
:10879000F901C591D491FA0185909490882777FDCD
:1087A0008095982F0F9461186B017C01B2016619B6
:1087B0007709882777FD8095982F0F9461182B01F2
:1087C0003C01B501601B710B882777FD8095982FC0
:1087D0000F9461189B01AC01C301B2010F94C01842
:1087E0002B013C01BE0168197909882777FD809526
:1087F000982F0F9461189B01AC01C301B2010F9433
:108800006A1D9B01AC01C701B6010F948E1C11C0FB
:1088100001962C5F3F4F8032910509F090CFEFEB2E
:10882000F7E065917491882777FD8095982F0F94D4
:108830006118DF91CF911F910F91FF90EF90DF9022
:10884000CF90BF90AF909F908F907F906F905F90F0
:108850004F9008956091530670915406809155068B
:1088600090915606089567FD5CC0823021F128F48E
:10887000882349F0813069F054C0833071F184302D
:1088800009F43DC04EC0662311F0A19A8FC0A19893
:108890008DC09FB7662329F0F89480910801806805
:1088A00004C0F894809108018F77809308019FBFDE
:1088B00047FF4CC07FC09FB7662329F0F894809192
:1088C0000801806404C0F894809108018F7B809334
:1088D00008019FBF47FF40C06FC09FB7662329F0C4
:1088E000F89480910801886004C0F8948091080190
:1088F000877F809308019FBF47FF3EC05AC09FB744
:10890000662329F0F89480910801826004C0F894ED
:10891000809108018D7F809308019FBF47FF39C078
:108920004AC047FD49C08230B9F028F4882341F09D
:10893000813061F008958330F9F0843051F1089569
:10894000442311F0A09A0895A0980895442311F0AB
:10895000A29A0895A29808959FB7442329F0F89405
:1089600080910801806204C0F894809108018F7D95
:10897000809308019FBF08959FB7442329F0F8947E
:10898000809108018061F4CFF894809108018F7E76
:10899000EFCF9FB7442329F0F894809108018460B9
:1089A000E7CFF894809108018B7FE2CF47FFC8CFD3
:1089B00008950895089508950895643079F028F48D
:1089C000613041F0623041F00895683051F060311B
:1089D00041F0089540E003C040E004C041E060E0A1
:1089E00002C041E061E03FCFF894823041F5209130
:1089F0000901247015989FB7662329F0F894809197
:108A00000B01846004C0F89480910B018B7F8093EC
:108A10000B019FBF429A8BE090E00197F1F74298DB
:108A20009FB7222329F0F89480910B01846004C041
:108A3000F89480910B018B7F80930B019FBF7894FA
:108A4000089524E08202C0011124FC01E455F14F95
:108A50004081518162817381FC01E657F84F408368
:108A6000518362837383E091DF0EF091E00E82897F
:108A70009389A489B5898093BC0E9093BD0EA09371
:108A8000BE0EB093BF0E089580E043DD60932609CB
:108A900070932709809328099093290981E039DD93
:108AA00060932A0970932B0980932C0990932D09C8
:108AB00082E02FDD60932E0970932F098093300997
:108AC0009093310908958091DE0E9FB780FF09C011
:108AD000F89480910B018D7F80930B019FBF8FEFE6
:108AE00008C0F89480910B01826080930B019FBFB6
:108AF00081E080938A028091DE0E9FB781FF09C0DA
:108B0000F89480910B01816080930B019FBF8FEFE0
:108B100008C0F89480910B018E7F80930B019FBF5A
:108B200081E080938B028091DE0E9FB782FF09C0A7
:108B3000F89480910B018B7F80930B019FBF8FEF87
:108B400008C0F89480910B01846080930B019FBF53
:108B500081E080938C028091DE0E9FB783FF09C075
:108B6000F89480910B01806480930B019FBF8FEF7D
:108B700008C0F89480910B018F7B80930B019FBFFD
:108B800081E080938D0208954F925F926F927F9261
:108B9000AF92BF92CF92DF92EF92FF920F931F930B
:108BA000CF93DF938C01EB01FC0147A050A461A49B
:108BB00072A4AFA0B8A4C9A4DAA49501A601C30108
:108BC000B2010F945B1887FF40C0A3019201C3015B
:108BD000B2010F94C0182B013C01F80183A994A99C
:108BE000A5A9B6A9BC01CD0190589B01AC010F9479
:108BF0008E1CF80127A530A941A952A90F94C018CD
:108C00009B01AC01C301B2010F948D1C0F94F91E9E
:108C10007B018C019B01AC01B501C6010F945B186F
:108C200087FF02C0750186019701A801B501C60141
:108C30000F945B18882349F0A701B8014FA358A7E8
:108C400069A77AA7888181608883DF91CF911F917E
:108C50000F91FF90EF90DF90CF90BF90AF907F90FB
:108C60006F905F904F9008958F929F92AF92BF92B6
:108C7000CF92DF92EF92FF920F931F93CF93DF93E8
:108C800000D01F92CDB7DEB713E0812E11E1912EF7
:108C90000CEAA02E0FE0B02E0EEB16E0C12CD12C6A
:108CA0007601C394F40161917191819191914F0189
:108CB000F50121913191419151915F0129833A83CD
:108CC0004B835C830F945F1829813A814B815C81CF
:108CD0000F94C0180F94D71DF8016193719381937D
:108CE00091938F01C616D706E806F90610F46B01BA
:108CF0007C01F3E18F16F1E19F06A1F66FEF7FEFA4
:108D0000CB01A70196010F94301C2093600F309384
:108D1000610F4093620F5093630F0F900F900F906D
:108D20000F90DF91CF911F910F91FF90EF90DF9007
:108D3000CF90BF90AF909F908F9008958EBD0DB44F
:108D400007FEFDCF08958FEF8EBD0DB407FEFDCF5A
:108D50008EB508959091C00095FFFCCF8093C6001A
:108D60000895EF92FF921F93CF93DF931F92CDB799
:108D7000DEB7182FE7E4F8E084917F012FEFE21AC5
:108D8000F20A882329F09983E5DFF7019981F4CF6E
:108D9000E12FF92F84917F019FEFE91AF90A8823C7
:108DA00019F0D8DFF701F6CFEEE2F8E084917F0109
:108DB000AFEFEA1AFA0A882319F0CCDFF701F6CFF1
:108DC0000F90DF91CF911F91FF90EF9008953FB7E3
:108DD000F8942091B5098091B409821759F0E22FD7
:108DE000F0E0EC5CF64F808190E02F5F2F772093CE
:108DF000B50902C08FEF9FEF3FBF0895809197069E
:108E000090919806009731F04AE050E060E070E001
:108E10000D949B1660E070E0CB0108958091970659
:108E200090919806009731F04AE050E060E070E0E1
:108E30000D946A1560E070E0CB010895EFDF97FDB7
:108E40000CC0ECDF6F3F71058105910509F014F44A
:108E5000E5DF01C06FEF862F089580E008958091CF
:108E6000970690919806892B39F0E8DF91E08111FF
:108E700001C090E0892F089581E008951F93CF935A
:108E8000DF9380919706909198060097E1F0FC019E
:108E9000EF011191212F2F7D79F0153411F0153646
:108EA000B9F7188260E070E00F9402141883562F0F
:108EB000472F382F292F0BC060E070E0DF91CF9152
:108EC0001F910D94021450E040E030E020E0652F47
:108ED000742F832F922FDF91CF911F910895149AB1
:108EE0000895179A10925507169A10925607159AD8
:108EF00010925707F4CFCF92DF92EF92FF92C0907B
:108F0000CF06D090D006E090D106F090D2068091A6
:108F1000D306882321F120E030E0A901C701B60182
:108F20000F945B188823D9F020E030E040E05FE345
:108F3000C701B6010F94C0189B01AC010F94C01873
:108F40002BED3FE049E450E40F94C0189B01AC01C5
:108F500060E070E080E89FE30F946A1D04C060E069
:108F600070E080E89FE36093650F7093660F8093D5
:108F7000670F9093680FFF90EF90DF90CF90089568
:108F8000CF92DF92EF92FF92CF93DF93EC0180912B
:108F90007402882309F442C0C0905702D09058024E
:108FA000E0905902F0905A02A701960168817981F8
:108FB0008A819B810F94B41E181624F4C882D9822A
:108FC000EA82FB82C0905B02D0905C02E0905D027E
:108FD000F0905E02A70196016C817D818E819F8158
:108FE0000F94B41E181624F4CC82DD82EE82FF8228
:108FF000C0905F02D0906002E0906102F090620247
:10900000A7019601688579858A859B850F94B41E92
:10901000181624F4C886D986EA86FB86DF91CF919C
:10902000FF90EF90DF90CF90089580E1E5E6F7E0C4
:10903000A6E3B4E001900D928A95E1F7089580E1EE
:10904000E6E3F4E0A5E6B7E001900D928A95E1F73A
:109050000895AF92BF92CF92DF92EF92FF920F935B
:109060001F93CF93DF93C82FDD27C7FDD0958E01C7
:10907000000F111F000F111FF801E75AF84F20E0F1
:1090800030E0A90160817181828193810F948E1CEF
:10909000F801E656FE4E20813181428153810F94C2
:1090A0008E1C6B017C01F801EF59F94F60837183CD
:1090B000828393830552184FF801659175918591CC
:1090C00094918E01000F111F000F111F9801235959
:1090D000394F5901A70196010F948E1CF501608349
:1090E0007183828393830951184FF80165917591BB
:1090F00085919491CC0FDD1FCC0FDD1FC95ADD4F38
:10910000A70196010F948E1C688379838A839B83C1
:10911000DF91CF911F910F91FF90EF90DF90CF9053
:10912000BF90AF9008959091DB0FE92FF0E0EB58DE
:10913000F84F80839F5F943018F49093DB0F02C048
:109140001092DB0F809118098F5F809318090895A2
:10915000CF93FC01C62F80818B3399F08091180941
:10916000843078F42091DB0F30E6239FC001112476
:10917000BF018956984F0F94CE1F8C2FD4DF81E00A
:1091800001C080E0CF91089581548A3148F5482F7D
:1091900050E0FA0163E0F595E7956A95E1F7EE5C3A
:1091A000FB4F208130E0877002C0359527958A9566
:1091B000E2F720FF15C0FA01E85EFB4F2081222371
:1091C00039F08091860690918706820F911D02C02A
:1091D00080E090E0909398068093970681E0089550
:1091E00080E00895CF93DF9385E4CEDF882369F094
:1091F00036DE882351F0EEEDFAE18491EF012196FD
:10920000882319F0A7DDFE01F8CF81E4BDDF8823B4
:1092100069F025DE882351F0E3EFF7E08491EF0158
:109220002196882319F096DDFE01F8CFC0915C06E7
:10923000D0915D068991882311F08CDDFBCF8AE007
:10924000DF91CF9187CD83E59FDF882349F016DE3C
:109250006093970F7093980F8093990F90939A0F44
:1092600084E592DF882349F009DE6093930F7093C1
:10927000940F8093950F9093960F82E485DF882357
:1092800049F0BCDD6093E0067093E1068093E2064E
:109290009093E30688E578DF882349F0EFDD60935B
:1092A000C90F7093CA0F8093CB0F9093CC0F89E5B1
:1092B0006BDF882349F0E2DD6093CD0F7093CE0F12
:1092C0008093CF0F9093D00F8AE55EDF882349F01B
:1092D000D5DD6093D10F7093D20F8093D30F90930D
:1092E000D40F85E451DF882349F0C8DD6093D50FA2
:1092F0007093D60F8093D70F9093D80F089583E57E
:1093000043DF882319F0ABDD8093790708950F932D
:109310001F93CF93DF93CCE2D3E00BE91FE0899159
:1093200033DF882331F0AADDF80160837183828303
:1093300093830C5F1F4FF3E0C033DF0781F7DF91AA
:10934000CF911F910F91089583E51EDF882389F047
:1093500095DD20E030E04AE754E40F94C0180F9404
:10936000D71D6093580F7093590F80935A0F9093A5
:109370005B0F089509DF882339F081E0209197067B
:1093800030919806232B09F480E00895DF92EF9244
:10939000FF920F931F93CF93DF9383E5EBDF882337
:1093A00011F04CDD01C080E080939006EEEDFAE113
:1093B0008491EF012196882319F0CCDCFE01F8CFCF
:1093C000E7E2F8E08491EF012196882319F0C2DCEE
:1093D000FE01F8CF80919006882371F109E118E031
:1093E000C0E0D0E020E08091900690E00C2E02C01A
:1093F000959587950A94E2F780FF15C0DD24D394F4
:10940000D20E222311F08CE2A5DCF80125913491D3
:10941000F90184917901FFEFEF1AFF0A882321F007
:1094200099DC9701F5CFD22E21960E5F1F4FC530E4
:10943000D10561F02D2DD7CFE3E2F8E08491EF0163
:109440002196882319F086DCFE01F8CF8AE0DF91AF
:10945000CF911F910F91FF90EF90DF907BCCCF9336
:10946000DF9383E587DF882311F0D8DC02C060E05A
:1094700070E0EB01DD27C230D105A8F0E3EAFAE1A4
:109480008491EF012196882319F064DCFE01F8CF66
:10949000E7EFF7E08491EF012196882309F447C0B4
:1094A00059DCFE01F7CF88E465DF8823A1F0B6DC44
:1094B000683771053CF0633281E078072CF062E296
:1094C00071E002C068E770E0FE01EE0FFF1FE4529A
:1094D000F94F7183608386E44DDF882391F09EDC31
:1094E0006F3F710519F014F06FEF70E0FE01EE0FA1
:1094F000FF1FEC52F94F77FF02C060E070E071830C
:10950000608382E437DF882391F088DC6530710561
:1095100034F0683871052CF067E870E002C065E04F
:1095200070E0CC0FDD1FC852D94F79836883DF917B
:10953000CF91089583E51EDF882329F06FDC7093B7
:10954000A7026093A6020895CF92DF92EF92FF9256
:109550000F931F93CF93DF93CCE2EC2EC3E0FC2E4E
:1095600006E314E0C5E6D7E088E8C82E86E0D82EEA
:10957000F70181917F0108DE8823C9F07FDCF601C5
:109580002081211104C020918C06222329F02881FA
:1095900039814A815B8103C020E030E0A9010F944A
:1095A0008E1CF801608371838283938309C0888154
:1095B0009981AA81BB81F80180839183A283B383BF
:1095C0000C5F1F4F2496FFEFCF1ADF0A80E3E816E7
:1095D00083E0F80669F686E4CDDE8823B9F04EDC38
:1095E00020E030E0A9010F94B41E18167CF446DC8C
:1095F00020E030E040E752E40F946A1D60930A02D5
:1096000070930B0280930C0290930D02DF91CF9127
:109610001F910F91FF90EF90DF90CF900895809170
:109620002F1290913012891B8F7008958CE0E6E222
:10963000F9E0A5E6B7E001900D928A95E1F708956B
:109640000B96FC01849108950A96FC01849108957B
:1096500068E00C94D44266E00C94D442FC018491FE
:109660000895FCDF882311F0823011F486E008951C
:1096700083E00895FB014181DC0112962C91129741
:10968000421768F013962C911397241740F06081CD
:1096900015962C91621718F424810C94E1420895D8
:1096A000FC0120818281820F82839181891760F47D
:1096B00084818F5F84838381820F891710F08FEFFD
:1096C000890F838381E0089580E00895FC01128270
:1096D0008081815083831482089588E290E001970D
:1096E000F1F708952EE93FE0009729F0F90131974D
:1096F000F1F70197F9CF08950F93FC010150040F82
:1097000084A996A9941718F0081728F402C008171E
:1097100050F0041740F42150260F83A995A99617FD
:1097200020F4281720F480E007C0281720F481E0F7
:10973000261710F0F8CF81E00F910895DB01ED912D
:10974000FC911994EF92FF920F931F93CF93DF93A5
:109750001F92CDB7DEB78C01DC011296ED90FC9024
:109760001397D196ED91FC91D29782E0199520E064
:1097700030E04AE0B701C801E1DFF82ED801D19608
:10978000ED91FC91D29783E01995D801D196ED9196
:10979000FC91D29780E01995FF2081F1F801628158
:1097A00073819E012F5F3F4F46E4C801C7DF898167
:1097B000D8018C9312966D917C9113979E012F5F27
:1097C0003F4F47E4C801BADF8981F8018183628194
:1097D000738120E030E048E4C801B0DFD8011B9677
:1097E0008C931B9798012D5C3F4F12966D917C9145
:1097F000139747E1C801A2DF81E001C080E00F902C
:10980000DF91CF911F910F91FF90EF9008958F926C
:109810009F92AF92BF92CF92DF92EF92FF926B0135
:109820007C010E9467434B015C01C114D104E10437
:10983000F104E1F00E946743681979098A099B09DC
:10984000683E73408105910580F321E0C21AD1087A
:10985000E108F10888EE880E83E0981EA11CB11C77
:10986000C114D104E104F10429F7DFCFFF90EF9098
:10987000DF90CF90BF90AF909F908F900895CF933F
:10988000DF93282F30E0F901E550F84E8491F9017B
:10989000E258F74ED491F901EC53F74EC491CC2322
:1098A00091F081110E941343EC2FF0E0EE0FFF1FA7
:1098B000EF53F84FA591B4912C912D2381E090E0C6
:1098C00021F480E002C080E090E0DF91CF91089524
:1098D0000F931F93CF93DF931F92CDB7DEB7282F3F
:1098E00030E0F901E550F84E8491F901E258F74E65
:1098F0001491F901EC53F74E04910023C9F0882329
:1099000021F069830E9413436981E02FF0E0EE0F9C
:10991000FF1FEF51F84EA591B4919FB7F8948C9129
:10992000611103C01095812301C0812B8C939FBFCF
:109930000F90DF91CF911F910F91089561E0FC018D
:109940008081C6CF2FB7F89460912D1170912E11A0
:1099500080912F11909130112FBF08950F931F9375
:10996000CF93DF93EB01EEDF8B01EDD98F3F41F019
:10997000E9DF601B710B6C177D07B8F380E001C055
:1099800081E0DF91CF911F910F910895CF92DF92E7
:10999000FF920F931F93CF93DF9300D01F92CDB709
:1099A000DEB76C01F62EFC018281982F906A9695A5
:1099B0009CBD80FD06C091E0863009F490E0892FBF
:1099C00001C080E08DBD60E0F601808129833A838B
:1099D0004B835C837DDF6CE271E0C601BFDF8F2DBE
:1099E0008064ACD908E110E05C814B813A81298127
:1099F000DA01C901002E04C0B695A7959795879501
:109A00000A94D2F729833A834B835C8397D9085011
:109A1000110929813A814B815C81083FFFEF1F07C3
:109A200039F7FF2029F088E0F81621F08FEF03C006
:109A300085E901C087E882D9ECE0FE1201C083D934
:109A400010E081D9F601838387FF04C01F3F11F026
:109A50001F5FF7CF0F900F900F900F90DF91CF9176
:109A60001F910F91FF90DF90CF9008956BDF60936F
:109A700046047093470480934804909349040895E2
:109A80008091930690919406A0919506B0919606C8
:109A900080930A0290930B02A0930C02B0930D02E4
:109AA00080919106909192069093A7028093A602CE
:109AB000DDCF80910A0290910B02A0910C02B0912F
:109AC0000D028093930690939406A0939506B0930D
:109AD00096068091A6029091A70290939206809399
:109AE000910684E690E09093A7028093A602BECFF1
:109AF0008F929F92AF92BF92CF92DF92EF92FF929E
:109B0000CF93C82FC0906402D0906502E0906602A7
:109B1000F0906702A7019601C701B6010F943A1FA2
:109B20008090190990901A09A0901B09B0901C0907
:109B3000811129C0C11127C080916006882319F1C5
:109B4000A7019601C501B4010F948D1C2091B40F9B
:109B50003091B50F4091B60F5091B70F0F94C018C8
:109B60000F94BF1E719561957109809157078823E5
:109B700051F08091EB0E9091EC0E860F971F909311
:109B8000EC0E8093EB0E8092640290926502A0929C
:109B90006602B0926702CF91FF90EF90DF90CF9076
:109BA000BF90AF909F908F900895CF92DF92EF92E9
:109BB000FF92CF93DF936A017B01FC018491EF0157
:109BC0002196882319F0C6D8FE01F8CF42E0C701DC
:109BD000B601DF91CF91FF90EF90DF90CF900D9481
:109BE000B702CF92DF92EF92FF92EEEDFAE184910D
:109BF0007F019FEFE91AF90A882319F0ABD8F70122
:109C0000F6CFE6EDFBE084917F019FEFE91AF90AB8
:109C1000882319F09FD8F701F6CF8AE5B5DA8823B3
:109C2000B9F12CD96B017C0120E030E040E050EC30
:109C30000F94B41E87FD20C020E030E040EA50E4DD
:109C4000C701B6010F945B181816B4F0C092190939
:109C5000D0921A09E0921B09F0921C0980E048DFBB
:109C60006091190970911A0980911B0990911C0942
:109C700042E00F94B70217C0E1ECFBE084917F0152
:109C80009FEFE91AF90A882371F064D8F701F6CF3B
:109C90004091190950911A0960911B0970911C0992
:109CA0008EEB9BE082DF8AE0FF90EF90DF90CF9019
:109CB00051C8AF92BF92CF92DF92EF92FF920F9373
:109CC0001F93CF93C82F882319F0E6EAFBE00BC05F
:109CD000EEEDFAE184918F010F5F1F4F8823A9F306
:109CE00039D8F801F7CF84918F010F5F1F4F882378
:109CF00019F030D8F801F7CFCC2319F0E9E8FBE0F0
:109D00000BC0EEEDFAE184918F010F5F1F4F8823A6
:109D1000A9F320D8F801F7CF84918F010F5F1F4F6F
:109D2000882319F017D8F801F7CF8AE013D8C111AA
:109D30002CC0EEEDFAE184918F010F5F1F4F882355
:109D400019F008D8F801F7CFE6E7FBE084918F011E
:109D50000F5F1F4F882321F00E94AA46F801F6CF1B
:109D60008091D306882321F08AE00E94AA46AFC3DF
:109D7000EBE6FBE084918F010F5F1F4F882309F40E
:109D8000A6C30E94AA46F801F5CF4091CF06509194
:109D9000D0066091D1067091D20682E69BE005DF85
:109DA0008AE00E94AA468091D30681111BC0CC2371
:109DB00019F0E7E5FBE00CC0EEEDFAE184918F01CC
:109DC0000F5F1F4F8823A9F30E94AA46F801F6CF20
:109DD00084918F010F5F1F4F882321F00E94AA46B4
:109DE000F801F6CFC11124C0EEEDFAE184918F01A4
:109DF0000F5F1F4F882321F00E94AA46F801F6CF7B
:109E0000E6E4FBE084918F010F5F1F4F882321F070
:109E10000E94AA46F801F6CFEEEDFAE184918F0197
:109E20000F5F1F4F882321F00E94AA46F801F6CF4A
:109E30004091AC0F5091AD0F6091AE0F7091AF0F8C
:109E40008EE39BE0B2DE4091B00F5091B10F609174
:109E5000B20F7091B30F8BE39BE0A7DE4091B40F7C
:109E60005091B50F6091B60F7091B70F88E39BE0EA
:109E70009CDE4091B80F5091B90F6091BA0F70916C
:109E8000BB0F85E39BE091DE8AE00E94AA46C111E8
:109E900024C0EEEDFAE184918F010F5F1F4F8823FC
:109EA00021F00E94AA46F801F6CFE7E1FBE0849199
:109EB0008F010F5F1F4F882321F00E94AA46F801EF
:109EC000F6CFEEEDFAE184918F010F5F1F4F8823EB
:109ED00021F00E94AA46F801F6CF40919B0F5091C5
:109EE0009C0F60919D0F70919E0F8EE09BE05DDE58
:109EF00040919F0F5091A00F6091A10F7091A20F00
:109F00008BE09BE052DE4091A30F5091A40F609133
:109F1000A50F7091A60F88E09BE047DE4091A70F48
:109F20005091A80F6091A90F7091AA0F85E09BE056
:109F30003CDE8AE00E94AA46C11124C0EEEDFAE19F
:109F400084918F010F5F1F4F882321F00E94AA4642
:109F5000F801F6CFE3EEFAE084918F010F5F1F4F17
:109F6000882321F00E94AA46F801F6CFEEEDFAE12F
:109F700084918F010F5F1F4F882321F00E94AA4612
:109F8000F801F6CF40910311509104116091051131
:109F9000709106118AED9AE00E94838B409107111F
:109FA000509108116091091170910A1187ED9AE0A2
:109FB0000E94838B40910B1150910C1160910D11F7
:109FC00070910E1184ED9AE00E94838B40910F11E5
:109FD00050911011609111117091121181ED9AE060
:109FE0000E94838B8AE00E94AA46C11124C0EEED34
:109FF000FAE184918F010F5F1F4F882321F00E94A7
:10A00000AA46F801F6CFE7E8FAE084918F010F5FE6
:10A010001F4F882321F00E94AA46F801F6CFEEEDEB
:10A02000FAE184918F010F5F1F4F882321F00E9476
:10A03000AA46F801F6CF40911B1150911C11609176
:10A040001D1170911E118EE79AE0AFDD409117113E
:10A05000509118116091191170911A118BE79AE0C3
:10A06000A4DD40911311509114116091151170915C
:10A07000161188E79AE099DD8AE00E94AA46C1118C
:10A0800024C0EEEDFAE184918F010F5F1F4F88230A
:10A0900021F00E94AA46F801F6CFE4E0FAE08491AC
:10A0A0008F010F5F1F4F882321F00E94AA46F801FD
:10A0B000F6CFEEEDFAE184918F010F5F1F4F8823F9
:10A0C00021F00E94AA46F801F6CF4091970F5091D7
:10A0D000980F6091990F70919A0F8BEF99E065DD61
:10A0E0004091930F5091940F6091950F7091960F3E
:10A0F00088EF99E05ADD4091E0065091E1066091C9
:10A10000E2067091E30685EF99E00E94838B40910F
:10A11000C90F5091CA0F6091CB0F7091CC0F82EF95
:10A1200099E043DD4091CD0F5091CE0F6091CF0F5C
:10A130007091D00F8FEE99E038DD4091D10F5091A2
:10A14000D20F6091D30F7091D40F8CEE99E02DDD7A
:10A150004091D50F5091D60F6091D70F7091D80FC5
:10A1600089EE99E022DD8AE00E94AA46C11124C04E
:10A17000EEEDFAE184918F010F5F1F4F882321F0EC
:10A180000E94AA46F801F6CFEBEDF9E084918F0129
:10A190000F5F1F4F882321F00E94AA46F801F6CFD7
:10A1A000EEEDFAE184918F010F5F1F4F882321F0BC
:10A1B0000E94AA46F801F6CF4091590750915A07DC
:10A1C00060915B0770915C0782ED99E0EEDC409155
:10A1D0005D0750915E0760915F07709160078FEC9B
:10A1E00099E0E3DC40916107509162076091630759
:10A1F000709164078CEC99E0D8DC8AE00E94AA4652
:10A20000C11124C0EEEDFAE184918F010F5F1F4F61
:10A21000882321F00E94AA46F801F6CFE8EBF9E086
:10A2200084918F010F5F1F4F882321F00E94AA465F
:10A23000F801F6CFEEEDFAE184918F010F5F1F4F29
:10A24000882321F00E94AA46F801F6CF60916006AB
:10A2500070E08FEA99E00E946A8B8AE00E94AA4629
:10A26000CC2379F09CEDA92E96E0B92E28EDC22ED4
:10A2700026E0D22E34EDE32E36E0F32E00E010E09F
:10A2800024C0EEEDFAE184918F010F5F1F4F882308
:10A2900021F00E94AA46F801F6CFE2E9F9E08491A4
:10A2A0008F010F5F1F4F882321F00E94AA46F801FB
:10A2B000F6CFEEEDFAE184918F010F5F1F4F8823F7
:10A2C00089F20E94AA46F801F6CFB80189E899E020
:10A2D0000E946A8BF501619171915F0186E899E0B6
:10A2E0000E946A8BF601619171916F0183E899E098
:10A2F0000E946A8BF701619171917F0180E899E07A
:10A300000E946A8B8AE00E94AA460F5F1F4F0230AC
:10A310001105D9F6C11124C0EEEDFAE184918F0147
:10A320000F5F1F4F882321F00E94AA46F801F6CF45
:10A33000E1E7F9E084918F010F5F1F4F882321F03F
:10A340000E94AA46F801F6CFEEEDFAE184918F0162
:10A350000F5F1F4F882321F00E94AA46F801F6CF15
:10A360004091360F5091370F6091380F7091390F2F
:10A3700088E699E01ADC2CEA35EC47E25EE360916E
:10A38000320F7091330F8091340F9091350F0F94ED
:10A390006A1DAB01BC0185E699E00F946C032CEAC1
:10A3A00035EC47E25EE360912E0F70912F0F8091A4
:10A3B000300F9091310F0F94C018AB01BC0182E6B1
:10A3C00099E00F946C038AE00E94AA46C1110CC068
:10A3D000EEEDFAE184918F010F5F1F4F882321F08A
:10A3E0000E94AA46F801F6CF4091420F5091430FC8
:10A3F0006091440F7091450F89E599E0D6DB2CEA16
:10A4000035EC47E25EE360913E0F70913F0F809123
:10A41000400F9091410F0F946A1DAB01BC0186E57E
:10A4200099E00F946C032CEA35EC47E25EE360910F
:10A430003A0F70913B0F80913C0F90913D0F0F941C
:10A44000C018AB01BC0183E599E00F946C038AE06E
:10A450000E94AA46C11124C0EEEDFAE184918F0159
:10A460000F5F1F4F882321F00E94AA46F801F6CF04
:10A47000EDE3F9E084918F010F5F1F4F882321F0F6
:10A480000E94AA46F801F6CFEEEDFAE184918F0121
:10A490000F5F1F4F882321F00E94AA46F801F6CFD4
:10A4A0004091190950911A0960911B0970911C097A
:10A4B00084E399E07ADB8AE0CF911F910F91FF90BE
:10A4C000EF90DF90CF90BF90AF900C94AA46EEED46
:10A4D000FAE184918F010F5F1F4F882309F455CC57
:10A4E0000E94AA46F801F5CF83E50E94C44888235C
:10A4F00019F00E942F4701C081E091E08927D9CB54
:10A5000083E50E94C4488823D1F00E943E47AB01F6
:10A51000BC0140931B1150931C1160931D1170934B
:10A520001E114093131150931411609315117093E1
:10A5300016118CE099E039DB8AE00E94AA4680E59A
:10A540000E94C448882391F00E943E47AB01BC01A1
:10A5500040931B1150931C1160931D1170931E1199
:10A560008FEE98E022DB8AE00E94AA4682E50E94F4
:10A57000C448882391F00E943E47AB01BC01409340
:10A580001711509318116093191170931A1180EDDF
:10A5900098E00BDB8AE00E94AA4684E50E94C4484A
:10A5A000882391F00E943E47AB01BC0140931311F8
:10A5B00050931411609315117093161182EB98E06B
:10A5C000F4DA8AE00C94AA460895CF93DF9385E4E9
:10A5D0000E94BA49811110C080E50E94C4488823B6
:10A5E00091F00E943E476093360F7093370F80932F
:10A5F000380F9093390F07C00E941E47882361F3DC
:10A60000E3EAFAE16CC089E40E94C448882381F03F
:10A610000E943E472CEA35EC47E25EE30F94C018F7
:10A620006093320F7093330F8093340F9093350FF4
:10A6300084E40E94C448882381F00E943E472CEAAB
:10A6400035EC47E25EE30F946A1D60932E0F709322
:10A650002F0F8093300F9093310FEEEDFAE184913C
:10A66000EF012196882321F00E94AA46FE01F7CF30
:10A670004091360F5091370F6091380F7091390F1C
:10A680008EEA98E092DA2CEA35EC47E25EE36091DC
:10A69000320F7091330F8091340F9091350F0F94DA
:10A6A0006A1DAB01BC018AEA98E00F946C032CEAA6
:10A6B00035EC47E25EE360912E0F70912F0F809191
:10A6C000300F9091310F0F94C018AB01BC0186EA96
:10A6D00098E00F946C0310C00E94AA46FE0184917A
:10A6E000EF0121968111F8CFCFE0D3E08991882343
:10A6F00019F00E94AA46FACF8AE0DF91CF910C941C
:10A70000AA46CF93DF93EEEDFAE18491EF01219613
:10A71000882321F00E94AA46FE01F7CF83E50E941C
:10A72000C448882321F00E942F4780937402E6E9F1
:10A73000F8E08491EF012196882321F00E94AA4637
:10A74000FE01F7CF80917402882319F0EEE8F8E05B
:10A7500002C0E2E9F8E08491EF012196882321F01C
:10A760000E94AA46FE01F7CFE6E8F8E08491EF01E7
:10A770002196882321F00E94AA46FE01F7CF40913E
:10A780006D0650916E0660916F067091700684E8B8
:10A7900098E00BDA40917106509172066091730651
:10A7A0007091740681E898E000DA40917506509146
:10A7B000760660917706709178068EE798E0F5D975
:10A7C000E6E7F8E08491EF012196882321F00E94CA
:10A7D000AA46FE01F7CF409157025091580260916E
:10A7E000590270915A0284E798E0DFD940915B02E8
:10A7F00050915C0260915D0270915E0281E798E089
:10A80000D4D940915F0250916002609161027091D1
:10A8100062028EE698E0C9D98AE0DF91CF910C946C
:10A82000AA46CF93DF9380E50E94C448882351F065
:10A830000E943E476093420F7093430F8093440FF2
:10A840009093450F89E40E94C448882381F00E94B8
:10A850003E472CEA35EC47E25EE30F94C018609364
:10A860003E0F70933F0F8093400F9093410F84E40D
:10A870000E94C448882381F00E943E472CEA35ECB0
:10A8800047E25EE30F946A1D60933A0F70933B0FAB
:10A8900080933C0F90933D0FEEEDFAE18491EF0130
:10A8A0002196882321F00E94AA46FE01F7CF40910D
:10A8B000420F5091430F6091440F7091450F8AE60B
:10A8C00098E073D92CEA35EC47E25EE360913E0FE5
:10A8D00070913F0F8091400F9091410F0F946A1D2E
:10A8E000AB01BC0186E698E00F946C032CEA35ECD2
:10A8F00047E25EE360913A0F70913B0F80913C0F0D
:10A9000090913D0F0F94C018AB01BC0182E698E016
:10A910000F946C038AE0DF91CF910C94AA46BC019E
:10A9200080E090E04AE00E94DE8A8DE00E94AA4624
:10A930008AE00C94AA46FF920F931F93CF93DF9364
:10A94000EC0184E50E94BA49882351F10E941E4718
:10A95000F82E181614F5EEEDFAE184918F010F5FD1
:10A960001F4F882321F00E94AA46F801F6CF8DE4FC
:10A970000E94AA46BE0180E090E04AE00E94DE8A82
:10A980006F2D772767FD70958FE498E00E946A8BA2
:10A990008AE00E94AA4681E008C080935B0604C05A
:10A9A0008091850680935B0680E0DF91CF911F91B7
:10A9B0000F91FF900895CF93DF9388EC90E0BBDF79
:10A9C000811143C084E40E94C4488823D1F10E94CD
:10A9D0003E47C1E020E030E0A9010F945B188111EF
:10A9E00001C0C0E0C093D306CC2359F1C0915B06EF
:10A9F000D0E00E943E47FE01EE0FFF1FEE0FFF1F4B
:10AA0000E153F94F608371838283938320E030E0C8
:10AA1000A9016091CF067091D0068091D1069091E6
:10AA2000D2060F945B1881110CC080E090E0A0E486
:10AA3000B0E48093CF069093D006A093D106B09354
:10AA4000D206DF91CF910C947B47DF91CF9108958F
:10AA5000CF93DF938DED90E06EDF811111C083E520
:10AA60000E94BA49882361F0C0915B06D0E00E9441
:10AA70000E47FE01EE0FFF1FEC55FD4F7183608303
:10AA8000DF91CF910895CF93DF93C0912814CC2309
:10AA9000C1F0C150C09328148FE1C89FE001112478
:10AAA000CE50DD4E8BE1FE013496A7EDB2E1019070
:10AAB0000D928A95E1F78A819B819093D6128093BB
:10AAC000D5121092201181E08093211183E08093B0
:10AAD000A802DF91CF910895CF92DF92EF92FF927B
:10AAE0000F931F93CF93DF93EC010E94A24C0E8132
:10AAF0001F8128853985011511052105310559F575
:10AB00003C853323A9F12A8531503C8731E0320F4F
:10AB10003A874D85341301C01A86FE0134E0239F25
:10AB2000E00DF11D112406851785208931890A83DE
:10AB30001B832C833D836B017C01C00ED11EE11C65
:10AB4000F11CCE82DF82E886F9868C819D81892B7B
:10AB500079F0769A0DC06B017C01C01AD10AE20A25
:10AB6000F30AF7FC05C076981E821F8218861986A4
:10AB7000DF91CF911F910F91FF90EF90DF90CF90D9
:10AB800008958F929F92BF92CF92DF92EF92FF92A1
:10AB90000F931F93CF93DF931F92CDB7DEB74C0176
:10ABA000D62EE42E522FF22EC62EC20EBB24BA94FD
:10ABB0008C01045E1F4F2C2D2F1987E08F1588F410
:10ABC000F40162817381248FE58E178EB68E980111
:10ABD0004BE3C40159830E949E4BF8EFFF0E59814D
:10ABE000EACF852F887F8D0D577021F137E035270B
:10ABF000F40162817381848FE58E178E3F5F377019
:10AC00008FEF90E001C0880F3A95EAF7868F9401A4
:10AC1000245E3F4F4BE3C4010F90DF91CF911F9112
:10AC20000F91FF90EF90DF90CF90BF909F908F900B
:10AC30000C949E4B0F90DF91CF911F910F91FF903D
:10AC4000EF90DF90CF90BF909F908F900895EF92FC
:10AC5000FF920F931F93CF93DF93EC01F62EE22E1A
:10AC6000142F040F2E2D412F6F2DCE018ADF1F5F71
:10AC70000113F8CFDF91CF911F910F91FF90EF90CB
:10AC80000895DF92EF92FF920F931F93CF93DF937C
:10AC9000EC01162FF42EE22E0E947C4B882329F023
:10ACA0002E2D4F2D612FCE01D2DFDF91CF911F913D
:10ACB0000F91FF90EF90DF9008950F934CE0849FE9
:10ACC000402D1124E1E0E40FE093900F2CE0240FDD
:10ACD0002093910FA091E111B0E030E02E5F3F4F43
:10ACE0002A173B07FCF0F0E02091E31130E0E21777
:10ACF000F307C4F4662369F081E08093CD114D5FC2
:10AD00000BE020E860E08DEA91E1BBDF1092CD110D
:10AD100003C081E08093CD118091910F1092E411D6
:10AD20008093E5110F910895AF92BF92DF92EF9259
:10AD3000FF920F931F93CF93DF931F92CDB7DEB790
:10AD40005B01622F4983B9DF9091E1118091910FEE
:10AD50004981891708F443C09091E3118091900FC5
:10AD6000981708F43CC041110FC086E1F82E1F145B
:10AD700024F4F501849181112BC01F1484F580E225
:10AD80000E949491FA94F9CF20E030E0F501E20FAF
:10AD9000F31FE491EE2319F02F5F3F4FF7CF86E1C9
:10ADA00090E0821B930B97FD019695958795E82E71
:10ADB00000E010E036E1D32EFD2CF01A0F5F1F4F9C
:10ADC0008E2D801B87FDD3CF80E20E949491F4CF1B
:10ADD0000E949F91F81AFFEFAF1ABF0AC8CF0F90D9
:10ADE000DF91CF911F910F91FF90EF90DF90BF9077
:10ADF000AF900895EF92FF920F931F93CF93DF933D
:10AE00001F92CDB7DEB7182F062F682F802F4983EA
:10AE100054DF9091E1118091910F4981891708F4D5
:10AE20005AC09091E3118091900F981708F453C085
:10AE300080916E12882309F44BC0112371F1602FA9
:10AE400080E0E82FF0E0E45AFD4E9581992329F047
:10AE5000660F611D69278F5FF4CF80919A06861770
:10AE6000B1F0EEE6F2E120E030E08191882319F0C4
:10AE70002F5F3F4FFACF2531310514F0255101C026
:10AE800020E02093AD0660939A061092AE060091E2
:10AE9000AE0610E002591D4E02C00EE612E1442338
:10AEA00019F082E00E94B391780115E1F7018191D8
:10AEB0007F01882331F0112321F00E949F91181BFC
:10AEC000F5CF112341F080E20E9494911150F9CF07
:10AED00001E612E1E4CF0F90DF91CF911F910F9126
:10AEE000FF90EF9008950F931F93CF93DF93982FC8
:10AEF000862FEA01022F692FE0DE9091E111809107
:10AF0000910F891750F19091E3118091900F98174C
:10AF100020F114E1FE018491811102C0C12F05C00E
:10AF20000E949F91181B2196F5CFCC2329F080E237
:10AF30000E949491C150F9CF8091910F9AE790931C
:10AF4000E4118093E511802F0E94B39180E2DF919C
:10AF5000CF911F910F910C949491DF91CF911F91FC
:10AF60000F9108950F931F93CF93DF93082F709342
:10AF70009D0660939C061092271180912311909159
:10AF80002411A0912511B091261181309048A1057E
:10AF9000B10540F010922311109224111092251146
:10AFA00010922611C091231140919B061416D4F4DF
:10AFB000842F992787FD909501972C2F332727FD04
:10AFC00030952817390774F0CFEFC40F8C2F90E01D
:10AFD000A0E0B0E08093231190932411A093251159
:10AFE000B09326111092211180912011C81714F4EA
:10AFF000C093201180912011992787FD9095049688
:10B000002C2F332727FD30958217930724F48CEFDC
:10B010008C0F8093201110912011D0E081E001303D
:10B0200049F1023009F44BC001116EC0111193C0F7
:10B030008823B1F01C16A4F0809123119091241163
:10B04000A0912511B09126110196A11DB11D8093EB
:10B05000231190932411A0932511B0932611CF5F53
:10B060008091A802882309F4EFC021E041E066E462
:10B070007CE06EC011116FC08823B9F01C16ACF0D3
:10B080004091231150912411609125117091261146
:10B090004F5F5F4F6F4F7F4F4093231150932411A9
:10B0A0006093251170932611CF5F8091A8028823A9
:10B0B00009F4CAC021E041E06FE37CE049C011110E
:10B0C0004AC08823B9F01C16ACF04091231150916E
:10B0D000241160912511709126114F5F5F4F6F4FC2
:10B0E0007F4F409323115093241160932511709347
:10B0F0002611CF5F8091A802882309F4A5C021E022
:10B1000041E068E37CE024C0111125C08823B9F038
:10B110001C16ACF04091231150912411609125111F
:10B12000709126114F5F5F4F6F4F7F4F40932311F8
:10B13000509324116093251170932611CF5F809155
:10B14000A802882309F480C021E041E06FE27CE09E
:10B150008D2FEADD79C01130D9F480911F11811152
:10B1600006C08091A802882309F46EC009C0C130CE
:10B17000C1F70E941D8680912111882391F36CC034
:10B1800081E0C13009F080E024E045E25CE05AC093
:10B190001230E9F480911F11811106C08091A8023C
:10B1A000882309F451C00BC0C230C1F782E196E890
:10B1B0000E94E28580912111882381F34DC081E0B6
:10B1C000C23009F080E023E04BE15CE03BC013308B
:10B1D000E1F480911F11811105C08091A80288239C
:10B1E00099F10BC0C330C9F78DE096E80E94E28563
:10B1F00080912111882389F32FC081E0C33009F0A9
:10B2000080E023E042E15CE01DC01430E9F480916D
:10B210001F11811105C08091A8028823A9F00BC0DD
:10B22000C430C9F788E096E80E94E2858091211138
:10B23000882389F311C081E0C43009F080E023E065
:10B2400047E05CE06D2F4FDEDF5F1F5FD53011F010
:10B2500080E0E5CED0939B06DF91CF911F910F91B7
:10B2600008951F93CF93DF9310922711809123119C
:10B2700090912411A0912511B09126118130904810
:10B28000A105B10540F010922311109224111092E3
:10B29000251110922611C091231140919906141680
:10B2A000D4F4842F992787FD909501972C2F33276D
:10B2B00027FD30952817390774F0CFEFC40F8C2F76
:10B2C00090E0A0E0B0E08093231190932411A0932C
:10B2D0002511B09326111092211180912011C817C9
:10B2E00014F4C093201180912011992787FD909527
:10B2F00004962C2F332727FD30958217930724F4CB
:10B300008CEF8C0F8093201110912011D0E011113F
:10B310001AC080911F11811106C08091A802882354
:10B3200009F48CC009C0C111F8CF0E941D8680911C
:10B330002111882391F389C081E0C11180E024E0CC
:10B340004EEF5BE079C01130E9F480911F1181115B
:10B3500006C08091A802882309F470C00BC0C130D8
:10B36000C1F78AE59BEB0E94E28580912111882339
:10B3700081F36BC081E0C13009F080E023E047EF4A
:10B380005BE05AC01230E9F480911F11811106C0B0
:10B390008091A802882309F451C00BC0C230C1F7C4
:10B3A00085E59BEB0E94E28580912111882381F342
:10B3B0004CC081E0C23009F080E023E040EF5BE068
:10B3C0003BC01330E1F480911F11811105C08091C1
:10B3D000A802882399F10BC0C330C9F780E59BEB25
:10B3E0000E94E28580912111882389F32EC081E09B
:10B3F000C33009F080E023E049EE5BE01DC014306B
:10B40000E9F480911F11811105C08091A802882361
:10B41000A9F00BC0C430C9F78BE49BEB0E94E28516
:10B4200080912111882389F310C081E0C43009F094
:10B4300080E023E040EE5BE06D2F55DDDF5F1F5FB6
:10B44000D53009F064CFD0939906DF91CF911F9149
:10B4500008950F931F93CF93DF938C01EB01DC01D1
:10B4600013968C918823C1F18250823028F48FE2A8
:10B470008883198281E031C0F801648575858685ED
:10B48000978540E00E94E266882339F1D801509602
:10B49000EC91B0E2EB9FF0011124E65BFB4F30979B
:10B4A000D9F090E020E03EE24081403269F028305F
:10B4B00029F4DE01A90FB11D3C939F5F4081DE019D
:10B4C000A90FB11D4C939F5F2F5F31962B3061F711
:10B4D000C90FD11D188201C080E0DF91CF911F916B
:10B4E0000F910895CF93DF938091E611811107C0EA
:10B4F00081E08093E6118DEA91E10E94A24BC09118
:10B50000AF11D091B011E091DE11F091DF1182E026
:10B510001995E091DE11F091DF1181E0199520E09D
:10B5200030E044E1BE018DEA91E10E949E4B20EEA5
:10B5300031E147E1BE018DEA91E10E949E4BE0912D
:10B54000DE11F091DF1180E0DF91CF91199410921C
:10B55000F20E1092F10E80E00E9450871092EE0ED3
:10B560001092ED0E0E9405870E94746B1092F20EED
:10B570001092F10E80E00E9450871092070F9FB743
:10B58000F894E2E0F1E080818F7B80839FBF10928E
:10B59000EE0E1092ED0E1092050F75980895109210
:10B5A000FB101092FA101092FD101092FC10CFDFD9
:10B5B0000C94178690912F1280913012981731F0C9
:10B5C000809130128F5F8F708093301208950F93A7
:10B5D0001F93CF93DF93EC01FC01E65AFF4F1082DB
:10B5E000138234971382128284E293E091838083E2
:10B5F000B5961082138234971382128291838083CE
:10B600008E010A561F4F9E0124533E4FF801B80188
:10B610006C5F7F4FAC01CF01801B910B860F971F92
:10B62000DC011C9213961C92138212825183408378
:10B630007F96E217F30779F7CE0183539E4F29E1F6
:10B64000DC0111962C93119714961C920596DC013F
:10B6500057961C928296DC011C9213961C920497BA
:10B66000DC0113961C921E92129724E233E02D9374
:10B670003C93198218821B821A828F549F4FDC01DF
:10B680001D921D921D921C9213970496DC011D922F
:10B690001D921D921C9213971082FE01E15FFD4FD7
:10B6A000108286E391E0F8019C0111922150304014
:10B6B000E1F7FE01E355FD4F81E08083E955F2405B
:10B6C000118210820E94A24CC755DD4F68577C4EF4
:10B6D0008F4F9F4F688379838A839B83DF91CF91BC
:10B6E0001F910F9108952F923F924F925F926F9208
:10B6F0007F928F929F92AF92BF92CF92DF92EF9202
:10B70000FF920F931F93CF93DF93CDB7DEB7689768
:10B710000FB6F894DEBF0FBECDBF1C015B018A01DE
:10B72000DC01D7966D917D918D919C91DA970F9464
:10B730005F186B017C01F5012081318142815381C9
:10B740000F94C0180F94541D0F94D71D69877A87E2
:10B750008B879C87D8012D913D914D915C91C701BC
:10B76000B6010F94C0180F94541D0F94D71D6D8708
:10B770007E878F87988B29853A854B855C8528370E
:10B7800031054105510540F488E790E0A0E0B0E0C4
:10B7900089879A87AB87BC872D853E854F855889D9
:10B7A000283731054105510540F488E790E0A0E0D5
:10B7B000B0E08D879E87AF87B88B91012D5B3F4F9F
:10B7C000D9018D919D910D90BC91A02D8D839E836B
:10B7D000AF83B887BC01CD010F94611869837A8368
:10B7E0008B839C8369857A858B859C850F945F18F4
:10B7F000698B7A8B8B8B9C8B20E030E0A90169816F
:10B800007A818B819C810F945B18882339F1A70181
:10B810009601C701B6010F94C0184B015C0129893C
:10B820003A894B895C89CA01B9010F94C0189B0100
:10B83000AC01C501B4010F948D1C4B015C01298141
:10B840003A814B815C81CA01B9010F948E1C9B0126
:10B85000AC01C501B4010F946A1D03C060E070E043
:10B86000CB010F94541D0F94D21D2B013C016D810F
:10B870007E818F81988590958095709561957F4F99
:10B880008F4F9F4F0F9461184B015C016D857E8532
:10B890008F8598890F945F186D837E838F83988737
:10B8A00020E030E0A901C501B4010F945B188823A2
:10B8B00049F12D813E814F815885CA01B9010F940C
:10B8C000C0186D8B7E8B8F8B988FA7019601C70157
:10B8D000B6010F94C0189B01AC016D897E898F89D8
:10B8E000988D0F948D1C6B017C01A5019401C501FD
:10B8F000B4010F948E1C9B01AC01C701B6010F94DB
:10B900006A1D03C060E070E0CB010F94031EF101DB
:10B9100082889388A488B58875016401C418D50805
:10B92000E608F7080F94D21DC61AD70AE80AF90AE2
:10B93000F7FE6BC020E030E0A90169817A818B813C
:10B940009C810F945B18882309F447C029813A81B0
:10B950004B815C81CA01B9010F948E1C6B017C0183
:10B96000C501B4010F945F189B01AC01C701B6017A
:10B970000F94C0186B017C0129893A894B895C8935
:10B98000CA01B9010F94C0189B01AC01C701B601EF
:10B990000F948D1C6B017C012D813E814F81588558
:10B9A000CA01B9010F94C0189B01AC01C701B601CF
:10B9B0000F948E1C6B017C0120E030E040E850E4E5
:10B9C00069817A818B819C810F94C0189B01AC01A5
:10B9D000C701B6010F946A1D03C060E070E0CB019F
:10B9E0000F94541D0F94D21D2B013C0197FF03C0EF
:10B9F000412C512C3201481459046A047B0410F084
:10BA000024013501C12CD12C76018FB7F894D101D6
:10BA10009C9193FD22C0F101468A578A608E718EF7
:10BA2000C40CD51CE61CF71C5A96CD92DD92ED9203
:10BA3000FC925D9729853A854B855C85DB962D9335
:10BA40003D934D935C93DE97FF962D853E854F8504
:10BA5000588920833183428353838FBF68960FB602
:10BA6000F894DEBF0FBECDBFDF91CF911F910F9134
:10BA7000FF90EF90DF90CF90BF90AF909F908F900E
:10BA80007F906F905F904F903F902F9008955F98B8
:10BA90008EBD00000DB407FEFDCF8EB56EBD00005B
:10BAA0000DB407FEFDCF8EB55F9A0895CF93DF9357
:10BAB00000D01F921F92CDB7DEB795E0E9EAF2E021
:10BAC000DE01119601900D929A95E1F7E1E0F0E028
:10BAD000EC0FFD1FE80FF11D808190E00F900F909B
:10BAE0000F900F900F90DF91CF91D1CF1F93CF93F5
:10BAF000DF93CCE2D3E010E089910E94C448882310
:10BB000021F00E940E47812FD1DF1F5F1430A1F773
:10BB100082E40E94C448882321F00E940E4784E0FA
:10BB2000C5DF83E50E94C448882341F0C0E00E943D
:10BB30000E478C2FBBDFCF5FC530C9F7DF91CF91A8
:10BB40001F910895CF93DF93EC018B81882391F1AE
:10BB5000898187FF2BC06C857D858E859F8541E01F
:10BB60000E94E266882331F1E88980E2E89FF001D3
:10BB70001124E65BFB4F3097E9F08081853ED1F0E0
:10BB80008B81823040F449895A896B897C89448F42
:10BB9000558F668F778F4D895E896F89788D538F2A
:10BBA000428F758B648B89818F778983DF91CF91E9
:10BBB0000C94A46681E0888380E0DF91CF910895A2
:10BBC000CF93DF93EC018B81813099F4898181FFE0
:10BBD00010C049895A896B897C89452B462B472B94
:10BBE00059F140E050E0BA01CE010E948C68811109
:10BBF00002C080E022C04D895E896F89788D898D71
:10BC00009A8D0E946B6A8823A1F31D8A1E8A1F8A5F
:10BC1000188E198A1A8A1B8A1C8A898180688983EE
:10BC2000CE0190DF882329F340E050E0BA01CE0135
:10BC3000DF91CF910C948C6881E0DF91CF910895D2
:10BC40006F927F928F929F92AF92BF92CF92DF922C
:10BC5000EF92FF920F931F93CF93DF931F92CDB775
:10BC6000DEB78C015B014A01722EDB0159968D9182
:10BC70009C915A97F801928F818F40E050E0BA0171
:10BC8000C5010E948C68E12CF50180859185A28513
:10BC9000B385418952896389748984179507A607FA
:10BCA000B70708F0CEC025E0B695A795979587957C
:10BCB0002A95D1F7F82FFF70FF2ED50113968C919E
:10BCC000823008F498C141E050E0BE016F5F7F4FC1
:10BCD000C5010E949867019719F4898190E002C01C
:10BCE0008FEF9FEF019609F486C1F501808591855C
:10BCF000A285B3854F96A11DB11D80879187A2872C
:10BD0000B387F0E2FF9EB0011124665B7B4F6115A3
:10BD1000710509F470C1DB018C91882311F0853E17
:10BD2000B9F4E1100EC08091A1069091A206A091F5
:10BD3000A306B091A406F80184879587A687B787E4
:10BD4000F08ADB018C91EE24E39481119DCF79C0C0
:10BD50004BE050E0C4010F948F1F892B09F094CF62
:10BD600077FC49C120E2F29EF0011124E65BFB4F13
:10BD70008385817121F0872D827109F05EC0409129
:10BD8000A1065091A2066091A3067091A406D80165
:10BD90001C964D935D936D937C931F975096FC92E8
:10BDA0004489558960E070E0BA0155274427828DA7
:10BDB000938DA0E0B0E0482B592B6A2B7B2BD80148
:10BDC00055964D935D936D937C93589783858871B9
:10BDD00059F4848D958DA68DB78DF801818B928B4A
:10BDE000A38BB48B81E010C0803139F598012F5EB0
:10BDF0003F4FD80159968D919C915A970E94256981
:10BE00008823D9F084E0F8018383872D8F70D801CF
:10BE100011968C931197F80114821582168217825D
:10BE200018961D921D921D921C921B9774FED6C0EF
:10BE3000C801C6DE8111D2C0DFC0D80113961C92A2
:10BE4000DAC0872D8274823409F0D5C0EE20D9F093
:10BE5000D8015096FC9050971C966D917D918D91D4
:10BE60009C911F9741E0AED7882309F4C4C0F80124
:10BE70008089F0E28F9FC0011124865B9B4F009761
:10BE800009F08DC0B8C0D50113968C9113978230FC
:10BE900009F4B1C051968D919D910D90BC91A02D4A
:10BEA000803E9F4FAF41B10508F0A5C0C5010E947B
:10BEB0005FBB882309F49FC047D7882309F49BC040
:10BEC000D5015996ED91FC915A971496CD90DD903D
:10BED000ED90FC901797B2E0CB1AD108E108F10879
:10BEE000058404C0CC0CDD1CEE1CFF1C0A94D2F7A8
:10BEF00086859785A089B189C80ED91EEA1EFB1ECA
:10BF000081E08093A006C092A106D092A206E092A2
:10BF1000A306F092A40680E092E0EAE4F4E0DF01F8
:10BF20009C011D9221503040E1F766246394D501B5
:10BF30005996ED91FC915A978481681690F42AE401
:10BF400034E0B701A601460D511D611D711D8091A0
:10BF50009E0690919F068CD6882309F44CC063946A
:10BF6000E6CF40E052E060E070E0058404C0440F9A
:10BF7000551F661F771F0A94D2F751968D919D9198
:10BF80000D90BC91A02D840F951FA61FB71FF50122
:10BF9000818B928BA38BB48B8AE494E0F12C20E20A
:10BFA000DC011D922A95E9F72BE0F401DC010190F8
:10BFB0000D922A95E1F721E238E2FC01318B208BCA
:10BFC00040E058E057874687338B228B318F208F94
:10BFD000578B468BB9D68111C5CE0DC075FE09C0F1
:10BFE000F8014189528963897489C8010E948C686B
:10BFF00003C081E001C080E00F90DF91CF911F91DD
:10C000000F91FF90EF90DF90CF90BF90AF909F90F7
:10C010008F907F906F9008952F923F924F925F92F2
:10C020006F927F928F929F92AF92BF92CF92DF9248
:10C03000EF92FF920F931F93CF93DF9300D01F9245
:10C040001F92CDB7DEB78C015B014D83252EDC013D
:10C0500013968C9113978130C9F411968C9181FFBE
:10C0600015C082FF19C0F80141895289638974891A
:10C0700080859185A285B38584179507A607B707A4
:10C0800059F0C8010E948C68811106C081E0F80156
:10C0900080838FEF9FEF2AC1ED80F22C7FC0D80103
:10C0A0005996ED91FC915A9734803A94DB01CA017C
:10C0B00039E0B695A795979587953A95D1F73822A7
:10C0C0004A01B1E09B22332009F474C080E092E081
:10C0D0008819990967018E159F0508F46C01D8012C
:10C0E0005996ED91FC915A9714964D905D906D90F4
:10C0F0007C901797B2E04B1A5108610871080584CB
:10C1000004C0440C551C661C771C0A94D2F7868523
:10C110009785A089B189480E591E6A1E7B1E430C63
:10C12000511C611C711CC114E2E0DE0609F08AC0DA
:10C130008091A1069091A206A091A306B091A406B9
:10C1400084159505A605B70569F41092A0068FEF32
:10C150009FEFDC018093A1069093A206A093A30613
:10C16000B093A4069501B301A20180919E0690911F
:10C170009F067ED5882309F489CFF80180859185B3
:10C18000A285B3858C0D9D1DA11DB11D8087918752
:10C19000A287B387AC0CBD1CEC18FD08D80118961B
:10C1A0004D915D916D917C911B97E114F10409F023
:10C1B00076CF7CC08114910409F088CFD801149601
:10C1C0004D915D916D917C911797411551056105D8
:10C1D000710559F455968D919D910D90BC91A02DAE
:10C1E0000097A105B10541F521C09E012F5F3F4F8A
:10C1F000CF011FD6882309F449CF89819A81AB8169
:10C20000BC81F801218D328DF9012789203139F463
:10C21000883FFFEF9F07A105B10540F40DC0883F9F
:10C220002FEF9207A2072FE0B20730F0C8010E945B
:10C230005FBB81114BCF2ACFF80184839583A683FE
:10C24000B78344CF8114910411F5D80118964D910C
:10C250005D916D917C911B9751968D919D910D9063
:10C26000BC91A02D481759076A077B0780F06CD551
:10C27000882309F40BCF81E08093A0064092A106A9
:10C280005092A2066092A3067092A40607C041E0F5
:10C29000C301B20197D5882309F4F8CEA601B501F0
:10C2A000C401865B9B4F0F949C1F67CF51968D9165
:10C2B0009D910D90BC91A02D84179507A607B707F7
:10C2C00040F4F801418B528B638B748B81818068C1
:10C2D0008183D80111968C9183FD03C08D81922DAD
:10C2E00005C0C8012FDC8111F9CFD0CE0F900F907F
:10C2F0000F900F900F90DF91CF911F910F91FF90B2
:10C30000EF90DF90CF90BF90AF909F908F907F90F5
:10C310006F905F904F903F902F900895CF93DF9351
:10C320001F92CDB7DEB7698341E050E0BE016F5F79
:10C330007F4F049671DE0F90DF91CF910895CF93D8
:10C34000DF93EC01FFDB1B82DF91CF910895109208
:10C350005E1280915314882319F080E594E1EFCFA9
:10C360000895CF92DF92EF92FF921F93CF93DF93C6
:10C3700010925F128091B912882319F086EB92E136
:10C38000DEDF10922D1410922A1485E38093291475
:10C390000E94A24CEB01A895809129140E940B9059
:10C3A00089E294E10E949E4C2398229A219A209A35
:10C3B000289A85E080932B1482E58CBD1DBC1AE081
:10C3C0008FEF0E949E461150D9F720E030E0A9017E
:10C3D00060E089E294E10E94C64C182F80932C14EF
:10C3E000813049F00E94A24C6C1B7D0B613D77406F
:10C3F00060F381E054C02AEA31E040E050E068E0B8
:10C4000089E294E10E94C64C82FF03C010932D1470
:10C410000EC014E00E94A34680932C141150D1F753
:10C420008A3A11F082E03BC082E080932D14809123
:10C430002D14823031F4C12CD12CE12C40E4F42EA7
:10C4400003C0C12CD12C760120E030E0A90167E3C4
:10C4500089E294E10E94C64CA701960169E289E253
:10C4600094E10E94C64C80932C14882349F00E94CA
:10C47000A24C6C1B7D0B613D774030F38AE00FC00E
:10C4800080912D14823011F520E030E0A9016AE39B
:10C4900089E294E10E94C64C882351F088E08093A1
:10C4A0002A1489E294E10E949E4CEEEDFAE11AC052
:10C4B0000E94A346807C803C19F483E080932D1475
:10C4C0000E94A3460E94A3460E94A34689E294E1EB
:10C4D0000E949E4C10922B1481E00E943592811193
:10C4E00032C015C08491EF012196882321F00E946B
:10C4F000AA46FE01F7CFEEE7FCE08491EF0121961A
:10C50000882309F456C00E94AA46FE01F6CF80E0B7
:10C510000E943592811117C0E3EAFAE18491EF019C
:10C520002196882321F00E94AA46FE01F7CFEAE671
:10C53000FCE08491EF012196882309F43AC00E941F
:10C54000AA46FE01F6CF6EE274E186EB92E1E3D6F5
:10C55000811116C0E3EAFAE18491EF012196882364
:10C5600021F00E94AA46FE01F7CFE9E5FCE08491A4
:10C57000EF0121968823E9F00E94AA46FE01F7CF39
:10C5800081E080935F12EEEDFAE18491EF01219654
:10C59000882321F00E94AA46FE01F7CFEDE4FCE0DB
:10C5A0008491EF012196882321F00E94AA46FE0182
:10C5B000F7CF8BE1E6EBF2E1A7EDB2E101900D924E
:10C5C0008A95E1F78091B4129091B5129093D612AA
:10C5D0008093D51282EB92E19093D2128093D11284
:10C5E000DF91CF911F91FF90EF90DF90CF90089552
:10C5F000FC0123812111A3CE08952F923F924F92E7
:10C600005F926F927F928F929F92AF92BF92CF92E2
:10C61000DF92EF92FF920F931F93CF93DF93CDB7EB
:10C62000DEB7C454D1090FB6F894DEBF0FBECDBF3C
:10C630004C015B017A01322E1C8E1F8E19821C82E6
:10C640006115710511F410E0ABC0FC01838181110B
:10C65000FACFFA0180818F3261F4CA017C01019620
:10C66000F70120812F32D1F3F5018381825082308E
:10C6700010F465010AC0618D728DCE0101964BD612
:10C68000882309F3CE0101966C018E01045E1F4FD1
:10C69000280157E3652E712C6C0E7D1E9BE0690E00
:10C6A000711CFE0131962496FFAFEEAF24972596BC
:10C6B0000FAF2597212E35C080E28193E615F7054F
:10C6C000D9F7D70120E097E04A2F3B2F8D918111B8
:10C6D0002BC08FA9803209F4B6CF842F932F7C0111
:10C6E000FC01208101962F32D1F3222309F450C09E
:10C6F00021E0AE01495C5F4FB601C801A1DA882391
:10C7000009F4A1CFCA14DB0411F0C60118DE041528
:10C710001505B9F125969FAD2597822D6801092F42
:10C72000182FFE01F796C8CF8F3299F28E3219F08A
:10C73000ECE8FCE00AC09A3009F485CF28E09AE0E2
:10C74000C3CF3196381709F47ECF34913111F9CF28
:10C75000921708F478CF813208F475CF8F3709F437
:10C7600072CF31E0320FE7E3F0E0EC0FFD1FE20F94
:10C77000F11D2FE9280F2A3108F480528083232FDE
:10C78000A3CF23969FAD239724968FAD2497C6CF32
:10C79000232DAE01495C5F4FB601C40151DA182F59
:10C7A000CE01019625DFCE014C9622DF812FCC5B96
:10C7B000DF4F0FB6F894DEBF0FBECDBFDF91CF9134
:10C7C0001F910F91FF90EF90DF90CF90BF90AF90AF
:10C7D0009F908F907F906F905F904F903F902F90A1
:10C7E000089524E233E0FC0131832083049600CFD6
:10C7F0002F923F924F925F926F927F928F929F9271
:10C80000AF92BF92CF92DF92EF92FF920F931F935E
:10C81000CF93DF93CDB7DEB7C057D1090FB6F894E9
:10C82000DEBF0FBECDBF7C016B014A012DB73EB705
:10C83000AF963FAF2EAFAF97AD961FAEAD9734E03A
:10C84000C30ED11C8E01015A1F4F74E2672E73E094
:10C85000772EE0E42E2E312C2C0E3D1E84E0280E87
:10C86000311C4EE652E1BE016F5F7F4FC6010E9450
:10C87000909318160CF057C12C85922F9871903117
:10C8800009F0CDC080910A158150823008F4C7C0EC
:10C890004DB65EB6BE016F5F7F4FC8010E94EF8646
:10C8A00081E0F70190819111B2C0E1E0F0E0D801A0
:10C8B0000D900020E9F7E01BF10BEA0FFB1F31960A
:10C8C0002DB73EB72E1B3F0B0FB6F8943EBF0FBEE1
:10C8D0002DBFEDB7FEB731965F01882319F060E3F5
:10C8E00073E001C0B701C5010F94CE1FB801C501A7
:10C8F0000F94B81F60E373E0C5010F94B81F25962D
:10C900001FAE259728961FAE289724961FAE1EAE01
:10C91000249722967FAE6EAE229721E0A801B60141
:10C92000C1016BDE81114DC080910A15811149C092
:10C93000EEEDFAE184919F012F5F3F4F882381F054
:10C94000E0962FAFE097E1963FAFE1970E94AA46AD
:10C95000E0962FADE097E1963FADE197F901EACF80
:10C96000ECE9FCE084919F012F5F3F4F811102C0F1
:10C97000980110C0E0962FAFE097E1963FAFE197A6
:10C980000E94AA46E0962FADE097E1963FADE19771
:10C99000F901E8CFF90181919F01882379F0E096B0
:10C9A0002FAFE097E1963FAFE1970E94AA46E1964C
:10C9B0003FADE197E0962FADE097ECCF8AE00E9483
:10C9C000AA468BE1FE01EC5BFF4FDE0195960190DC
:10C9D0000D928A95E1F724968EAD9FAD24979CA386
:10C9E0008BA37AA269A240E050E0BE016F5D7F4F49
:10C9F000C501FEDECE018196F4DECE01805C9F4F44
:10CA0000F0DE0FB6F8945EBE0FBE4DBE2ACF80E0BA
:10CA100001900020E9F73197EE19FF0948CF89818D
:10CA2000882309F480C0853E09F41BCF8E3209F4B7
:10CA300018CF80916E128E3209F413CF2A7009F04C
:10CA400010CF81E0903109F080E080936012811175
:10CA500008C08985873409F004CF8A858E3709F4A8
:10CA600000CF80910A15813021F068F08230A9F161
:10CA7000F8CE80910B1590910C15019690930C15A2
:10CA800080930B15EECEBE016F5F7F4F81E692E182
:10CA90000E94EF865701F50181915F01882319F00B
:10CAA0000E94AA46F8CF61E6A62E62E1B62EF501F5
:10CAB00081915F01882319F00E94AA46F8CF80E295
:10CAC0000E94AA466D8D7E8D8F8D98A14AE00E94AE
:10CAD000DE8A8AE00E94AA46C4CEBE016F5F7F4F05
:10CAE00081E692E10E94EF868114910441F061E6B3
:10CAF00072E1C4010F94A51F892B69F414C0AD968F
:10CB0000FFADAD972F2F30E080910B1590910C1554
:10CB10002817390741F0AD963FADAD973F5FAD9611
:10CB20003FAFAD979ECEAF962EAD3FADAF970FB650
:10CB3000F8943EBF0FBE2DBFC059DF4F0FB6F8941B
:10CB4000DEBF0FBECDBFDF91CF911F910F91FF9040
:10CB5000EF90DF90CF90BF90AF909F908F907F909D
:10CB60006F905F904F903F902F900895FB01408110
:10CB7000FC0120813181342768E0A901440F551F51
:10CB800037FD07C09A016150C1F7FC013183208352
:10CB900008959A01F1E22F27F0E13F27F4CFEF92B9
:10CBA000FF920F931F93CF93DF93EC0189018C8148
:10CBB000833039F0E9E0440F551F661F771FEA956F
:10CBC000D1F79A01AB0161E1CE010E94C64C8823E6
:10CBD00031F084E08983CE010E949E4C41C00E94C6
:10CBE000A24C7B010E94A3468B838F3F49F40E9495
:10CBF000A24C6E197F096D327140A0F381E103C030
:10CC00008E3F49F08FE08983CE010E949E4C8FEFCA
:10CC10000E949E4625C08FEF8EBDF80180E090E017
:10CC20002FEF0DB407FEFDCF3EB531932EBD01961B
:10CC30008F3F31E09307A9F70DB407FEFDCF8EB506
:10CC4000F801E150FE4F80830E94A3460E94A34654
:10CC5000CE010E949E4C8FEF0E949E4681E001C053
:10CC600080E0DF91CF911F910F91FF90EF90089599
:10CC70000F931F93CF93DF93EC0189018C81833055
:10CC800039F0F9E0440F551F661F771FFA95D1F769
:10CC90009A01AB0168E1CE010E94C64C882311F0D5
:10CCA00086E034C08EEF8EBD80E090E00DB407FECC
:10CCB000FDCFF801E80FF91F20812EBD0DB407FE4E
:10CCC000FDCF21812EBD0296811522E0920771F7DA
:10CCD0000DB407FEFDCF8FEF0E949E468FEF0E949E
:10CCE0009E460E94A3468B838F71853031F083E18D
:10CCF0008983CE010E949E4C0AC068E572E0CE0195
:10CD00000E94AE4C182F811107C087E18983CE01A4
:10CD10000E949E4C10E012C020E030E0A9016DE0BE
:10CD2000CE010E94C64C811104C00E94A3468823F4
:10CD300011F086E1EBCFCE010E949E4C812FDF9156
:10CD4000CF911F910F910895CF938091A0068823D2
:10CD5000A9F14091A1065091A2066091A30670919D
:10CD6000A4062AE434E080919E0690919F0680DF1D
:10CD7000C82F882321F140914207509143076091C9
:10CD8000440770914507411551056105710589F00A
:10CD90002AE434E080919E0690919F0669DF882303
:10CDA00059F01092420710924307109244071092D4
:10CDB00045071092A0068C2FC82F01C0C1E08C2F10
:10CDC000CF910895CF92DF92EF92FF92CF936B01B4
:10CDD0007C01C42F8091A1069091A206A091A30688
:10CDE000B091A4068C159D05AE05BF05C1F0ACDF62
:10CDF000811102C080E017C02AE434E0B701A60127
:10CE000080919E0690919F06CADE882399F3C09276
:10CE1000A106D092A206E092A306F092A40681E0B9
:10CE2000C1118093A006CF91FF90EF90DF90CF903B
:10CE300008958F929F92AF92BF92CF92DF92EF921E
:10CE4000FF920F931F93CF93DF93EC016A017B0155
:10CE5000890189859A85AB85BC850196A11DB11D87
:10CE600084179507A607B70710F480E054C08F8990
:10CE7000803129F49927872F762F652F0BC08032B8
:10CE8000A1F7CB01BA0127E096958795779567952D
:10CE90002A95D1F78B889C88AD88BE88680D791D4E
:10CEA0008A1D9B1D8090A1069090A206A090A306CB
:10CEB000B090A406681579058A059B0581F48F89D1
:10CEC000803191F4DD24EE24FF24F601EE0FFF1FE4
:10CED000E65BFB4F80819181A0E0B0E016C040E0AE
:10CEE00071DF8111ECCFC1CFE894C7F8DD24EE24C7
:10CEF000FF24F601EE0FFF1FEE0FFF1FE65BFB4F57
:10CF000080819181A281B381BF70F8018083918378
:10CF1000A283B38381E0DF91CF911F910F91FF90A6
:10CF2000EF90DF90CF90BF90AF909F908F9008953B
:10CF30002F923F924F925F926F927F928F929F9229
:10CF4000AF92BF92CF92DF92EF92FF920F931F9317
:10CF5000CF93DF93EC015B016A018B81811103C0E8
:10CF60008FEF9FEFC6C0898180FFFACF49895A8928
:10CF70006B897C8988859985AA85BB852601612C6A
:10CF8000712C8A019B01081B190B2A0B3B0B041502
:10CF900015052605370518F46A01C81AD90A76015D
:10CFA0003E0124E0620E711CE114F10409F476C024
:10CFB000488559856A857B854A0181E098222B81C5
:10CFC0001A012B01E9E05694479437942794EA9587
:10CFD000D1F7898D9A8DFC01223049F4628D738DD1
:10CFE000848D958D620D731D841D951D3CC014812B
:10CFF0001150122181149104C1F4111116C0452B56
:10D00000462B472B49F48D899E89AF89B88D8C8337
:10D010009D83AE83BF8309C04C815D816E817F811A
:10D02000930107DF882309F49BCFE98DFA8D6C818A
:10D030007D818E819F8162507109810991090584EA
:10D0400004C0660F771F881F991F0A94D2F72685A0
:10D05000378540895189620F731F841F951F610FA7
:10D06000711D811D911D20E032E0281939098701C9
:10D070002E153F0508F489010115F2E01F0761F53F
:10D080002091A1063091A2064091A3065091A406DA
:10D09000621773078407950719F41EC0C60129C0DB
:10D0A0009501AB01BC0180919E0690919F0677DDB2
:10D0B000882309F455CFA00EB11E88859985AA85CD
:10D0C000BB85800F911FA11DB11D88879987AA87F5
:10D0D000BB87E01AF10A68CF40E074DE882309F4C8
:10D0E0003FCFB401665B7B4FA801C5010F949C1F25
:10D0F000E2CFDF91CF911F910F91FF90EF90DF90E2
:10D10000CF90BF90AF909F908F907F906F905F90E7
:10D110004F903F902F9008954F925F926F927F9221
:10D12000AF92BF92CF92DF92EF92FF920F931F9335
:10D13000CF93DF93EC016A017B012B81222349F01D
:10D1400089899A89AB89BC8984179507A607B7078F
:10D1500010F480E06BC0223009F463C0C114D10424
:10D16000E104F10449F41C821D821E821F8218868C
:10D1700019861A861B8659C088859985AA85BB851C
:10D18000E98DFA8DE585F0E03996AC01BD0141509D
:10D190005109610971090E2E04C07695679557955E
:10D1A00047950A94D2F79701860101501109210988
:10D1B000310904C03695279517950795EA95D2F75A
:10D1C000041715072607370720F0892B8A2B8B2B8E
:10D1D00049F48D899E89AF89B88D8C839D83AE83F8
:10D1E000BF8304C0041B150B260B370B2801390124
:10D1F0005E0184E0A80EB11C411451046104710465
:10D2000081F04C815D816E817F819501898D9A8D40
:10D2100010DE91E0491A5108610871088111ECCFC4
:10D2200005C0C886D986EA86FB8681E0DF91CF916A
:10D230001F910F91FF90EF90DF90CF90BF90AF9034
:10D240007F906F905F904F9008954F925F926F9292
:10D250007F92AF92BF92CF92DF92EF92FF920F93A5
:10D260001F93CF93DF9300D01F92CDB7DEB78C0111
:10D2700049835A836B837C835901C12CD12C76015D
:10D28000412CF2E05F2E612C712C49815A816B8117
:10D290007C819E012F5F3F4FC801CBDD882341F188
:10D2A000D301C201F801058404C0880F991FAA1F89
:10D2B000BB1F0A94D2F7C80ED91EEA1EFB1E498175
:10D2C0005A816B817C818789803139F481E0483FC4
:10D2D0005F4F6105710538F4D8CF81E0483F5F4F5B
:10D2E0006F4F7F4090F2F501C082D182E282F382DB
:10D2F0000F900F900F900F90DF91CF911F910F9192
:10D30000FF90EF90DF90CF90BF90AF907F906F90A5
:10D310005F904F9008950F931F93CF93DF93EC018D
:10D320008B018B81882311F080E041C0FB0187894C
:10D33000803131F18032C1F783E08B83F801428D77
:10D34000538D648D758D4D8B5E8B6F8B788F9E01A9
:10D350002F5E3F4FC80179DF882331F31A8F098F81
:10D3600081E089831C821D821E821F821886198695
:10D370001A861B861C861D861E861F86188A17C065
:10D3800082E08B831D8A1E8A1F8A188EFB01408DC6
:10D39000518D60E070E0A5E0440F551F661F771FB8
:10D3A000AA95D1F7498B5A8B6B8B7C8BD7CFDF91AA
:10D3B000CF911F910F9108954F925F926F927F923C
:10D3C0008F929F92AF92BF92CF92DF92EF92FF9295
:10D3D0000F931F93CF93DF93EC014A015B01280168
:10D3E0003901423051056105710508F462C0498573
:10D3F0005A856B857C854F5F5F4F6F4F7F4F481518
:10D4000059056A057B0508F454C08F89803129F4D9
:10D41000FF24EB2CDA2CC92C0CC0803209F049C057
:10D420007501640107E0F694E794D794C7940A95D0
:10D43000D1F74B895C896D897E89C40ED51EE61EA5
:10D44000F71E41E0C701B601BDDC882391F19F8939
:10D45000903159F49924AA24BB24F401EE0FFF1F44
:10D46000E65BFB4F5182408210C0E89487F8992414
:10D47000AA24BB24F401EE0FFF1FEE0FFF1FE65B93
:10D48000FB4F40825182628273829A89923090F07F
:10D490004D815E816F8178854C0D5D1D6E1D7F1DF8
:10D4A00040934207509343076093440770934507A6
:10D4B00001C080E0DF91CF911F910F91FF90EF901D
:10D4C000DF90CF90BF90AF909F908F907F906F90A4
:10D4D0005F904F900895AF92BF92CF92DF92EF92FC
:10D4E000FF920F931F93CF93DF9300D01F92CDB77E
:10D4F000DEB75C016A017B0182E090E0A0E0B0E071
:10D50000F50180839183A283B3839E012F5F3F4FF8
:10D51000B701A601C5018DDC811102C080E023C0E6
:10D5200000E010E09801B701A601C50145DF88239E
:10D53000A9F3C980DA80EB80FC80F501878980310E
:10D5400049F481E0F8EFCF16FFEFDF06E104F104C4
:10D5500050F4DBCF81E098EFC9169FEFD906E906BA
:10D560009FE0F90690F20F900F900F900F90DF91CF
:10D57000CF911F910F91FF90EF90DF90CF90BF90D0
:10D58000AF900895CF93DF93CDB7DEB78091840637
:10D59000811110C09E01275F3F4F4F81588562E483
:10D5A00070E08EE092E00F9423180E946F8483E075
:10D5B0008093A802DF91CF910895FF920F931F935C
:10D5C000CF93DF93C091790681E0C827D0917A0686
:10D5D000D827F0907B06F826C11102C0DD2319F090
:10D5E000EEEDFAE104C0F110FBCF80E077C084914A
:10D5F0008F010F5F1F4F882321F00E94AA46F80178
:10D60000F6CFE7EFFCE084918F010F5F1F4F882377
:10D6100021F00E94AA46F801F6CFCC2361F0E5EF95
:10D62000FCE084918F010F5F1F4F882321F00E943F
:10D63000AA46F801F6CFDD2361F0E3EFFCE0849128
:10D640008F010F5F1F4F882321F00E94AA46F80127
:10D65000F6CFF11003C0E9EEFCE00CC0E1EFFCE016
:10D6600084918F010F5F1F4F8823A9F30E94AA4660
:10D67000F801F6CF84918F010F5F1F4F882321F0AF
:10D680000E94AA46F801F6CFFF2019F042E353E0CA
:10D6900002C043E853E0DD2319F024E333E002C085
:10D6A00023E833E0CC2319F086E393E002C083E85B
:10D6B00093E05F934F933F932F939F938F9387EDC7
:10D6C0009CE09F938F931F925DDF8DB79EB7099665
:10D6D0000FB6F8949EBF0FBE8DBF81E0DF91CF9152
:10D6E0001F910F91FF90089580914F1281508230C9
:10D6F00010F080E0089510924F120E94A24C6093A7
:10D7000058127093591280935A1290935B1281E0D1
:10D7100008950F931F9380914F12813019F40E9446
:10D72000A24C08C0609158127091591280915A12FF
:10D7300090915B1200915412109155122091561243
:10D7400030915712601B710B820B930B28EE33E064
:10D7500040E050E00F94301C809150129091511293
:10D76000A0915212B0915312280F391F4A1F5B1F0C
:10D77000CA01B9011F910F91089580914F12813014
:10D7800099F1823051F4C5DF6093501270935112B9
:10D79000809352129093531218C010925412109208
:10D7A000551210925612109257121092581210924F
:10D7B000591210925A1210925B121092501210923B
:10D7C0005112109252121092531281E080934F1214
:10D7D0000E94A24C6093541270935512809356127B
:10D7E0009093571281E0089580E00895CF92DF92E0
:10D7F000EF92FF92C0907107D0907207E09073078C
:10D80000F09074072091B80F3091B90F4091BA0F82
:10D810005091BB0FC701B6010F94C0180F94BF1EE3
:10D8200060932B1270932C1280932D1290932E12D2
:10D83000C701B6010F94D21D2FB7F8946093B80EAC
:10D840007093B90E8093BA0E9093BB0E2FBF1092B7
:10D850001B1210921C1210921D1210921E12FF9099
:10D86000EF90DF90CF90089580914F12813079F43E
:10D8700082E080934F120E94A24C609358127093E2
:10D88000591280935A1290935B1281E0089580E0C0
:10D890000895E82FF0E0E550F84E849190E0FC0107
:10D8A0003797EC30F105F8F4EC57FF4F0D947D1FDE
:10D8B0008091B100887F84608093B1000895809149
:10D8C0009100887F84608093910008958091A100E9
:10D8D000887F84608093A100089580912101887FD2
:10D8E00084608093210108958F929F92AF92BF929E
:10D8F000CF92DF92EF92FF920F931F93CF93DF931C
:10D900001F921F92CDB7DEB77C0149018091CE06F0
:10D91000811147C08B015B01A40EB51E0A151B05C2
:10D9200009F43FC0F701C080D180F80161918F01F7
:10D930006983C6016A830F94111B6A81681729F1F4
:10D94000C6010F94191BC6010F94111B99818917E9
:10D95000E1F0EEEDFAE184918F010F5F1F4F882314
:10D9600021F00E94AA46F801F6CFEDEBFCE084918D
:10D970008F010F5F1F4F882321F00E94AA46F801F4
:10D98000F6CF81E08093CE060CC0BE016F5F7F4F63
:10D99000C401ECD8F7018081918101969183808345
:10D9A000BDCF0F900F90DF91CF911F910F91FF90FE
:10D9B000EF90DF90CF90BF90AF909F908F900895A1
:10D9C000AF92BF92CF92DF92EF92FF920F931F938D
:10D9D000CF93DF931F92CDB7DEB78C016B017A0135
:10D9E00059018091CE0681111BC0F801808191817F
:10D9F0000F94111B8983F60181936F01BE016F5F44
:10DA00007F4FC501B3D8F801408151814F5F5F4F0F
:10DA100051834083F1E0EF1AF108E114F10429F792
:10DA20000F90DF91CF911F910F91FF90EF90DF90BA
:10DA3000CF90BF90AF900895CF92DF92EF92FF9278
:10DA40000F931F93CF93DF937C018B016A01E90150
:10DA50000E94298583E08093A802F092C80FE0928B
:10DA6000C70F1093C60F0093C50F1092C10F1092ED
:10DA7000C20F1092C30F1092C40FA601662757FD64
:10DA80006095762F4093BD0F5093BE0F6093BF0FEC
:10DA90007093C00FF80180819181AA2797FDA0950E
:10DAA000BA2F8093231190932411A0932511B09342
:10DAB000261180E792EC9093950280939402D09384
:10DAC0006B0FC0936A0F1092690FDF91CF911F9176
:10DAD0000F91FF90EF90DF90CF900895CF92DF925B
:10DAE000EF92FF920F931F93CF93DF9300D01F927B
:10DAF000CDB7DEB77C018B01CA01B90129837A83D6
:10DB00008B839C830E94298523E02093A802F092B6
:10DB1000C80FE092C70F1093C60F0093C50F2AE0FD
:10DB200037ED43E25CE369817A818B819C810F94BC
:10DB3000C0180F94D21D6093C10F7093C20F8093D1
:10DB4000C30F9093C40F0F9461186B017C019B016C
:10DB5000AC0160E070E887E794E40F948D1C0F94AB
:10DB6000D21D6093BD0F7093BE0F8093BF0F909333
:10DB7000C00F2AE037ED43E25CE3F8016081718178
:10DB8000828193810F94C018A70196010F948D1C78
:10DB90000F94D71D60932311709324118093251146
:10DBA0009093261185EB90EC9093950280939402CC
:10DBB0000F900F900F900F90DF91CF911F910F91C9
:10DBC000FF90EF90DF90CF9008950F931F93CF9326
:10DBD000DF938C01EB010E94298583E08093A802EA
:10DBE0001093C80F0093C70FD093C60FC093C50FF3
:10DBF00084EF91E0A0E0B0E08093C10F9093C20F5A
:10DC0000A093C30FB093C40F88EE9FE3AFE0B0E0E2
:10DC10008093BD0F9093BE0FA093BF0FB093C00F22
:10DC200020E030E048EC52E4688179818A819B8170
:10DC30000F94C01820E030E04AEF53E40F948D1C9D
:10DC40000F94D71D60932311709324118093251195
:10DC50009093261188E49FEB909395028093940211
:10DC60008EEC90EF90936B0F80936A0F1092690F78
:10DC7000DF91CF911F910F910895CF92DF92EF9294
:10DC8000FF920F931F93CF93DF9300D01F92CDB7D6
:10DC9000DEB77C018B0129833A834B835C830E942E
:10DCA000298583E08093A802F092C80FE092C70F05
:10DCB0001093C60F0093C50F29813A814B815C8177
:10DCC000CA01B9010F945F182AE037ED43E25CE323
:10DCD0000F94C0180F94D21D6093C10F7093C20FA0
:10DCE0008093C30F9093C40F0F9461186B017C0154
:10DCF0009B01AC0160E070E887E794E40F948D1C11
:10DD00000F94D21D6093BD0F7093BE0F8093BF0F11
:10DD10009093C00FF80160817181828193810F948B
:10DD20005F182AE037ED43E25CE30F94C018A701C7
:10DD300096010F948D1C0F94D71D6093231170933F
:10DD40002411809325119093261187E49CED9093E4
:10DD50009502809394028AE79EE790936B0F8093DD
:10DD60006A0F1092690F0F900F900F900F90DF9134
:10DD7000CF911F910F91FF90EF90DF90CF9008957A
:10DD80008F929F92AF92BF92CF92DF92EF92FF92CB
:10DD9000CF9320E030E04AE754E4FC0160817181D8
:10DDA000828193810F94C0180F94D21D6B017C0166
:10DDB000611571058105910561F097FF0AC0F09426
:10DDC000E094D094C094C11CD11CE11CF11C8DE2E4
:10DDD00001C080E28093DF0FC701B60128EE33E077
:10DDE00040E050E00F94521C9AE0892E912CA12C17
:10DDF000B12CCA01B901A50194010F94521C605DB8
:10DE00006093E00F8EE28093E10FC701B60124E634
:10DE100030E040E050E00F94521CCA01B901A50166
:10DE200094010F94521C605D6093E20FC701B6012C
:10DE3000A50194010F94521CC62FCA01B901A50176
:10DE400094010F94521C605D6093E30FC05DC0931A
:10DE5000E40F8FED9FE0CF91FF90EF90DF90CF9098
:10DE6000BF90AF909F908F9008950F931F93CF9383
:10DE7000DF931F921F92CDB7DEB7FC0184918F0113
:10DE80000F5F1F4F811102C08B0108C069837A8325
:10DE90000E94AA46F80169817A81F0CFD8018D915C
:10DEA0008D01882319F00E94AA46F8CF0F900F9099
:10DEB000DF91CF911F910F9108950F931F93CF93EF
:10DEC000DF938C01EEEDFAE18491EF012196882336
:10DED00021F00E94AA46FE01F7CFB80180EB9CE03A
:10DEE000C4DF82E20E94AA468AE00E94AA4681E03C
:10DEF000DF91CF911F910F9108958F929F92AF92D2
:10DF0000BF92CF92DF92EF92FF92CF93FC01C0803D
:10DF1000D180E280F38020E030E0A901C701B601A2
:10DF20000F945B1887FF08C0C701B601905820E026
:10DF300030E048EC52E406C020E030E048EC52E427
:10DF4000C701B6010F94C0180F94D21D6B017C015C
:10DF5000603AF6E87F07F1E08F07910584F020EA48
:10DF600036E841E050E00F94521CCA01B9012AE0A2
:10DF700030E040E050E00F94521C605D01C060E270
:10DF80006093DE0F80E1C81687E2D806E104F10451
:10DF900094F0C701B60120E137E240E050E00F9471
:10DFA000521CCA01B9012AE030E040E050E00F9471
:10DFB000521C605D01C060E26093DF0FE8EECE1698
:10DFC000E3E0DE06E104F10494F0C701B60128EEB7
:10DFD00033E040E050E00F94521CCA01B9012AE03E
:10DFE00030E040E050E00F94521C605D01C060E200
:10DFF0006093E00FC701B60124E630E040E050E056
:10E000000F94521C6AE0862E912CA12CB12CCA01CF
:10E01000B901A50194010F94521C605D6093E10F5A
:10E020008EE28093E20FC701B601A50194010F941F
:10E03000521CC62FCA01B901A50194010F94521CAC
:10E04000605D6093E30FC05DC093E40F8EED9FE0D1
:10E05000CF91FF90EF90DF90CF90BF90AF909F90C7
:10E060008F9008958F929F92AF92BF92CF92DF923E
:10E07000EF92FF92CF9320E030E048EC52E4FC01B5
:10E0800060817181828193810F94C0180F94D21D99
:10E090006B017C0197FF0AC0F094E094D094C09487
:10E0A000C11CD11CE11CF11C8DE201C08BE28093EC
:10E0B000DE0FC701B60120E137E240E050E00F94E7
:10E0C000521C7AE0872E912CA12CB12CCA01B901E7
:10E0D000A50194010F94521C605D6093DF0FC7018E
:10E0E000B60128EE33E040E050E00F94521CCA0124
:10E0F000B901A50194010F94521C605D6093E00F7B
:10E10000C701B60124E630E040E050E00F94521C15
:10E11000CA01B901A50194010F94521C605D60937E
:10E12000E10F8EE28093E20FC701B601A5019401D1
:10E130000F94521CC62FCA01B901A50194010F9476
:10E14000521C605D6093E30FC05DC093E40F8EEDE1
:10E150009FE0CF91FF90EF90DF90CF90BF90AF9076
:10E160009F908F9008958F929F92AF92BF92CF927F
:10E17000DF92EF92FF92FC01C080D180E280F380B9
:10E1800020E030E0A901C701B6010F945B1887FFBA
:10E1900004C0C701B601905802C0C701B6010F9470
:10E1A000D21D6B017C016031F7E27F07810591058B
:10E1B00084F020E137E240E050E00F94521CCA01A5
:10E1C000B9012AE030E040E050E00F94521C605D5D
:10E1D00001C060E26093E00F88EEC81683E0D806C5
:10E1E000E104F10494F0C701B60128EE33E040E009
:10E1F00050E00F94521CCA01B9012AE030E040E01F
:10E2000050E00F94521C605D01C060E26093E10F2A
:10E21000E4E6CE16D104E104F10494F0C701B6019E
:10E2200024E630E040E050E00F94521CCA01B901EE
:10E230002AE030E040E050E00F94521C605D01C0E5
:10E2400060E26093E20FFAE0CF16D104E104F1043A
:10E250009CF0EAE08E2E912CA12CB12CC701B601C6
:10E26000A50194010F94521CCA01B901A5019401A2
:10E270000F94521C605D01C060E26093E30FC70120
:10E28000B6012AE030E040E050E00F94521C605D9F
:10E290006093E40F80EE9FE0FF90EF90DF90CF90CF
:10E2A000BF90AF909F908F90089520E030E040E2C3
:10E2B00051E4FC0160817181828193810F94C018C7
:10E2C0000F94D21D9B0177FF06C022273327261B00
:10E2D000370B8DE201C08BE28093DF0FC90168EE3E
:10E2E00073E00F946A1FCB01EAE0F0E0BF010F94E6
:10E2F0006A1F805D8093E00FC90164E670E00F94AF
:10E300006A1FCB01BF010F946A1F805D8093E10FEC
:10E31000C901BF010F946A1F282FCB01BF010F94C1
:10E320006A1F805D8093E20F8EE28093E30F205D91
:10E330002093E40F8FED9FE0089590912F1280912C
:10E340003012981721F080E00E94A9CDF6CF0895F1
:10E350002F923F924F925F926F927F928F929F92F5
:10E36000AF92BF92CF92DF92EF92FF920F931F93E3
:10E37000CF93DF9300D01F92CDB7DEB77B018A0128
:10E3800019012091AC0F3091AD0F4091AE0F50911B
:10E39000AF0FDC016D917D918D919C910F94C01810
:10E3A0000F94BF1E4B015C0160931F1270932012EB
:10E3B00080932112909322122091B00F3091B10FCF
:10E3C0004091B20F5091B30FF7016081718182814A
:10E3D00093810F94C0180F94BF1E6B017C01609352
:10E3E0002312709324128093251290932612209169
:10E3F000B40F3091B50F4091B60F5091B70FD801BF
:10E400006D917D918D919C910F94C0180F94BF1EBA
:10E410002B013C01609327127093281280932912DC
:10E4200090932A122091B80F3091B90F4091BA0FF2
:10E430005091BB0FF10160817181828193810F94B2
:10E44000C0180F94BF1E60932B1270932C128093F0
:10E450002D1290932E1269837A838B839C836DDFB8
:10E460002FB7F8948092AC0E9092AD0EA092AE0EA3
:10E47000B092AF0EC092B00ED092B10EE092B20E3A
:10E48000F092B30E4092B40E5092B50E6092B60E5A
:10E490007092B70E69817A818B819C816093B80EEE
:10E4A0007093B90E8093BA0E9093BB0E2FBF10924B
:10E4B0000B1210920C1210920D1210920E1280E19B
:10E4C000EFE0F2E1DF011D928A95E9F70F900F90DE
:10E4D0000F900F90DF91CF911F910F91FF90EF90D0
:10E4E000DF90CF90BF90AF909F908F907F906F9074
:10E4F0005F904F903F902F900895EF92FF920F936F
:10E500001F93CF93DF93CDB7DEB72C970FB6F89458
:10E51000DEBF0FBECDBF0CEA1FE08AE7E82E87E022
:10E52000F82EF80121913191419151918F0160E0D4
:10E5300070E080E89FE30F946A1DF7016193719387
:10E54000819391937F01FFE00C3B1F0751F780916E
:10E55000650790916607A0916707B0916807898366
:10E560009A83AB83BC838091690790916A07A091DD
:10E570006B07B0916C078D839E83AF83B8878091C2
:10E580006D0790916E07A0916F07B0917007898712
:10E590009A87AB87BC87AE01475F5F4FBE016B5F59
:10E5A0007F4FCE0101960E94478321E737E0AE01FD
:10E5B000475F5F4FBE016B5F7F4FCE010196C8DEA4
:10E5C0000E9434462C960FB6F894DEBF0FBECDBF26
:10E5D000DF91CF911F910F91FF90EF9008950E94CE
:10E5E00034468BDF0E947B4780E00E94294881E00F
:10E5F0000E94294882E00E94294880E00C94784DCE
:10E60000CF93DF936CEA7FE04BE95FE0C3E0D1E1B9
:10E6100020E030E0F901E55AF24F85919591A591FE
:10E62000B491FB0181939193A193B193BF01F9013F
:10E63000E55BF24F85919591A591B491FA01819393
:10E640009193A193B193AF01F901E55CF24F8591EC
:10E650009591A591B49189939993A993B9932C5FBE
:10E660003F4F20313105B1F680E090E0AAE7B3E4F6
:10E6700080931B1190931C11A0931D11B0931E1138
:10E6800040E050E86BE375E4409317115093181184
:10E690006093191170931A118093131190931411B0
:10E6A000A0931511B09316111092970F1092980F16
:10E6B0001092990F10929A0F80E29EE4A0E0B0E0D1
:10E6C0008093E0069093E106A093E206B093E30600
:10E6D0001092930F1092940F1092950F1092960F24
:10E6E00080E090E0A0E0B1E48093C90F9093CA0F5E
:10E6F000A093CB0FB093CC0F8093CD0F9093CE0F00
:10E70000A093CF0FB093D00F8DEC9CECACECBEE39C
:10E710008093D10F9093D20FA093D30FB093D40FC7
:10E7200080E090E0A0E2B1E48093D50F9093D60F03
:10E73000A093D70FB093D80F8CE0E9E5F7E0DF01A5
:10E740001D928A95E9F70E94CDBC8AE999E9A9E969
:10E75000BFEB8093190990931A09A0931B09B093FA
:10E760001C0984EB90E09093DD068093DC0680EF3B
:10E7700090E09093DF068093DE0686E490E090932D
:10E78000D9068093D8068EE690E09093DB068093BE
:10E79000DA061092D5061092D4061092D70610927F
:10E7A000D6068CE59FE8AEE5B2E48093360F9093F1
:10E7B000370FA093380FB093390F89E895E6AEE88C
:10E7C000BFE38093320F9093330FA093340FB09335
:10E7D000350F81ED9BEDADE2B4E480932E0F909365
:10E7E0002F0FA093300FB093310F80E090E0A2E2A2
:10E7F000B3E48093420F9093430FA093440FB093E0
:10E80000450F87E092E4A2E3B0E480933E0F90933B
:10E810003F0FA093400FB093410F80E192E3A0E13E
:10E82000B5E480933A0F90933B0FA0933C0FB093C5
:10E830003D0F1092D30680E090E0A0E4B0E4809316
:10E84000CF069093D006A093D106B093D20681E074
:10E850008093540780935E06C2DEEEEDFAE1849168
:10E86000EF012196882321F00E94AA46FE01F7CFEE
:10E87000E8E1FDE08491EF012196882321F00E94D8
:10E88000AA46FE01F7CFDF91CF9108952F923F92D4
:10E890004F925F926F927F928F929F92AF92BF92B0
:10E8A000CF92DF92EF92FF920F931F93CF93DF935C
:10E8B000CDB7DEB7C655D1090FB6F894DEBF0FBE8F
:10E8C000CDBF2DB73EB765963FAF2EAF65972B9660
:10E8D0001FAE1EAE2B9784E690E029969FAF8EAFB9
:10E8E00029979E01275B3F4F44E050E0BE01635CE7
:10E8F0007F4FCE01895B9F4F63D89E01275B3F4FBF
:10E9000042E050E0BE016B5B7F4FCE01895B9F4FC1
:10E9100057D843E050E0BE01635C7F4F88E493E04A
:10E920000F94D51F892B91F18DAD863519F08FE3AA
:10E930008DAF1EAEEEEDFAE184918F010F5F1F4F98
:10E94000882321F00E94AA46F801F6CFE4EEFDE00C
:10E9500084918F010F5F1F4F882321F00E94AA46E8
:10E96000F801F6CFBE01635C7F4F8BED9DE07DDA51
:10E97000EDECFDE084918F010F5F1F4F882321F0A4
:10E980000E94AA46F801F6CF3BDE3AC46DB67EB6C9
:10E9900019AE1AAE1BAE1CAE2B961FAE1EAE2B9739
:10E9A0009E01275B3F4F41E050E0BE016F5A7F4F11
:10E9B000CE01895B9F4F04D880E1EEEAF2E0DE01F0
:10E9C000919601900D928A95E1F780E1EEEBF2E0ED
:10E9D000DE01519601900D928A95E1F780E1EEEC0F
:10E9E000F2E09E012F5F3F4F7901D90101900D9216
:10E9F0008A95E1F76296CFAC6297D12C33E0C30ED3
:10EA0000D11CCC0CDD1CCC0CDD1C8DB79EB78C1939
:10EA10009D090FB6F8949EBF0FBE8DBFEDB7FEB730
:10EA200031964F012DB73EB72C193D090FB6F8941A
:10EA30003EBF0FBE2DBF8DB79EB701965C01EDB7EF
:10EA4000FEB7EC19FD090FB6F894FEBF0FBEEDBF7F
:10EA50000DB71EB70F5F1F4F9E01275B3F4FA601EB
:10EA6000B401CE01895B9F4F0E94E06C9E01275B41
:10EA70003F4FA601B501CE01895B9F4F0E94E06C1C
:10EA80009E01275B3F4FA601B801CE01895B9F4FD6
:10EA90000E94E06C62964FAD629750E04E5F5F4F10
:10EAA00023E031E167963FAF2EAF67976BE97FE0D8
:10EAB000ACEABFE080E090E020E030E0421753078E
:10EAC00014F0640105C0F1E2CF2ED12CCC0EDD1E76
:10EAD000C80ED91EF60120803180428053802D92CD
:10EAE0003D924D925D924217530714F0650105C0A7
:10EAF000E1E1CE2ED12CCC0EDD1EC80ED91EF601C2
:10EB00002080318042805380FB01219231924192DA
:10EB10005192BF014217530714F0680101C0670109
:10EB2000C80ED91EF601208031804280538067963E
:10EB3000EEADFFAD67972192319241925192679667
:10EB4000FFAFEEAF67972F5F3F4F0496243031053C
:10EB500009F0B4CF9E01275B3F4F44E050E06BE1EA
:10EB600071E1CE01895B9F4F0E94E06C9E01275BA3
:10EB70003F4F44E050E067E171E1CE01895B9F4F78
:10EB80000E94E06C9E01275B3F4F44E050E063E150
:10EB900071E1CE01895B9F4F0E94E06C9E01275B73
:10EBA0003F4F44E050E067E97FE0CE01895B9F4F33
:10EBB0000E94E06C9E01275B3F4F44E050E063E918
:10EBC0007FE0CE01895B9F4F0E94E06C9E01275B36
:10EBD0003F4F44E050E060EE76E0CE01895B9F4F0E
:10EBE0000E94E06C9E01275B3F4F40E150E069ECE2
:10EBF0007FE0CE01895B9F4F0E94E06C9E01275B06
:10EC00003F4F4CE050E069E577E0CE01895B9F4FD4
:10EC10000E94E06C9E01275B3F4F44E050E0BE0144
:10EC2000675C7F4FCE01895B9F4F0E94E06C9E0125
:10EC3000275B3F4F41E050E0BE01605B7F4FCE015C
:10EC4000895B9F4F0E94E06C9E01275B3F4F44E031
:10EC500050E0BE01675C7F4FCE01895B9F4F0E94F1
:10EC6000E06C9E01275B3F4F41E050E0BE01615BDD
:10EC70007F4FCE01895B9F4F0E94E06C9E01275B16
:10EC80003F4F41E050E0BE01625B7F4FCE01895BA8
:10EC90009F4F0E94E06C6096EFAC60972F968FAD0F
:10ECA0002F97E89E7001112400E010E00E151F055B
:10ECB00081F09E01275B3F4F44E050E0BE01675C5E
:10ECC0007F4FCE01895B9F4F0E94E06C0F5F1F4F0B
:10ECD000EDCF2B960EAD1FAD2B9729968EAD9FAD28
:10ECE000299790936B0280936A029E01275B3F4FA6
:10ECF00044E050E069E179E0CE01895B9F4F0E94DA
:10ED0000E06C2B961FAF0EAF2B979E01275B3F4FFA
:10ED100044E250E067EE71E1CE01895B9F4F0E94B3
:10ED2000E06C9E01275B3F4F41E050E0BE01635B1A
:10ED30007F4FCE01895B9F4F0E94E06C9E01275B55
:10ED40003F4F41E050E0BE01645B7F4FCE01895BE5
:10ED50009F4F0E94E06C9E01275B3F4F44E050E0D4
:10ED6000BE016B5C7F4FCE01895B9F4F0E94E06CC0
:10ED70009E01275B3F4F44E050E0BE016F5C7F4F38
:10ED8000CE01895B9F4F0E94E06C2E96EFAC2E97D0
:10ED90002D968FAD2D97E89E7001112400E010E0B4
:10EDA0009E01275B3F4F0E151F0569F044E050E0C0
:10EDB000BE01675C7F4FCE01895B9F4F0E94E06C74
:10EDC0000F5F1F4FEDCF41E050E0BE016E5A7F4F05
:10EDD000CE01895B9F4F0E94E06C9E01275B3F4FF5
:10EDE00044E050E0BE01675C7F4FCE01895B9F4FDE
:10EDF0000E94E06C9E01275B3F4F41E050E0BE0166
:10EE0000655B7F4FCE01895B9F4F0E94E06C19AE1E
:10EE10001AAE1BAE1CAE1DE011509E01275B3F4F8A
:10EE200044E050E0112349F0BE01675C7F4FCE0102
:10EE3000895B9F4F0E94E06CEFCF6CED76E0CE01D6
:10EE4000895B9F4F0E94E06C9E01275B3F4F44E02F
:10EE500050E068ED76E0CE01895B9F4F0E94E06C48
:10EE60009E01275B3F4F44E050E064ED76E0CE0129
:10EE7000895B9F4F0E94E06C9E01275B3F4F44E0FF
:10EE800050E0BE01675C7F4FCE01895B9F4F0E94BF
:10EE9000E06C112311F004E03CC0C9ACDAACEBAC7F
:10EEA000FCAC20E030E84BE355E4C701B6010F9419
:10EEB0005B18882381F3C092360FD092370FE0920F
:10EEC000380FF092390F9E01275B3F4F44E050E02E
:10EED00062E37FE0CE01895B9F4F0E94E06C9E0160
:10EEE000275B3F4F44E050E06EE27FE0CE01895B5C
:10EEF0009F4F0E94E06C9E01275B3F4F44E050E033
:10EF0000BE01675C7F4FCE01895B9F4F0E94E06C22
:10EF100010C0015071F09E01275B3F4F44E050E06C
:10EF2000BE01675C7F4FCE01895B9F4F0E94E06C02
:10EF3000F0CF1F5F153009F09FCF9E01275B3F4F39
:10EF400042E050E0BE016D5B7F4FCE01895B9F4F79
:10EF50000E94E06C9E01275B3F4F44E050E0BE0101
:10EF6000675C7F4FCE01895B9F4F0E94E06CC9AC0C
:10EF7000DAACEBACFCAC20E030E84BE355E4C70185
:10EF8000B6010F945B18882301F1C092420FD09212
:10EF9000430FE092440FF092450F9E01275B3F4FD5
:10EFA00044E050E06EE37FE0CE01895B9F4F0E941A
:10EFB000E06C9E01275B3F4F44E050E06AE37FE056
:10EFC000CE01895B9F4F0E94E06C9E01275B3F4F03
:10EFD00042E050E0BE016F5B7F4FCE01895B9F4FE7
:10EFE0000E94E06C9E01275B3F4F41E050E0BE0174
:10EFF0006E5A7F4FCE01895B9F4F0E94E06C19E0F3
:10F0000011509E01275B3F4F112359F044E050E01F
:10F01000BE01675C7F4FCE01895B9F4F0E94E06C11
:10F02000EFCF41E050E063ED76E0CE01895B9F4F8A
:10F030000E94E06C9E01275B3F4F44E050E0BE0120
:10F04000675C7F4FCE01895B9F4F0E94E06C11117E
:10F050000CC089AD9AADABADBCAD8093CF0690939B
:10F06000D006A093D106B093D2061F5F153011F7DA
:10F070001BE09E01275B3F4F42E050E0BE016B5C0E
:10F080007F4FCE01895B9F4F0E94E06C115089F742
:10F090009E01275B3F4F44E050E0BE01675C7F4F1D
:10F0A000CE01895B9F4F0E94E06C9E01275B3F4F22
:10F0B00044E050E0BE01675C7F4FCE01895B9F4F0B
:10F0C0000E94E06C14E0115071F09E01275B3F4FED
:10F0D00044E050E0BE016F5C7F4FCE01895B9F4FE3
:10F0E0000E94E06CF0CF2B962EAD3FAD2B9727966C
:10F0F0008EAD9FAD27972817390709F039C06FDA11
:10F10000EEEDFAE184918F010F5F1F4F811103C073
:10F1100008E413E004C00E94AA46F801F3CFF80106
:10F1200081918F01882319F00E94AA46F8CF299671
:10F130006EAD7FAD29976456710980EB9DE00E940A
:10F140006A8B2B964EAD5FAD2B9760E070E083EA43
:10F150009DE00E94838BE0EAFDE084918F010F5FC8
:10F160001F4F882309F447C00E94AA46F801F5CF33
:10F17000E3EAFAE184918F010F5F1F4F882321F0AA
:10F180000E94AA46F801F6CFE0E8FDE084918F01E5
:10F190000F5F1F4F882321F00E94AA46F801F6CF87
:10F1A00027966EAD7FAD279780E090E04AE00E9401
:10F1B000DE8AEBE7FDE084918F010F5F1F4F88230C
:10F1C00021F00E94AA46F801F6CF2B966EAD7FADD6
:10F1D0002B9780E090E04AE00E94DE8AEBE6FDE0BB
:10F1E00084918F010F5F1F4F882321F00E94AA4650
:10F1F000F801F6CF05DA0FB6F8947EBE0FBE6DBEED
:10F2000080E00E94594E9091CE0681E08927659654
:10F210002EAD3FAD65970FB6F8943EBF0FBE2DBF24
:10F22000CA5ADF4F0FB6F894DEBF0FBECDBFDF91D5
:10F23000CF911F910F91FF90EF90DF90CF90BF90F3
:10F24000AF909F908F907F906F905F904F903F9086
:10F250002F9008957F928F929F92AF92BF92CF92FC
:10F26000DF92EF92FF920F931F93CF93DF930CE205
:10F2700013E0CCEADFE0712CF80181918F010E944C
:10F28000C448882309F46CC0F3E07F1263C00E9475
:10F290003E476B017C0120E030E040EA51E40F94EE
:10F2A0005B1887FF4EC0A70196016091B80F70915F
:10F2B000B90F8091BA0F9091BB0F0F946A1D4B014B
:10F2C0005C019B01AC016091D50F7091D60F8091CC
:10F2D000D70F9091D80F0F94C0186093D50F7093EB
:10F2E000D60F8093D70F9093D80FA501940160910A
:10F2F000A70F7091A80F8091A90F9091AA0F0F945A
:10F30000C0186093A70F7093A80F8093A90F9093D4
:10F31000AA0F6091CA067091CB068091CC0690919D
:10F32000CD060F945F18A50194010F94C0180F9497
:10F33000D71D6093CA067093CB068093CC0690933A
:10F34000CD06C092B80FD092B90FE092BA0FF092EA
:10F35000BB0F06C00E943E47688379838A839B83E4
:10F360007394249684E0781287CFDF91CF911F9118
:10F370000F91FF90EF90DF90CF90BF90AF909F9054
:10F380008F907F90BAC80F931F93CF93DF93CDB721
:10F39000DEB72C970FB6F894DEBF0FBECDBF8091BD
:10F3A0006D0790916E07A0916F07B0917007409123
:10F3B000690750916A0760916B0770916C07009123
:10F3C00065071091660720916707309168070983E8
:10F3D0001A832B833C834D835E836F837887898771
:10F3E0009A87AB87BC87AE01475F5F4FBE016B5FFB
:10F3F0007F4FCE0101960E94478321E737E0AE019F
:10F40000475F5F4FBE016B5F7F4FCE0101960E9449
:10F41000A8712C960FB6F894DEBF0FBECDBFDF915A
:10F42000CF911F910F9108959F92AF92BF92CF926B
:10F43000DF92EF92FF920F931F93CF93DF93BCE283
:10F44000AB2EB3E0BB2E05E617E0C9E5D7E0912C63
:10F45000F50181915F010E94C4488823F9F00E9460
:10F460003E476B017C01288139814A815B810F9481
:10F470008D1C9B01AC01F8016081718182819381B7
:10F480000F948E1CF8016083718382839383C882FA
:10F49000D982EA82FB82892D0E94294893940C5FCD
:10F4A0001F4F2496F3E09F12D3CF6DDFDF91CF91F2
:10F4B0001F910F91FF90EF90DF90CF90BF90AF9092
:10F4C0009F900D9488034F925F926F927F928F92DC
:10F4D0009F92AF92BF92CF92DF92EF92FF920F93E3
:10F4E0001F93CF93DF93CDB7DEB72E970FB6F89467
:10F4F000DEBF0FBECDBF109168021F3FE9F00E9432
:10F50000A24CC090A506D090A606E090A706F09069
:10F51000A8066C197D098E099F0997FD0DC02091E1
:10F52000301280912F1230E090E001968F70992771
:10F530002817390709F02DC20E941A848091BD0650
:10F5400082FF3EC08091BC0681113CC091E0909347
:10F55000BC0680913209892780931F1110923209CD
:10F5600083E08093A8021092BD060E94A24C6C50CA
:10F570007E4F8F4F9F4F6093A9067093AA0680938A
:10F58000AB069093AC0688E893E19E878D8782E076
:10F5900090E09A838983BE01635F7F4FCE0101961D
:10F5A0000E94ADE316E0115069F081E392E10E9400
:10F5B0006C5562E070E080E090E00E94074CF3CF71
:10F5C0001092BC06F9B0F4FAFF24F0F881E0F826B6
:10F5D0004091BB062F2D30E0842F90E0281739078B
:10F5E000A9F0FF2009F427C20E94B1618091BB06F7
:10F5F000823029F060E08AE09DE00E949E84F092D3
:10F60000BB0683E08093A8020E94C7C50E94A24C5B
:10F610006B017C018091B7069091B806A091B90664
:10F62000B091BA06A7019601281B390B4A0B5B0B58
:10F6300057FF05C08091B606882309F448C2D70158
:10F64000C6018C599F4FAF4FBF4F8093B706909321
:10F65000B806A093B906B093BA068091B5061816FD
:10F660002CF48091B506823074F408C08091B50600
:10F67000992781950CF4909502972CF480911F1195
:10F6800081119DC0ADC080912711882309F470C0FD
:10F690008091B50618165CF48091B506992787FD10
:10F6A000909597FD0196BC01759567950DC0809169
:10F6B000B506992787FD909597FD019695958795B5
:10F6C00066277727681B790B8090FE109090FF10BB
:10F6D000A0900011B090011181149104A104B10413
:10F6E00029F421E030E040E050E039C0882777FD80
:10F6F0008095982F0F9461182B013C01C701B6012A
:10F70000681979098A099B090F945F189B01AC015C
:10F71000C301B2010F946A1D20E030E04AE754E4CF
:10F720000F94C0184B015C0120E030E040E253E44C
:10F730000F94B41E87FF0FC020E030E046E952E48A
:10F74000C501B4010F94B41E87FDCBCF2AE030E091
:10F7500040E050E004C024E630E040E050E0C092D9
:10F76000FE10D092FF10E0920011F092011104C03F
:10F7700021E030E040E050E0A091B506BB27A7FDB6
:10F78000B0950F94781C22E030E040E050E00F94F8
:10F79000521C8091231190912411A0912511B091B8
:10F7A0002611820F931FA41FB51F809323119093DE
:10F7B0002411A0932511B09326111092B506D701FC
:10F7C000C6018856954CAF4FBF4F8093B1069093BA
:10F7D000B206A093B306B093B40681E08093A8026A
:10F7E000209194023091950247EF223F340749F46B
:10F7F000809169029FEF980F90936902882309F422
:10F8000025C12B5A3E4F79F48091AE069091AD06FA
:10F81000891748F4909169022FEF290F209369020C
:10F82000992309F423C12FB7F8948091B8099091D6
:10F83000B909A091BA09B091BB092FBF4091A802A4
:10F84000411105C02091B606222309F465C00AE0E3
:10F85000B695A795979587950A95D1F7009721E0DA
:10F86000A207B10520F08FEF9FEFA0E0B0E09695E2
:10F870008795009741F02091AF063091B006281788
:10F88000390708F049C08091B606811111C0423095
:10F8900050F0443028F0443031F41092A80203C0F4
:10F8A00081E08093A8020E94725A81E08093B6069C
:10F8B00084E00E947C9181E08093CD11E0919402DC
:10F8C000F0919502199510921F118091B606882328
:10F8D00051F00E94EE9091E0811101C090E0909370
:10F8E000B6069111DBC08090AF069090B006A12CB7
:10F8F000B12C0E94A24C6C197D098E099F098616B5
:10F900009706A806B90640F40E94A24C6C197D091E
:10F910007093B0066093AF06809194029091950227
:10F92000825F974F21F080917D06882379F048E926
:10F93000C40E4AE3D41EE11CF11CC092B106D09261
:10F94000B206E092B306F092B4060FC08091B10601
:10F950009091B206A091B306B091B406C81AD90A24
:10F96000EA0AFB0AF7FE0E9417868091B60681110B
:10F97000AEC08091A802813049F008F4A8C084305C
:10F9800008F0A5C081E08093A802A1C01092A8024F
:10F990009EC054E01502F0011124E85CFC4F20E009
:10F9A00030E040E752E460817181828193810F945D
:10F9B0006A1D4B015C018091650790916607A091DB
:10F9C0006707B091680789839A83AB83BC83809172
:10F9D000690790916A07A0916B07B0916C078D83BE
:10F9E0009E83AF83B88780916D0790916E07A09139
:10F9F0006F07B091700789879A87AB87BC87AE0184
:10FA0000475F5F4FBE016B5F7F4FCE0101963FD6D0
:10FA1000C12C8501740121E737E0AE01475F5F4FDC
:10FA2000BE016B5F7F4FCE0101960E94A9CF8FEF81
:10FA30008093680281CD10925E1210925F12423064
:10FA400009F4DDCD60E08DEF9CE0D7CD8CE08093B4
:10FA500069028091AF069091B00601979093B0062D
:10FA60008093AF0681E08093A802CBCE96E090937E
:10FA7000690291E09093A8028F5F8093AE06D70150
:10FA8000C6018856954CAF4FBF4F8093B1069093F7
:10FA9000B206A093B306B093B406C5CE8090AF066D
:10FAA0009090B006A12CB12C0E94A24C6C197D093B
:10FAB0008E099F0986169706A806B90640F40E948B
:10FAC000A24C6C197D097093B0066093AF062E9618
:10FAD0000FB6F894DEBF0FBECDBFDF91CF911F915F
:10FAE0000F91FF90EF90DF90CF90BF90AF909F90DD
:10FAF0008F907F906F905F904F900895CF92EF928C
:10FB0000FF920F931F93CF93DF93CDB7DEB72C9760
:10FB10000FB6F894DEBF0FBECDBFC09085068091B2
:10FB20006D0790916E07A0916F07B091700740919B
:10FB3000690750916A0760916B0770916C0700919B
:10FB40006507109166072091670730916807098360
:10FB50001A832B833C834D835E836F8378878987E9
:10FB60009A87AB87BC87AE01475F5F4FBE016B5F73
:10FB70007F4FCE0101968BD5E0900A02F0900B02E8
:10FB800000910C0210910D0221E737E0AE01475FB2
:10FB90005F4FBE016B5F7F4FCE0101960E94A9CFE0
:10FBA0002C960FB6F894DEBF0FBECDBFDF91CF917C
:10FBB0001F910F91FF90EF90CF9008958F929F9299
:10FBC000AF92BF92CF92EF92FF920F931F93CF937A
:10FBD000DF93CDB7DEB72C970FB6F894DEBF0FBE1C
:10FBE000CDBF4B015C01C090850680913E04909191
:10FBF0003F04A0914004B091410440913A045091D7
:10FC00003B0460913C0470913D04009136041091D6
:10FC10003704209138043091390409831A832B83E7
:10FC20003C834D835E836F83788789879A87AB8710
:10FC3000BC87AE01475F5F4FBE016B5F7F4FCE0158
:10FC4000019625D58501740122E434E0AE01475FB9
:10FC50005F4FBE016B5F7F4FCE0101960E94A9CF1F
:10FC60002C960FB6F894DEBF0FBECDBFDF91CF91BB
:10FC70001F910F91FF90EF90CF90BF90AF909F900A
:10FC80008F900895FC01138212828DEB93E0918393
:10FC9000808313AE14AE15AECF0104961186108684
:10FCA00013861286158621E0248722E22687138A8E
:10FCB000128A20E030E04FEFDC01A20FB31F9396D1
:10FCC0004C932F5F3F4F2E303105B1F741E044A3F5
:10FCD00022ED32E4328F218F438F148E158E20E473
:10FCE000268F178E20EE32E436AB25AB7783668302
:10FCF0000C94A24B0C943446492F441F4427441FB4
:10FD000029F022273327281B390B01C09C01883E8C
:10FD10009340ACF0C90168EE73E00F946A1FCB0109
:10FD2000EAE0F0E0BF010F946A1F805D8093E10F6D
:10FD3000C90164E670E00F946A1FCB0112C024363B
:10FD40003105B4F0442311F08DE201C080E28093CC
:10FD5000E10FC90164E670E00F946A1FCB01EAE08D
:10FD6000F0E0BF010F946A1F805D8093E20F11C025
:10FD700080E28093E10F8093E20F2A3031059CF0FE
:10FD8000442311F08DE201C080E28093E20FEAE0AB
:10FD9000F0E0C901BF010F946A1FCB01BF010F94AE
:10FDA0006A1F805D05C0442311F08DE201C080E22E
:10FDB0008093E30FC9016AE070E00F946A1F805DD1
:10FDC0008093E40F81EE9FE008959C0197FD0EC0A3
:10FDD0008436910584F064E670E00F946A1FCB01CD
:10FDE0006AE070E00F946A1F805D06C0319521952E
:10FDF00031098DE201C080E28093E20F2A303105A3
:10FE000064F0EAE0F0E0C901BF010F946A1FCB0182
:10FE1000BF010F946A1F805D01C080E28093E30FF1
:10FE2000C9016AE070E00F946A1F805D8093E40F5F
:10FE300082EE9FE00895CF92DF92EF92FF920F93B0
:10FE40001F93CF93DF93E091DF0EF091E00E82815C
:10FE50009381A481B581181619061A061B06D4F5DC
:10FE60008091DE0E909141076091400780FF10C0A5
:10FE700083B186FB222720F99E7F292B20934107FF
:10FE8000962F9170922331F18091960781601DC069
:10FE900080B1292F30E08695869591E08927482FFB
:10FEA000417050E088279927841B950B8227932760
:10FEB000807199278227932780934107962F90710D
:10FEC000982341F08091960780618093960780E0A7
:10FED0000E942145E091DF0EF091E00E868197812E
:10FEE000A085B185181619061A061B060CF040C02D
:10FEF0009091DE0E809141072091400791FF1AC03A
:10FF000033B190E035FBCC24C0F8D12CD194C1940E
:10FF1000D108C826D92632E0C322DD24C826D92636
:10FF2000C0924107822F82708C2111F18091960737
:10FF3000826019C030B190E031FBEE24E0F8F12C82
:10FF4000F194E194F108E826F92630E2E322FF2457
:10FF5000E826F926E0924107822F80728E2141F037
:10FF60008091960780628093960781E00E942145E8
:10FF7000E091DF0EF091E00E82859385A485B58532
:10FF8000181619061A061B060CF07CC08091DE0EAE
:10FF90002091410782FF59C080915807882309F1B9
:10FFA00083B130E082958F7091E08927082F01702E
:10FFB00010E01195019511090227132704701127EC
:10FFC0000227132700934107809140078470802304
:10FFD00041F08091960784608093960782E00E94AA
:10FFE000214580915807882309F44CC020B18091A5
:10FFF000410790E020952170C22F20E0D22FD195AB
:020000021000EC
:10000000C195D109C827D927C870DD27C827D927A6
:10001000C09341078091400788708C2399F1E0914B
:10002000DF0EF091E00E82859385A485B5851816C4
:1000300019061A061B069CF5809196078860809326
:10004000960782E00E9421452AC086B130E09927B8
:1000500087FD9095990F880B982F8227932780749E
:1000600099278227932780934107909140079074A6
:10007000982341F08091960780648093960782E0F0
:100080000E9421458091410780934007DF91CF91E5
:100090001F910F91FF90EF90DF90CF900895809186
:1000A0009607886080939607EDCF4F925F926F928C
:1000B0007F928F929F92AF92BF92CF92DF92EF92F8
:1000C000FF920F931F93CF93DF9300D01F92CDB772
:1000D000DEB78C01DC014D905D906D907C901397A4
:1000E00014968D909D90AD90BC90179718968D9119
:1000F0009D910D90BC91A02D89839A83AB83BC8385
:10010000A3019201C301B2010F94C0186B017C01DD
:10011000A5019401C501B4010F94C0189B01AC0165
:10012000C701B6010F948E1C6B017C0129813A81B5
:100130004B815C81CA01B9010F94C0189B01AC01CD
:10014000C701B6010F948E1C0F94F91E9B01AC01E0
:1001500060E070E080E89FE30F946A1D6B017C0112
:100160009B01AC01C301B2010F94C018F801608378
:10017000718382839383A7019601C501B4010F9413
:10018000C018D80114966D937D938D939C93179707
:10019000A701960169817A818B819C810F94C01897
:1001A000F80160877187828793870F900F900F9077
:1001B0000F90DF91CF911F910F91FF90EF90DF9003
:1001C000CF90BF90AF909F908F907F906F905F90F7
:1001D0004F9008954F925F926F927F928F929F926D
:1001E000AF92BF92CF92DF92EF92FF92CF93DF93C5
:1001F000CDB7DEB728970FB6F894DEBF0FBECDBFE0
:100200002496AEADBFAD24978D919D910D90BC917C
:10021000A02D89839A83AB83BC832296EEADFFAD7C
:100220002297C080D180E280F380AEADBFAD8D90CB
:100230009D90AD90BC902E8D3F8D48A159A1C501D8
:10024000B4010F94C0182B013C012AA53BA54CA575
:100250005DA5C701B6010F94C0189B01AC01C30195
:10026000B2010F948E1C2B013C012EA93FA948AD71
:1002700059AD69817A818B819C810F94C0189B0153
:10028000AC01C301B2010F948E1C6D837E838F83FA
:1002900098872AA13BA14CA15DA1C501B4010F948F
:1002A000C0182B013C012EA53FA548A959A9C7019B
:1002B000B6010F94C0189B01AC01C301B2010F94A9
:1002C0008E1C2B013C012AAD3BAD4CAD5DAD69816F
:1002D0007A818B819C810F94C0189B01AC01C30172
:1002E000B2010F948E1C2B013C012A8D3B8D4C8D4D
:1002F0005D8DC501B4010F94C0184B015C012EA1A6
:100300003FA148A559A5C701B6010F94C0189B018C
:10031000AC01C501B4010F948E1C6B017C012AA9AC
:100320003BA94CA95DA969817A818B819C810F943D
:10033000C0189B01AC01C701B6010F948E1CEEAD35
:10034000FFAD60837183828393838D819E81AF81B2
:10035000B8852296EEADFFAD229780839183A2836C
:10036000B3832496AEADBFAD24974D925D926D924E
:100370007C92139728960FB6F894DEBF0FBECDBFC0
:10038000DF91CF91FF90EF90DF90CF90BF90AF9033
:100390009F908F907F906F905F904F9008954F92B5
:1003A0005F926F927F928F929F92AF92BF92CF9205
:1003B000DF92EF92FF920F931F93CF93DF93CDB70E
:1003C000DEB7C454D1090FB6F894DEBF0FBECDBF5F
:1003D0008C0180916006882309F441C1C090EB1123
:1003E000D090EC11E090ED11F090EE112091EF1112
:1003F0003091F0114091F1115091F21129AB3AABCB
:100400004BAB5CAB4090F3115090F4116090F51140
:100410007090F6118091F7119091F811A091F91157
:10042000B091FA1125968CAF9DAFAEAFBFAF2597B7
:100430002091FB113091FC114091FD115091FE1162
:100440002DAB3EAB4FAB58AF8090FF119090001298
:10045000A0900112B0900212409103125091041228
:100460006091051270910612809107129091081206
:10047000A0910912B0910A1289AF9AAFABAFBCAF8D
:100480008091E7119091E811A091E911B091EA11E2
:1004900089839A83AB83BC834D825E826F82788628
:1004A00089869A86AB86BC86CD86DE86EF86F88AFC
:1004B00025968CAD9DADAEADBFAD2597898B9A8B42
:1004C000AB8BBC8B4D8B5E8B6F8B788F29A93AA938
:1004D0004BA95CA9298F3A8F4B8F5C8F8DA99EA960
:1004E000AFA9B8AD8D8F9E8FAF8FB8A329AD3AADB0
:1004F0004BAD5CAD29A33AA34BA35CA3209161064D
:10050000309162064091630650916406D8016D9166
:100510007D918D919C910F948D1C20E030E048E9F5
:1005200051E40F948E1C6DA77EA78FA798AB2091E6
:100530006506309166064091670650916806F8019D
:1005400064817581868197810F948D1C20E030E055
:1005500041E853E40F948D1C69A77AA78BA79CA749
:100560002091690630916A0640916B0650916C06A5
:10057000D80118966D917D918D919C911B970F9448
:100580008D1C6DA37EA38FA398A7CE0185969F9304
:100590008F9304969F938F9304969F938F93EDB7B9
:1005A000FEB7B4970FB6F894FEBF0FBEEDBFADB760
:1005B000BEB7119684E2FE01319601900D928A95A4
:1005C000E1F708DE20E030E048E951E46DA57EA5C2
:1005D0008FA598A90F948D1C209161063091620619
:1005E00040916306509164060F948E1CD8016D9360
:1005F0007D938D939C93139720E030E041E853E482
:1006000069A57AA58BA59CA50F948E1C20916506E3
:100610003091660640916706509168060F948E1CD3
:10062000F8016483758386839783209169063091EE
:100630006A0640916B0650916C066DA17EA18FA158
:1006400098A50F948E1CD80118966D937D938D9369
:100650009C931B970FB6F894DEBF0FBECDBFCC5B4B
:10066000DF4F0FB6F894DEBF0FBECDBFDF91CF9145
:100670001F910F91FF90EF90DF90CF90BF90AF90C0
:100680009F908F907F906F905F904F900895CF9242
:10069000DF92EF92FF920F931F93CF93DF93CDB72B
:1006A000DEB72C970FB6F894DEBF0FBECDBF6C013E
:1006B0007B018A0180916006882309F4ACC02091F7
:1006C0006106309162064091630650916406F6011E
:1006D00060817181828193810F948D1C20E030E0D4
:1006E00048E951E40F948E1C69877A878B879C8731
:1006F0002091650630916606409167065091680624
:10070000F70160817181828193810F948D1C20E0BB
:1007100030E041E853E40F948D1C6D837E838F831A
:1007200098872091690630916A0640916B06509136
:100730006C06F80160817181828193810F948D1C18
:1007400069837A838B839C83CE0101969F938F93D9
:1007500004969F938F9304969F938F938DB79EB724
:1007600084970FB6F8949EBF0FBE8DBFADB7BEB7CE
:10077000119684E2E7EEF1E101900D928A95E1F79E
:1007800029DD20E030E048E951E469857A858B85F0
:100790009C850F948D1C20916106309162064091DA
:1007A0006306509164060F948E1CF601608371837A
:1007B0008283938320E030E041E853E46D817E81C1
:1007C0008F8198850F948E1C209165063091660666
:1007D00040916706509168060F948E1CF701608364
:1007E0007183828393832091690630916A064091D8
:1007F0006B0650916C0669817A818B819C810F9484
:100800008E1CF80160837183828393830FB6F89402
:10081000DEBF0FBECDBF2C960FB6F894DEBF0FBE65
:10082000CDBFDF91CF911F910F91FF90EF90DF909F
:10083000CF9008950F931F930E94A24C0091A90698
:100840001091AA062091AB063091AC06601B710B8B
:10085000820B930B97FD0FC08091030185FB8827C6
:1008600080F991E089279091030196FF8260629B55
:1008700084608093BD068091BD0681709091BD0615
:1008800091FD826090913F07891731F18130A9F085
:1008900028F0823041F0833059F01CC0913089F04B
:1008A000923099F017C0992361F0933071F012C023
:1008B000913059F0923071F404C0992331F09330A3
:1008C00049F49091B5069F5F03C09091B506915091
:1008D0009093B50680933F071F910F910895EEE026
:1008E000F2E080E09191911105C0282F482F421B22
:1008F00050E204C0863181F426E1F8CF822F90E0E7
:10090000342F320FFC01E25FFD4F363118F4508373
:100910002F5FF4CF108208958F5FE4CF209184067B
:1009200021110BC042E450E0BC018EE092E00F9434
:10093000E31FD5DF83E08093A802089567FF03C01B
:100940001092840660E02091840630E0462F5527FF
:1009500047FD5095421753076CF06093840642E4BC
:1009600050E0BC018EE092E00F94CC17B8DF83E03A
:100970008093A8020895CF92DF92EF92FF920F9397
:100980001F930E94A24C00913B0710913C072091BD
:100990003D0730913E076B017C01C01AD10AE20A83
:1009A000F30AF7FC13C020913A07209520933A07E9
:1009B000DC01CB018A549C4FAF4FBF4F80933B0764
:1009C00090933C07A0933D07B0933E0781E0909140
:1009D0003A07911101C080E01F910F91FF90EF90B5
:1009E000DF90CF900895CF92DF92EF92FF92CF9356
:1009F000C82F0E94A24C6B017C0124EA30E74DE72E
:100A00005FE36091190F70911A0F80911B0F909105
:100A10001C0F0F945B1887FF04C040E050E0BA0140
:100A200004C04AEF50E060E070E04C0D5D1D6E1DAB
:100A30007F1D4093A5065093A6066093A70670936A
:100A4000A806C0936802CF91FF90EF90DF90CF90FF
:100A50000895209139072630D8F486E0289FF001C8
:100A60001124EB5EF84F809194029091950291834E
:100A700080838091231190912411A0912511B09130
:100A8000261182839383A483B5832F5F2093390734
:100A900008956F927F928F929F92AF92BF92CF9262
:100AA000DF92EF92FF920F931F93CF93DF9300D0CB
:100AB0001F92CDB7DEB76C013B0147015801298376
:100AC0003A834B835C83C5DF83E08093A802D09296
:100AD000C80FC092C70F7092C60F6092C50F2981D0
:100AE0003A814B815C81CA01B9010F94D21D609398
:100AF000C10F7093C20F8093C30F9093C40F0F94D4
:100B000061186B017C019B01AC01C501B4010F941C
:100B10008D1C0F94D21D6093BD0F7093BE0F8093F8
:100B2000BF0F9093C00FA7019601F30160817181FF
:100B3000828193810F948D1C0F94D71D6093231194
:100B400070932411809325119093261187E691ECE0
:100B500090939502809394020F900F900F900F90B6
:100B6000DF91CF911F910F91FF90EF90DF90CF9089
:100B7000BF90AF909F908F907F906F90089520913D
:100B800094023091950228173907D9F09093950275
:100B90008093940240932311509324116093251164
:100BA00070932611825F974F21F410927D06109268
:100BB000390782E08093A80281E08093211110928E
:100BC000B6060895CF93DF931F921F92CDB7DEB77D
:100BD00089839A833EDF40E050E0BA0189819A819F
:100BE0000F900F90DF91CF91CACF21E020937D0627
:100BF0006093190F70931A0F80931B0F90931C0F23
:100C000040E050E0BA0180919C0690919D06B7CFDC
:100C10006DEC7CEC8CEC9DE3E8CF60E070E080E86C
:100C20009FE3E3CF60E070E080E291E4DECF40E05C
:100C300050E0BA0182EF97EFA2CFE0913907EE239F
:100C400081F0E150E093390786E0E89FF00111243C
:100C5000EB5EF84F4281538164817581808191817F
:100C60008ECFE5CFCF93DF93EC016EE972E00AD827
:100C700081EB93E099838883DF91CF9108952FB71B
:100C8000F894909105019B7F909305012FBF87FDFC
:100C900096C0A3982FB7F894909105019460909313
:100CA00005012FBF880F2FB7F894909105019B7F06
:100CB000909305012FBF87FD8EC0A3982FB7F8949E
:100CC000909105019460909305012FBF880F2FB775
:100CD000F894909105019B7F909305012FBF87FDAC
:100CE00078C0A3982FB7F8949091050194609093E1
:100CF00005012FBF880F2FB7F894909105019B7FB6
:100D0000909305012FBF87FD62C0A3982FB7F89479
:100D1000909105019460909305012FBF880F2FB724
:100D2000F894909105019B7F909305012FBF87FD5B
:100D30004CC0A3982FB7F8949091050194609093BC
:100D400005012FBF880F2FB7F894909105019B7F65
:100D5000909305012FBF87FD36C0A3982FB7F89455
:100D6000909105019460909305012FBF982F990FE2
:100D70002FB7F894809105018B7F809305012FBFD9
:100D800097FD1FC0A3982FB7F89480910501846048
:100D9000809305012FBF2FB7F894809105018B7FB9
:100DA000809305012FBF96FD18C0A3989FB7F894B4
:100DB000809105018460809305019FBF0895A39AE7
:100DC00069CFA39AE0CFA39AC9CFA39AB3CFA39A2E
:100DD0009DCFA39A87CFA39A71CFA39AE7CFFC01A7
:100DE00020E03EE2DB014C91403241F0283011F42A
:100DF00030833196DB014C91408331962F5F6F5FDA
:100E00007F4F2B3079F710820895CF92DF92EF92C7
:100E1000FF92C0905706D0905806E0905906F09087
:100E20005A066091ED0E7091EE0E68507109882798
:100E300077FD8095982F0F9461189B01AC01C70135
:100E4000B6010F945B1887FF1DC020E030E040E042
:100E500050E4C701B6010F948E1C0F94D71D7093F8
:100E60007B0F60937A0F0E94A24C605A75418F4F9E
:100E70009F4F60937C0F70937D0F80937E0F9093B4
:100E80007F0F08C010927C0F10927D0F10927E0F82
:100E900010927F0FFF90EF90DF90CF900895B5CF25
:100EA000CF92DF92EF92FF92C0905306D0905406FB
:100EB000E0905506F09056066091F10E7091F20E9A
:100EC00065517109882777FD8095982F0F946118D7
:100ED0009B01AC01C701B6010F945B1887FF1DC0D1
:100EE00020E030E040E251E4C701B6010F948E1CCF
:100EF0000F94D71D7093810F6093800F0E94A24CB6
:100F0000605C73468F4F9F4F6093820F7093830F87
:100F10008093840F9093850F08C01092820F1092D7
:100F2000830F1092840F1092850FFF90EF90DF9047
:100F3000CF90089580E0B4CF4F925F926F927F92EE
:100F40008F929F92AF92BF92CF92DF92EF92FF92D9
:100F50000F931F93CF93DF932C0121E03EE081E0BC
:100F600090E0F90145915491441655060CF062C089
:100F7000AC0141505109DA01AA0FBB1FAA0FBB1FD8
:100F8000A150B24FFD0165917491440F551F440F5C
:100F9000551F4350524FFA0165907490FC01EE0FBB
:100FA000FF1FEE0FFF1FE150F24FA590B490FD011F
:100FB00005911491F901C591D491FA01859094900D
:100FC000882777FD8095982F0F9461186B017C011D
:100FD000B20166197709882777FD8095982F0F94BD
:100FE00061182B013C01B501601B710B882777FD4F
:100FF0008095982F0F9461189B01AC01C301B20139
:101000000F94C0182B013C01BE016819790988278B
:1010100077FD8095982F0F9461189B01AC01C30157
:10102000B2010F946A1D9B01AC01C701B6010F9478
:101030008E1C11C001962C5F3F4F8A33910509F039
:1010400090CFE3EEFEE065917491882777FD80955F
:10105000982F0F946118DF91CF911F910F91FF90FE
:10106000EF90DF90CF90BF90AF909F908F907F9048
:101070006F905F904F9008954F925F926F927F9222
:101080008F929F92AF92BF92CF92DF92EF92FF9298
:10109000CF93DF93CDB7DEB72C970FB6F894DEBFB2
:1010A0000FBECDBF8091570690915806A09159066A
:1010B000B0915A0689839A83AB83BC836091ED0E0D
:1010C0007091EE0E882777FD8095982F0F94611808
:1010D00029813A814B815C810F948D1C6B017C01CD
:1010E000609311077093120780931307909314076E
:1010F0002091420F3091430F4091440F5091450F82
:101100000F94C0186D837E838F83988760930D073B
:1011100070930E0780930F07909310072091090793
:1011200030910A0740910B0750910C07C701B60197
:101130000F948E1C4B015C016093090770930A07A2
:1011400080930B0790930C0720913E0F30913F0F37
:101150004091400F5091410F0F94C01869877A87D2
:101160008B879C876093050770930607809307071A
:101170009093080720ED3CEC4CE45DE360913A0F5E
:1011800070913B0F80913C0F90913D0F0F94C018D0
:101190002B013C0120910107309102074091030788
:1011A0005091040769817A818B819C810F948D1CF9
:1011B0009B01AC01C301B2010F94C0182B013C018B
:1011C00023E333E343E75FE36091FD067091FE069E
:1011D0008091FF06909100070F94C0189B01AC010D
:1011E000C301B2010F948E1C2B013C016093FD06DC
:1011F0007093FE068093FF069093000789819A8181
:10120000AB81BC818093010790930207A0930307F1
:10121000B093040729853A854B855C856D817E8175
:101220008F8198850F948E1CA30192010F948D1CC1
:101230002B013C0120E030E04EE453E40F94B41E57
:1012400020E030E0A9011816ACF4C701B6010F94F4
:10125000B41E18166CF5A7019601C501B4010F94D0
:101260008D1C6093090770930A0780930B07909376
:101270000C071EC0C301B2010F945B1887FF22C088
:1012800020E030E0A901C701B6010F945B1887FF89
:1012900016C0A7019601C501B4010F948D1C60937F
:1012A000090770930A0780930B0790930C0707C0F8
:1012B000412C512C8EE4682E83E4782E03C0412CFF
:1012C000512C3201C301B2012C960FB6F894DEBF47
:1012D0000FBECDBFDF91CF91FF90EF90DF90CF9009
:1012E000BF90AF909F908F907F906F905F904F9046
:1012F00008954F925F926F927F928F929F92AF92DA
:10130000BF92CF92DF92EF92FF920F931F93CF93F2
:10131000DF9300D01F92CDB7DEB70091F10E109190
:10132000F20E8090530690905406A0905506B0900F
:101330005606B801882777FD8095982F0F9461187D
:10134000A50194010F948D1C6B017C016093F9063B
:101350007093FA068093FB069093FC0620ED3CEC1C
:101360004CE45DE360912E0F70912F0F8091300F50
:101370009091310F0F94C0182B013C012091F5067C
:101380003091F6064091F7065091F806C501B40178
:101390000F948D1C9B01AC01C301B2010F94C018C6
:1013A0002B013C0123E333E343E75FE36091F10664
:1013B0007091F2068091F3069091F4060F94C01894
:1013C0009B01AC01C301B2010F948E1C69837A8327
:1013D0008B839C836093F1067093F2068093F306EF
:1013E0009093F4068092F5069092F606A092F70686
:1013F000B092F80680918206882321F081E08093E4
:10140000F006B9C020E030E040E251E4C701B60187
:101410000F94B41E181624F481E08093F006A4C043
:1014200020E030E040E251ECC701B6010F945B18B8
:1014300087FDE4CF012B11F38091F006882351F052
:101440001092EC061092ED061092EE061092EF0646
:101450001092F0062091360F3091370F4091380FDF
:101460005091390FC701B6010F94C0182B013C01F0
:101470006093E8067093E9068093EA069093EB0682
:101480002091EC063091ED064091EE065091EF066A
:10149000C701B6010F948E1C4B015C016093EC06F2
:1014A0007093ED068093EE069093EF062091320F35
:1014B0003091330F4091340F5091350F0F94C01875
:1014C0009B01AC016093E4067093E5068093E60609
:1014D0009093E706C301B2010F948E1C29813A81D3
:1014E0004B815C810F948D1C2B013C0120E030E08E
:1014F0004FE753E40F94B41E20E030E0A901181622
:10150000ACF4C701B6010F94B41E18166CF5A70110
:101510009601C501B4010F948D1C6093EC06709385
:10152000ED068093EE069093EF061EC0C301B20154
:101530000F945B1887FF22C020E030E0A901C701AB
:10154000B6010F945B1887FF16C0A7019601C5016D
:10155000B4010F948D1C6093EC067093ED0680939C
:10156000EE069093EF0607C0412C512C9FE7692EA1
:1015700093E4792E03C0412C512C3201C301B201F6
:101580000F900F900F900F90DF91CF911F910F91BF
:10159000FF90EF90DF90CF90BF90AF909F908F9093
:1015A0007F906F905F904F90089560915706709173
:1015B00058068091590690915A060895AF92BF92AD
:1015C000CF92DF92EF92FF920F931F93CF93DF930F
:1015D000CDB7DEB7A0970FB6F894DEBF0FBECDBF74
:1015E0006115710581059105B1F1B12CC42ED12C85
:1015F000E12CF12CAA24A394AB0C01E010E00C0F19
:101600001D1F0B0D111DB7FC1A95A70196010F9414
:10161000301CF8016083B901CA01611571058105AB
:10162000910511F41B2D12C0BA2CE4CFE1E0F0E0DB
:10163000EC0FFD1FE10FF11D17FDFA9580818A3037
:1016400040F490E3890F0E94AA4611501F3F71F7A2
:1016500015C097E3F7CF80E3A0960FB6F894DEBFEE
:101660000FBECDBFDF91CF911F910F91FF90EF90F3
:10167000DF90CF90BF90AF900C94AA46A0960FB683
:10168000F894DEBF0FBECDBFDF91CF911F910F91B8
:10169000FF90EF90DF90CF90BF90AF900895CF92E2
:1016A000DF92EF92FF926B017C0197FF0BC08DE2FE
:1016B0000E94AA46F094E094D094C094C11CD11C1E
:1016C000E11CF11C4AE0C701B601FF90EF90DF90EA
:1016D000CF9074CF0F931F93CF93DF938B01FC01B7
:1016E0008491EF012196882321F00E94AA46FE01F1
:1016F000F7CFB801882777FD8095982FDF91CF919C
:101700001F910F91CCCFCF92DF92EF92FF92CF93A8
:10171000DF936A017B01FC018491EF01219688230C
:1017200021F00E94AA46FE01F7CF4AE0C701B601A8
:10173000DF91CF91FF90EF90DF90CF903FCF8F92CE
:101740009F92AF92BF92CF92DF92EF92FF920F9350
:101750001F93CF93DF93CDB7DEB7CD54D1090FB62A
:10176000F894DEBF0FBECDBF1DAA1EAA1FAA18AED9
:1017700080E390E3A0E3B0E089AB9AABABABBCAB4A
:1017800021961FAE1EAE219784E690E025969FAF6E
:101790008EAF25971092CE069E01215C3F4F44E00C
:1017A00050E0BE016F5C7F4FCE018D5B9F4F0E946A
:1017B000746C25968EAD9FAD2597029625969FAFAA
:1017C0008EAF259721961FAE1EAE219781E02E96F3
:1017D0008FAF2E979E01215C3F4F41E050E0BE014C
:1017E000635B7F4FCE018D5B9F4F0E94746C9E01A7
:1017F000215C3F4F40E150E06CEA7FE0CE018D5B21
:101800009F4F0E94746C9E01215C3F4F40E150E06D
:101810006BE97FE0CE018D5B9F4F0E94746C9E014F
:10182000215C3F4F40E150E063E071E1CE018D5B10
:101830009F4F0E94746C9E01215C3F4F44E050E03A
:101840006BE171E1CE018D5B9F4F0E94746C9E0134
:10185000215C3F4F44E050E067E171E1CE018D5BD8
:101860009F4F0E94746C9E01215C3F4F44E050E00A
:1018700063E171E1CE018D5B9F4F0E94746C9E010C
:10188000215C3F4F44E050E067E97FE0CE018D5B93
:101890009F4F0E94746C9E01215C3F4F44E050E0DA
:1018A00063E97FE0CE018D5B9F4F0E94746C9E01C7
:1018B000215C3F4F44E050E060EE76E0CE018D5B6E
:1018C0009F4F0E94746C9E01215C3F4F40E150E0AD
:1018D00069EC7FE0CE018D5B9F4F0E94746C9E018E
:1018E000215C3F4F4CE050E069E577E0CE018D5B35
:1018F0009F4F0E94746C80E090E0A0E2B1E48DA75D
:101900009EA7AFA7B8AB9E01215C3F4F44E050E0DB
:10191000BE01635D7F4FCE018D5B9F4F0E94746C53
:101920002D961FAE2D971DAA1EAA1FAA18AE83E0E2
:101930002C968FAF2C972B968FAF2B979E01215C07
:101940003F4F41E050E0BE01645B7F4FCE018D5BB5
:101950009F4F0E94746C9E01215C3F4F44E050E019
:10196000BE016B5C7F4FCE018D5B9F4F0E94746CFC
:101970009E01215C3F4F41E050E0BE01655B7F4F1F
:10198000CE018D5B9F4F0E94746C9E01215C3F4F86
:1019900041E050E0BE01665B7F4FCE018D5B9F4F03
:1019A0000E94746C1AE0115071F09E01215C3F4F4F
:1019B00044E050E0BE016B5C7F4FCE018D5B9F4FDA
:1019C0000E94746CF0CF21960EAD1FAD2197259625
:1019D0008EAD9FAD259790936B0280936A029E0116
:1019E000215C3F4F44E050E069E179E0CE018D5B3E
:1019F0009F4F0E94746C21961FAF0EAF21979E01DE
:101A0000215C3F4F44E250E067EE71E1CE018D5B17
:101A10009F4F0E94746C83E02A968FAF2A97299675
:101A20008FAF299719A61AA61BA61CA61DA21EA237
:101A30001FA218A61DAA1EAA1FAA18AE9E01215CED
:101A40003F4F41E050E0BE01675B7F4FCE018D5BB1
:101A50009F4F0E94746C9E01215C3F4F41E050E01B
:101A6000BE01685B7F4FCE018D5B9F4F0E94746CFF
:101A70009E01215C3F4F44E050E0BE016B5D7F4F13
:101A8000CE018D5B9F4F0E94746C9E01215C3F4F85
:101A900044E050E0BE01675D7F4FCE018D5B9F4FFC
:101AA0000E94746C0AE010E0015011090115110543
:101AB00071F09E01215C3F4F44E050E0BE016B5C41
:101AC0007F4FCE018D5B9F4F0E94746CEDCF2896A7
:101AD0001FAE28971DAA1EAA1FAA18AE8FEF279621
:101AE0008FAF27979E01215C3F4F41E050E0BE0140
:101AF000695B7F4FCE018D5B9F4F0E94746C9E018E
:101B0000215C3F4F44E050E0BE016B5C7F4FCE0153
:101B10008D5B9F4F0E94746C9E01215C3F4F41E0A2
:101B200050E0BE016A5B7F4FCE018D5B9F4F0E94EC
:101B3000746C1DAA1EAA1FAA18AE1DE011509E01AA
:101B4000215C3F4F44E050E0112349F0BE016B5C43
:101B50007F4FCE018D5B9F4F0E94746CEFCF6CED79
:101B600076E0CE018D5B9F4F0E94746C9E01215CDC
:101B70003F4F44E050E068ED76E0CE018D5B9F4F33
:101B80000E94746C9E01215C3F4F44E050E064ED84
:101B900076E0CE018D5B9F4F0E94746CC12C80E873
:101BA000D82E8BE3E82E85E4F82E812C912C90E83A
:101BB000A92E9FE3B92E111136C09E01215C3F4F23
:101BC00044E050E066E37FE0CE018D5B9F4F0E94D2
:101BD000746C9E01215C3F4F44E050E062E37FE083
:101BE000CE018D5B9F4F0E94746C9E01215C3F4F24
:101BF00044E050E06EE27FE0CE018D5B9F4F0E949B
:101C0000746C8DAA9EAAAFAAB8AE9E01215C3F4F0C
